:020000040000FA
:107800005469616E59696E673130300000000000C4
:1078100054593230302E3038303030306200000071
:10782000424154333247313339474B3634464200B4
:1078300043414E5F5354440000000000000000002C
:1078400043414E5F43485F300000000000000000ED
:1078500043414E5F3530304B6270730000000000D2
:10786000E8070000E0070000DF070000000000005C
:020000040000FA
:10800000A8210020DD800000E5800000E78000005E
:108010000000000000000000000000000000000060
:10802000000000000000000000000000EF800000E1
:108030000000000000000000F3800000098401003F
:10804000B1050100F50501002506010055060100F6
:1080500085060100B5060100E506010015070100CF
:108060004507010075070100A9070100BD070100D0
:10807000CD070100010801001108010021080100DD
:108080005508010099080100E108010029090100D3
:1080900071090100B9090100C9090100FD090100C8
:1080A000310A0100610A0100950A0100C90A0100B4
:1080B000D90A0100E90A01001D0B0100510B010062
:1080C000EF3FE8FF0448854600F036F900480047D6
:1080D00075BC0100C046C046A82100201648804754
:1080E00016480047FEE7FEE7FEE7FEE7FEE7FEE78D
:1080F000FEE7FEE7FEE7FEE7FEE7FEE7FEE7FEE758
:10810000FEE7FEE7FEE7FEE7FEE7FEE7FEE7FEE747
:10811000FEE7FEE7FEE7FEE7FEE7FEE7FEE7FEE737
:10812000FEE7FEE7FEE7FEE7FEE7FEE7FEE7FEE727
:10813000FEE7FEE7FEE70000D9890100C5800000E8
:1081400030B50B46014600202022012409E00D46EF
:10815000D5409D4205D31D469540491B2546954077
:1081600040191546521E002DF1DC30BD70B50024BB
:108170002546002801DA01244042002901DA0125C0
:108180004942FFF7DDFFAC4200D04042002C00D056
:10819000494270BDF0B51FB40646002082B00546C6
:1081A0004024019100901BE0019922460F46304681
:1081B00000F0B1F8049A059B801A994110D310463B
:1081C0001946224600F097F8361A8F410197224649
:1081D00001200021009F00F08EF838184D410090DA
:1081E0002046641E0028DFDC019B009829463246A9
:1081F00007B0F0BDF0B51FB486B00020009001902C
:1082000002900698069980B204900798090C02041F
:108210000014114307900027089D099806913E46D7
:108220003C4603900398A9B20204000C0390049802
:108230002D0C154348430021224600F05CF8C71975
:10824000714110340E46402CECDB3846029A00F0A7
:1082500052F8009A019B80180090594102980191B0
:10826000103002904028CCDB00980BB0F0BD0346E4
:108270000B439B0703D009E008C9121F08C0042A5A
:10828000FAD203E00B780370401C491C521EF9D24D
:108290007047D2B201E00270401C491EFBD2704709
:1082A0000022F6E710B513460A4604461946FFF7C2
:1082B000F0FF204610BD30B504460020034600E024
:1082C0005B1C934203D2E05CCD5C401BF8D030BD18
:1082D0000321001D401E037812021A43491EF9D5DE
:1082E00010467047034603220870000A491C521EBC
:1082F000FAD51846704710B5202A04DB0146203A0B
:108300009140002010BD914020239C1A0346E34079
:108310001943904010BD10B5202A04DB0846203ACE
:10832000D040002110BD0B46D340D0402024A21ADB
:1083300091400843194610BD064C0125064E05E044
:10834000E36807CC2B430C3C98471034B442F7D376
:10835000FFF7BCFE88CD0100A8CD010070B58C18D8
:108360000578401C6B075B0F01D10378401C2A1174
:1083700006D10278401C03E006780E70401C491CB0
:108380005B1EF9D12B0705D40023521E0DD40B70B0
:10839000491CFAE70378401CCB1A921C03E01D78B5
:1083A0000D70491C5B1C521EF9D5A142D8D3002088
:1083B00070BD70B506F0B0FD0524204613F036FC04
:1083C0000025284606F09CFD204613F02FFC0126D0
:1083D000304606F071FD204613F028FC284606F0D2
:1083E0006BFD204613F022FC304606F089FD204646
:1083F00013F01CFC70BDB0B506F08EFD05242046C0
:1084000013F014FC0125284606F07AFD204613F0EF
:108410000DFC284606F050FD204613F007FC002016
:1084200006F04AFD204613F001FCB0BDF0B581B066
:1084300006F05EFD052013F0F9FB08270026012059
:1084400006F03AFD0524204613F0F0FB204613F019
:10845000EDFB06F043FD0546204613F0E7FB002048
:1084600006F02AFD204613F0E1FB76002E437F1E26
:108470003806E4D1F0B201B0F0BD70B5044600207A
:1084800006F01AFD06F048FD052013F0CFFB082684
:10849000E0B2C00906F034FD0525284613F0C6FBFE
:1084A000012006F009FD284613F0C0FB002006F06D
:1084B00003FD284613F0BAFB284613F0B7FB64000F
:1084C000761E3006E4D1052013F0B0FB012070BD0C
:1084D000F0B583B0019314460E4607460120384399
:1084E0000290032504E000F08EF86D1E280631D0BE
:1084F00000F067F83846FFF7C0FF00F0A7F8002843
:10850000F1D13046FFF7B9FF00F0A0F80028EAD11A
:1085100000F057F80298FFF7B0FF00F097F8002836
:10852000E1D1019802280BD3451E0026FFF77EFFFC
:108530002070FFF73EFF641C761CF0B28542F5DC2C
:10854000FFF774FF2070FFF756FF00F05CF8202063
:1085500003B0F0BD102003B0F0BDF0B583B01C46F1
:10856000009201910290032504E000F04CF86D1E8A
:10857000280623D000F025F80298FFF77EFF00F0D0
:1085800065F80028F1D10198FFF777FF00F05EF859
:108590000028EAD1002C0CD00026009F3878FFF785
:1085A0006CFF00F053F80028DFD1761C7F1CA64238
:1085B000F4D300F028F8082003B0F0BD102003B079
:1085C000F0BDB0B506F0A8FC0524204613F02EFB44
:1085D0000125284606F070FC204613F027FB2846AC
:1085E00006F08EFC204613F021FB0025284606F0FD
:1085F00087FC204613F01AFB284606F05DFC642039
:1086000013F014FBB0BDB0B506F086FC052420467F
:1086100013F00CFB0025284606F04EFC204613F014
:1086200005FB284606F06CFC204613F0FFFA0125F6
:10863000284606F041FC204613F0F8FA284606F0DA
:108640005FFC642013F0F2FAB0BD0000B0B506F094
:108650004FFC0524204613F0E9FA012006F02CFC1B
:10866000204613F0E3FA0B4D06F038FC044606F002
:108670001DFC002C02D06D1E2804F5D105252846CE
:1086800013F0D4FA002006F017FC284613F0CEFAB7
:108690002046B0BD33210000034801780B2901D8E2
:1086A000491C01707047C046971D002070B584B00A
:1086B0000025039502950195009506F0F7FB0F2024
:1086C000C6430E4C1036F1B2A0206A461023FFF7C5
:1086D00044FF204613F0AAFA204613F0A7FA912E81
:1086E000F0D3A020B0216A461023FFF736FF2046C2
:1086F00013F09CFA0248058004B070BD581B0000BE
:108700008A1D002070B5022902D2EB24E0B270BDB0
:10871000891EEB250022134605E0401C5B1CDDB2E0
:10872000A94225460EDB04786C40154604E0344629
:108730006E1C072D3546F0D26608E407F7D09A2460
:108740006640F4E7E0B270BDF0B591B00C914178AD
:1087500010AA117083781B025918C3780479240277
:10876000E3181B0459180B0ED3700C0C94700D0AEF
:1087700055700B9108956918099409190A93C9183D
:108780000278D2438918427983791B029A18C379F7
:10879000047A2402E3181B049A188918130A069312
:1087A000C918130C0593C9180792120E0492891860
:1087B000827AC37A1B029A18037B0F90447B2402AF
:1087C000E3181B0498180918020A02928918020C6F
:1087D000019289180D910390000E0E90002003461F
:1087E000014606E032409A40D2B211435B1C082B8E
:1087F0000ED0012635469D400746024602E07F1C0A
:10880000042FEFD010ACE45D2542F8D0521CF6E7FF
:108810000E9C0D980019C3B20F98827B934205D02D
:10882000427A914202D1002011B0F0BD1021FFF731
:1088300069FF0C99CC72019A8A72029A4A72039A61
:108840000A72049ACA71059A8A71069A4A71079A3D
:108850000A710A9ACA70099A8A70089A4A700B9A21
:108860000A7011B0F0BDF0B58DB05522027000272E
:1088700047720B784370CA79059202728A79049222
:10888000C2714A79039282710A7902924271CA7A5C
:10889000089242738A7A019202734E7AC6720C7AF7
:1088A00084720CAA13704D782D02EB188D78C9785C
:1088B000090249190904CB18190E01711D0CC57064
:1088C00009931B0A0B90837038460A91D170079563
:1088D00095700693537031020919089A1202019B90
:1088E000D21812045118089103990902029A8918A2
:1088F000059A1202049BD2181204511805913D46A4
:108900003A4605E02640AE4032436D1C082D0ED09D
:1089100001242146A9400346064602E05B1C042BC5
:10892000F0D00CAFFF5C3942F8D0761CF6E70B9B19
:108930005A72099806994018079940180A994018E0
:10894000059A8018110A4018110C4018110E401891
:10895000089A8018110A4018110C4018110E40187E
:108960005638987310211846FFF7CCFE0DB0F0BDB5
:10897000F0B58FB00446FF20E070A07060700F204B
:10898000C04302900F302070704813F04FF97049C7
:108990000868632801D8642008606E4F0020388082
:1089A0006D4E0190308008E00B99814222D33888C7
:1089B0001030388080B2A1286DD206F077FA39786D
:1089C000A02003AA1023FFF783FD30802028EED1DA
:1089D00003AD0BA92846FFF7B7FEE97B8842E6D135
:1089E00028785528E3D15D48017800290298DBD129
:1089F0000846D9E73888A0284DD8C0B20021019197
:108A000005E006F053FA3988C8B2A12943D2C1B2B1
:108A1000A02003AA1023FFF75BFD308039881031B6
:108A20003980202837D103AD07A92846FFF78CFEEF
:108A3000E97B8842E5D128785528E2D1474800787B
:108A40000028029900D1014607988842D9D24049AE
:108A50000A68962151430B9A824208D9081890421D
:108A600019D30BA90E222046FFF701FCC9E789188C
:108A7000814210D307A90E222046FFF7F8FB0BA86E
:108A80000A99818107980B9008980C9009980D908D
:108A900038880190B5E72078617809020818A17834
:108AA000E2781202511809040818401C24D1002051
:108AB00001903880A020B02103AA1023FFF708FD01
:108AC0003080202818D103AD0BA92846FFF73CFEC3
:108AD000E97B884210D1287855280DD11F480078AD
:108AE000002800D102900B980299884204D20BA969
:108AF0000E222046FFF7BBFB207861780902081898
:108B0000A178E2781202511809040818401C0CD10F
:108B10000020E072A07260722072E071A07160713A
:108B20002071E070A070607020700198388020780B
:108B3000617809020818A178E27812025118090434
:108B400008180749086030880FB0F0BD70110100A7
:108B5000841D00208A1D0020801D0020831D002010
:108B6000901D0020F0B581B00091064621480025F7
:108B70000570002A2ED01446C036631B71190F20D1
:108B800008401022101A834200D303461A48027884
:108B9000102A01D0042A1AD1C809FE2707405F2FE6
:108BA00013D80127B8436038C0B29E3282420CD33A
:108BB000009A5219C9B2DFB23B46FFF789FC0F4950
:108BC0000880ED19A542D8D304E0082000E0042075
:108BD0000A490880094801880020042902D0082990
:108BE00000D0012003490870411E8841400001B0B7
:108BF000F0BDC046961D0020821D0020941D00205F
:108C00000A4A012313700A4A10700A4A11600A4A7C
:108C100000211160042801D105218901102801D10A
:108C20001D208101054801807047C046831D00203A
:108C3000821D0020841D0020901D0020881D002022
:108C4000F0B587B0994D00262E80994B1B688B425A
:108C500024D1994C2188202925D102900092019697
:108C6000964C00272760964D964E2878062809D8FE
:108C700006F01CF92068401C2060B042F5D38D48F6
:108C8000042101802F70904C20880107029B31D075
:108C9000884820210180854D019E0BE00120400283
:108CA0008449088006E003A8FFF762FE208081481F
:108CB000802101807F4800883F2807DD874988425E
:108CC0000BDC402812D0802810D010E004280DD0F2
:108CD00008280AD0202809D009E001214A02904240
:108CE00004D0C902884201D001E002262E802888E3
:108CF00007B0F0BDA128019E00D32780009A012A69
:108D00006A4D1ED1187B012856D1DF719F715F71AA
:108D10001F711F73587B012804D1DF729F725F722D
:108D20001F725F7303AF38461946FFF79CFDF87357
:108D30002088002846D01038C1B2A02003AA1023F2
:108D400044E0002AB6D1614801780029B2D002700F
:108D500018785978090208189978DA7812025118A7
:108D6000090408185A490978002901D00F21C9437C
:108D7000884233D2274603AC20461946FFF773FDDD
:108D8000E0733978A02010232246FFF7E6FB029A11
:108D90004849088008288DD13888103038801078EC
:108DA0005178090208189178D278120251180904F2
:108DB0000818484908607DE7597B012911D101282D
:108DC000A3D0A7E7A02003AA10230146FFF7C5FB05
:108DD000384908803D48009901706BE70120C002C6
:108DE0005EE73D480078012812D103AC20461946C1
:108DF000FFF739FDE073A020B02110232246FFF7D2
:108E0000ACFB2C4908800828E4D133480770E1E71F
:108E100018785978090208189978DA7812025118E6
:108E2000090408182B490968214A12685118884218
:108E300003D2204840210180CCE725490978002948
:108E400001D00F21C94388422DD203AF38461946BD
:108E50001C46FFF708FDF8731B480178A02010237B
:108E60003A46FFF77AFB134908800828B2D1164921
:108E70000888103008802078617809020818A178E5
:108E8000E2781202511809040818124908600849CA
:108E90000A6815215143FFF753F900299AD101209F
:108EA0000D49087096E70120C00291E79C1D002043
:108EB000841D00209A1D0020801D0020A01D002080
:108EC000971D0020818D5B008A1D00208C1D0020D5
:108ED000831D0020901D0020981D0020FF01000030
:108EE000F0B585B00646434C002727800492101841
:108EF000414A1288904241D201910397404F00208D
:108F0000029038603F4C404D2078052809D805F084
:108F1000CDFF3868401C3860A842F5D3374804219B
:108F20000180029820703948018839480278102A57
:108F300001D0042A32D188190346C033049C651A33
:108F40000F2404401020001B854200DB0546DC098D
:108F5000603C01263002E7B27F09052F12D3B443EB
:108F6000E6B29E32B242234C039F0DD301984218C1
:108F7000D9B2EBB23046FFF7F0FA05E01F482021E6
:108F8000018011E01B4C039F1C49088008280BD16D
:108F9000E8B21E4A11880818108005E001208002FE
:108FA00016490880134C039F144800881F2809DDC8
:108FB000202813D001210A0290420FD08902884252
:108FC0000CD00CE0042809D0082808D10F480088EC
:108FD0000499884201D3022700E0012727802088D6
:108FE00002210143022902D1084900220A8005B06A
:108FF000F0BDC0469C1D0020881D00209A1D002049
:10900000A01D0020971D0020818D5B00A41D002065
:10901000821D0020F0B585B0044600200190042C8C
:109020006FD20AF06DFE002801D10AF0E9FE00209F
:10903000009000BF0098401C00900AF061FE039071
:109040000398002803D0484900988842F2D3039837
:10905000002856D1042145480AF034FE44484549C9
:1090600008802101444A515C4900404A505A414914
:109070000A880121090300F055F9029001200490AB
:1090800020013D4940184078002801D100264BE0DE
:109090002001394940184078012802D13548068816
:1090A00042E0200134494018407802282AD12001AA
:1090B000401805792901304A515C49002B4A505A21
:1090C0002C490A880121090300F02CF906462801E1
:1090D0002A494318280128494018028928014018C4
:1090E0000021C7683046B84706462801224BC01801
:1090F000C2882801C0188178304600F087F80646FB
:1091000012E02DE020011C4940184078032804D0CB
:10911000200140184078132804D120011649401836
:10912000868801E0002004900498002818D02001CF
:1091300012494318200110494018028920014018A3
:109140003146C7680298B847019020010A4BC01801
:10915000C2882001C0188178019800F057F801906A
:10916000019805B0F0BD000050C30000B60000201B
:1091700088130000B000002074C40100B4C40100D2
:10918000F8B505460E4614460020009001211C4803
:1091900001751C48007888431A4908700846807891
:1091A0000821084317498870002088710846007814
:1091B000012108431349087008460572002717E08B
:1091C00010480078802108430E49087000BF0E48FF
:1091D000007D0028FBD000200B4908750948C08994
:1091E0002080A41C0748C1890098081800907F1CA3
:1091F000B742E5D331460098FEF7A2FF80B2F8BD32
:1092000040610040005004404060004010B50346FB
:10921000012908D1094CA41A9C4202D99C18A0B279
:109220000BE0064809E0022906D1934202DD9C1AB0
:10923000A0B202E0002000E0184610BDFFFF0000D1
:1092400010B504460121202001F0B2FF0020324970
:109250000870012131480175002031490875152039
:1092600012F0CCF92C488078E17808432A498870BC
:10927000084680782178084327498870207880281C
:1092800006D108460079E17949000843224908716E
:1092900021488078E17A08431F498870A078002827
:1092A00003D10846007908710FE0A078012806D1A3
:1092B00019480079602108431749087105E01648EC
:1092C0000079802108431449087113488079217975
:1092D00008431149887108468079617908430E492D
:1092E0008871207AC872607A8872084600783821BE
:1092F000884309490870084600786178C900084326
:1093000005490870A07A08730846007801210843CF
:109310000149087010BD0000005004404061004049
:1093200040600040F8B504460E461746002E01D1B5
:1093300000250FE0A64201DC3D460BE00094009CB6
:1093400020467843009031460098FEF7F9FE0090E1
:10935000009885B22846F8BD0146042904D28A0047
:10936000024BD218508800E000207047A817002058
:109370000146042903D28A00024B985C00E00020D9
:1093800070470000A8170020FFB587B00446089872
:10939000844203DA0A988068002802D124480190A8
:1093A00042E00898001B82B20292002625460A98E5
:1093B000806800212F463A46334604960591069070
:1093C000FEF718FF05460E46002328463146029A4E
:1093D000FEF7E0FE05460E46304600210A464940AB
:1093E0005040014302D0124801901DE003950A98B5
:1093F000C068039DA84202D30020019014E00A989F
:10940000C1680398401A039009990398FEF798FEE3
:1094100003900398000C0004002802D00448019037
:1094200002E0039880B2019001980BB0F0BD0000FB
:10943000FFFF000010B508480078802188430649E6
:10944000087001210548017500200549087515209F
:1094500012F0D4F810BD00000050044040610040FC
:1094600040600040F8B505460E4614461F462146AA
:109470002846FEF77BFE80B2F8BD0000FFB587B03E
:1094800006460A984068002801D1029035E00A9803
:1094900001684068081803900025344600212746DB
:1094A000039806950491059038462946049B059A31
:1094B000FEF7A0FE04460D460A98406802460023C7
:1094C000019020462946FEF765FE04460D4600231E
:1094D00020462946099AFEF75DFE04460D462846B9
:1094E00007492140002359405840014303D0044814
:1094F000C043029001E0A0B2029002980BB0F0BD10
:109500000000FFFF10B5FE4800688079030012F0EC
:109510005BF807059ED8F5F4F3F2F100F84800680F
:109520004079030012F050F80805138A2A8A468A07
:10953000638A0EF0A1FE0020F1490968C873F04863
:1095400000684079401CEE49096848717DE0ED49AA
:109550004969EB4A1268D27A885C0EF005FFE84848
:1095600000684079401CE64909684871E448006891
:109570004079401CE2490968487166E009F054F9F5
:10958000002810D10EF0F0FEDD4800684079401C44
:10959000DB4909684871DA4800684079401CD849BD
:1095A0000968487105E00EF091FE0020D449096871
:1095B00048714AE009F038F9002811D111200EF065
:1095C000D3FECF4800684079401CCD4909684871F6
:1095D000CB4800684079401CC9490968487105E0DA
:1095E0000EF074FE0020C649096848712DE009F0AC
:1095F0001BF900281BD1C2480068C07A401CC04932
:109600000968C872BE480068C07ABE4909788842B5
:109610000DDB0020BA490968C872B9490968486277
:10962000B74800688079401CB549096888710EF018
:109630004DFE0020B2490968487106E00EF046FE72
:109640000020AF490968487100BF00BF32E3AC4851
:109650000068407C002817D0AA48C068002803D0C2
:10966000A848C168192088470020A54909684862B0
:10967000A34800688079401CA149096888710020CE
:109680009F49096848711BE09D480068406A282886
:1096900007D29B480068406A401C994909684862A3
:1096A0000EE0002096490968486295480068807974
:1096B000401C9349096888710020914909684871E4
:1096C000F8E28F4800684079030011F07DFF08053B
:1096D00018A42FA44CA480A40EF0CEFD002088492D
:1096E0000968C873864800684079401C8449096845
:1096F000487197E0D4E2C7E230E25DE194E081494D
:1097000049697F4A1268D27A885C0EF02DFE7C4847
:1097100000684079401C7A490968487178480068B7
:109720004079401C7649096848717BE009F07CF873
:10973000002811D101200EF017FE71480068407911
:10974000401C6F49096848716D4800684079401CA9
:109750006B490968487105E00EF0B8FD00206849C2
:10976000096848715EE009F05FF8002828D1644973
:109770000968C97A24225143634A12688918604AE9
:109780001268D27B885C0EF0EFFD5D480068C07BFC
:10979000401C5B490968C87359480068C07B24288D
:1097A00014D3574800684079401C554909684871EE
:1097B000534800684079401C51490968487105E0E8
:1097C0000EF084FD00204E49096848712AE009F036
:1097D0002BF8002818D14A480068C07A401C484934
:1097E0000968C87246480068C07A464909788842C4
:1097F0000ADB002042490968C87241480068807944
:10980000401C3F49096888710EF060FD00203C490A
:109810000968487106E00EF059FD002038490968D2
:10982000487100BF00BF45E2354800684079030039
:1098300011F0CAFE0A0614B92BB948B978B995B91E
:109840000EF01AFD00202E490968C8732C480068E4
:109850004079401C2A4909684871ABE029494969A7
:10986000274A1268D27A885C0EF07EFD2448006890
:109870004079401C224909684871214800684079B4
:10988000401C1F490968487194E008F0CDFF00288A
:1098900011D14A200EF068FD194800684079401C3B
:1098A000174909684871164800684079401C1449F6
:1098B0000968487105E00EF009FD002010490968AB
:1098C000487177E008F0B0FF002824D1FF200EF0A7
:1098D0004BFD0B480068C07B401C09490968C873F0
:1098E00007480068C07B24281BD3054800684079DE
:1098F000401C03490968487101480068407905E047
:109900006C070020681D002068070020401CEA4901
:109910000968487105E00EF0D9FC0020E6490968A5
:10992000487147E008F080FF002811D1FF200EF0B9
:109930001BFDE14800684079401CDF490968487117
:10994000DD4800684079401CDB490968487105E042
:109950000EF0BCFC0020D849096848712AE008F0E4
:1099600063FF002818D1D4480068C07A401CD2494F
:109970000968C872D0480068C07AD049097888421E
:109980000ADB0020CC490968C872CB48006880799E
:10999000401CC949096888710EF098FC0020C6492E
:1099A0000968487106E00EF091FC0020C249096880
:1099B000487100BF00BF7DE1BF48006840790300E7
:1099C00011F002FE0C0715C32CC349C366C382C342
:1099D0009FC30EF051FC0020B7490968C873B64810
:1099E00000684079401CB44909684871B4E0B34943
:1099F0004969B14A1268D27A885C0EF0B5FCAE486B
:109A000000684079401CAC4909684871AA48006860
:109A10004079401CA849096848719DE008F004FF9E
:109A2000002811D177200EF09FFCA34800684079F0
:109A3000401CA149096848719F4800684079401C52
:109A40009D490968487105E00EF040FC00209A49E4
:109A50000968487180E008F0E7FE002811D10C2069
:109A60000EF082FC944800684079401C92490968D5
:109A70004871914800684079401C8F4909684871D5
:109A800005E00EF023FC00208B490968487163E073
:109A900008F0CAFE002810D10EF066FC8648006867
:109AA0004079401C844909684871834800684079BE
:109AB000401C81490968487105E00EF007FC002050
:109AC0007D490968487147E008F0AEFE002811D1D1
:109AD00013200EF049FC784800684079401C764914
:109AE00009684871744800684079401C72490968E7
:109AF000487105E00EF0EAFB00206F4909684871E3
:109B00002AE008F091FE002818D16B480068C07A5E
:109B1000401C69490968C87267480068C07A67498B
:109B2000097888420ADB002063490968C8726248E4
:109B300000688079401C6049096888710EF0C6FB96
:109B400000205D490968487106E00EF0BFFB002067
:109B500059490968487100BF00BFABE0564800682A
:109B60004079030011F030FD080513872A874787E5
:109B700063870EF081FB00204F490968C8734E4887
:109B800000684079401C4C49096848717AE04B49AB
:109B90004969494A1268D27A885C0EF0E5FB46486A
:109BA00000684079401C444909684871424800688F
:109BB0004079401C40490968487163E008F034FE70
:109BC000002811D149200EF0CFFB3B4800684079B6
:109BD000401C394909684871374800684079401C81
:109BE00035490968487105E00EF070FB00203249E4
:109BF0000968487146E008F017FE002810D10EF001
:109C0000B3FB2D4800684079401C2B490968487116
:109C1000294800684079401C27490968487105E0D7
:109C20000EF054FB00202449096848712AE008F02E
:109C3000FBFD002818D120480068C07A401C1E494E
:109C40000968C8721C480068C07A1C4909788842B3
:109C50000ADB002018490968C87217480068807933
:109C6000401C1549096888710EF030FB002012492C
:109C70000968487106E00EF029FB00200E490968CA
:109C8000487100BF00BF15E000200B4909688871CA
:109C9000094909684871062007490968C87009E040
:109CA0000EF014FB00200449096848710249096854
:109CB000887100BF00BF10BD6C070020681D002028
:109CC00010B56A4800684079030011F07DFC090670
:109CD00010C627C644C6608EC6000EF0CDFA634893
:109CE00000684079401C614909684871BCE06049DE
:109CF00049695E4A1268D27A885C0EF035FB5B488F
:109D000000684079401C5949096848715748006803
:109D10004079401C554909684871A5E008F084FD68
:109D2000002811D17F200EF01FFB504800684079B9
:109D3000401C4E49096848714C4800684079401CF5
:109D40004A490968487105E00EF0C0FA0020474909
:109D50000968487188E008F067FD002810D10EF00E
:109D600003FB424800684079401C4049096848713B
:109D70003E4800684079401C3C490968487105E04C
:109D80000EF0A4FA00203949096848716CE008F027
:109D90004BFD002822D135480068C07A401C334969
:109DA0000968C87231480068C07A31490978884228
:109DB0000FDB00202D490968C8722C4800684079E3
:109DC000401C2A49096848710020284909684862EE
:109DD00008E0002025490968487103E00020234974
:109DE000096848710EF072FA3EE020480068407C35
:109DF000002816D01E48C068002803D01C48C1683F
:109E000019208847002019490968486217490968DC
:109E10004871164909688871052014490968C87095
:109E20001AE012480068406A282807D20F480068E4
:109E3000406A401C0D49096848620DE000200B494A
:109E400009684862094909684871084909688871C0
:109E5000052006490968C87006E00EF037FA0020B0
:109E600002490968487100BF00BF10BD6C0700209F
:109E7000681D002010B50024F7480068807A01288A
:109E80007ED1F5480068C07900287AD0F248006891
:109E90008079002804D0012874D0022873D191E180
:109EA000ED480068007B24286ED2EB480068C0793A
:109EB00001287AD1002475E0E7480068C07A24219F
:109EC0004843E64909684018E3490968097B415C51
:109ED000E1480068C07A24225043E14A12688018A1
:109EE000DD4A1268127B805C814229D0DA48006822
:109EF000C07A24214843DA4909684018D6490968DC
:109F0000097B415CD4480068C07A24225043D34A7C
:109F100012688018D04A1268127B8154CE480068BB
:109F2000407B242805D3CC480068007BCA490968D7
:109F30004873C9480068007BC7490968887308E00E
:109F4000C5480068407B242803D20120C249096823
:109F50008871C1480068007B401CBF4909680873CC
:109F6000BD480068007B242808D3BB480068407BBC
:109F7000242803D20120B84909688871B64805E051
:109F8000D3E1CDE169E0BAE138E00EE00068007BA2
:109F9000242804D2B04800688079012800D103E069
:109FA000601CC4B2242C87D356E0002413E0AA48D6
:109FB0000068C07A24214843A94909684018015D16
:109FC000A5480068C07A24225043A44A1268801829
:109FD0000155601CC4B2242CE9D300209E490968B5
:109FE000487323209C490968887301209A490968AD
:109FF000887124209849096808732DE0002096494B
:10A000000968087394480068C07A401C924909683E
:10A01000C87291480068C07A92490978884217DB73
:10A020008D480068007C012804D102208A49096813
:10A03000887106E0002088490968887186490968A6
:10A04000C871002084490968C87283490968087486
:10A05000002081490968487161E17F4800684079C2
:10A06000030011F0B1FA080513A62AA651A68EA680
:10A0700001207949096808740EF0FEF876480068F6
:10A080004079401C74490968487199E075494969EB
:10A09000714A1268D27A885C0EF066F96E480068E0
:10A0A0004079401C6C49096848716B4800684079E8
:10A0B000401C69490968487182E008F0B5FB002836
:10A0C0001BD165490968497B491CC8B20EF04CF99F
:10A0D00061480068407B60490968C8735E48006851
:10A0E0004079401C5C49096848715B4800684079C8
:10A0F000401C59490968487105E00EF0E7F8002056
:10A100005549096848715BE008F08EFB00282BD1A7
:10A1100051490968C97A24225143504A1268891862
:10A120004D4A1268D27B885C0EF01EF94A480068DE
:10A13000C07B401C48490968C87347480068C07B19
:10A1400045490968897B88421ADD4348006840799F
:10A15000401C4149096848713F4800684079401CEB
:10A160003D49096848710BE00EF0B0F83A480068C4
:10A17000407B39490968C87300203749096848712C
:10A180001EE008F051FB00280CD1334909688871A2
:10A19000242031490968C8732F49096848732E493A
:10A1A000096888730EF092F800202B4909684871FD
:10A1B00006E00EF08BF8002027490968487100BFBF
:10A1C00000BFACE0244800684079030011F0FCF9BE
:10A1D00008050F8E268E4C8E688E0EF04DF81E48A8
:10A1E00000684079401C1C490968487185E01D4998
:10A1F0004969194A1268D27A885C0EF0B5F8164897
:10A2000000684079401C1449096848711248006888
:10A210004079401C1049096848716EE008F004FB61
:10A22000002811D149200EF09FF80B4800684079B2
:10A23000401C094909684871074800684079401C7A
:10A2400005490968487105E00EF040F80020024910
:10A250000968487151E000006C0700206807002081
:10A2600064070020681D002008F0DEFA002810D1E5
:10A270000EF07AF89C4800684079401C9A490968B9
:10A280004871994800684079401C974909684871AD
:10A2900005E00EF01BF800209349096848712CE096
:10A2A00008F0C2FA00281AD18F480068C07A401C12
:10A2B0008D490968C8728C480068C07A8B49097852
:10A2C00088420CDB002088490968C8728649096801
:10A2D000887185490968487183490968C8710DF01A
:10A2E000F5FF002080490968487106E00DF0EEFF97
:10A2F00000207D490968487100BF00BF0FE00DF0E4
:10A30000E5FF002078490968487177490968887134
:10A3100075490968087374490968C87200BFE2E0AA
:10A320000020714909688872DDE06F480068807A12
:10A330000228F4D16C480068007A002879D06A4875
:10A3400000684079030011F03FF90B0711BB25BBF2
:10A3500041545EBB7590BB000DF08EFF62480068F3
:10A360004079401C604909684871B7E05F49496914
:10A3700008780DF0F9FF5C4800684079401C5A49A4
:10A3800009684871584800684079401C5649096876
:10A390004871A3E008F048FA002810D10DF0E4FF5E
:10A3A000514800684079401C4F49096848714E483F
:10A3B00000684079401C4C490968487105E00DF07F
:10A3C00085FF002048490968487187E008F02CFAA9
:10A3D000002807D1444800684079401C4249096878
:10A3E000487103E000204049096848710DF06EFF94
:10A3F00074E00DF041FF3C4800684079401C3A4948
:10A40000096848716AE0394949690978491CC8B244
:10A410000DF0AAFF344800684079401C32490968B1
:10A420004871314800684079401C2F4909684871DB
:10A4300054E054E008F0F8F900280FD10DF0EEFEDA
:10A4400029490968887001200DF062FF26480068DC
:10A450004079401C24490968487105E00DF036FF39
:10A46000002021490968487138E01F480068807859
:10A4700011280CD100201C4909680872AA201A4929
:10A4800009688870002018490968487011E016486A
:10A4900000684078401C14490968487012480068F8
:10A4A0004078032805D308F05FFA00200E490968B8
:10A4B00048700DF00BFF00200B49096848710DE052
:10A4C0000DF004FF00200849096848710649096831
:10A4D0004870AA2004490968887000BF03E0002082
:10A4E00001490968887210BD6C070020681D0020B2
:10A4F00070B5002508E06D1C1B48854202D209F0AA
:10A50000ABFC01E0002503E009F0FAFB0028F2D1E2
:10A5100000BF0221002009F001FC0321002009F006
:10A52000FDFB0521002009F0F9FB0721002009F0BF
:10A53000F5FB002408E00020A1000C4A5054A100C3
:10A5400089184880601CC4B2042CF4D30120084947
:10A55000087000204870052088700020C8700548E9
:10A560000549088070BD000050C30000A8170020F6
:10A57000B200002088130000B0000020F8B58D481C
:10A580000078030011F020F8060405163D5EFDFC7E
:10A590000EE109F035FC00208649C8704870084675
:10A5A0008078002802D10320087002E0022081494F
:10A5B0000870FDE07F488078002804D07D488078CE
:10A5C000401E7C49887009F09BFB00280BD109F0E4
:10A5D00017FC00207749C8700846807800280FD102
:10A5E000032008700CE07348C078401C7149C870A3
:10A5F0000846C078052803D30520087009F02CFC14
:10A60000D6E009F07DFB00280ED104216A4809F04C
:10A6100059FB00206749C87048706848684908803D
:10A620000420644908700CE06248C078401C61490D
:10A63000C8700846C078052803D30520087009F0C3
:10A640000BFCB5E05B49497809015E4A515C490061
:10A65000594A505A5A490A8801210903FEF762FEF5
:10A660000090012553484078000156494018407831
:10A67000002801D100243CE04E48407800015149B7
:10A6800040184078012802D14D48048831E04948FB
:10A69000407800014B4940184078022812D14549C2
:10A6A00049780901474A89180879FEF755FE04469A
:10A6B000404949780901434A89180879FEF758FE4C
:10A6C000054616E03B48407800013E494018407876
:10A6D000032806D0374840780001401840781328F6
:10A6E00006D134484078000136494018848800E09B
:10A6F0000025002D2FD02F48407800013249431803
:10A700002C48407800012F49401802892948407898
:10A71000000140182146C7680098B84706462548FA
:10A7200040780001274BC018C288224840780001B9
:10A73000C01881783046FEF769FD06461D4840780E
:10A74000800022494018468001201A494978890032
:10A750001E4A50540AE000201649497889001B4AD5
:10A760008918488013494978890050541148407825
:10A77000401C1049487008464078042809D301E07D
:10A7800013E007E009F03CFB00200A494870032071
:10A7900008700DE009F0B4FA002803D10120054942
:10A7A000087001E009F058FB02E0FFF7A1FE00BFCE
:10A7B00000BFF8BDB2000020B600002088130000E2
:10A7C000B000002074C40100B4C40100A817002028
:10A7D00010B509F05FFA002405E00020A100074A47
:10A7E0005054601CC4B2042CF7D3002004490870F4
:10A7F0000520887003480449088010BDA817002070
:10A80000B200002088130000B000002070B504469C
:10A81000002000F0AFF8002000F0DAF8002000F08F
:10A820009BF8002000F0C4F8002000F087F800201A
:10A8300000F0AEF800BF012000F08EF8012000F01B
:10A84000B7F8002521E0002000F086F8002000F095
:10A85000AFF880202040002806D0012000F08AF8C0
:10A86000012000F0B5F805E0002000F083F800209A
:10A8700000F0AEF800BF012000F06EF8012000F0FB
:10A8800097F86006040E681CC5B2082DDBDB0120BA
:10A8900000F054F8012000F07BF870BD70B504465C
:10A8A0000D46012000F066F8012000F091F800202C
:10A8B00000F052F8002000F07BF8002000F03EF895
:10A8C000002000F065F800BF012000F045F80120ED
:10A8D00000F06EF8002628E0002000F03DF800208F
:10A8E00000F066F880202040002803D0012000F00E
:10A8F00041F802E0002000F03DF8802028400028C8
:10A9000003D0012000F064F802E0002000F060F8BD
:10A9100000BF012000F020F8012000F049F8600697
:10A92000040E6806050E701CC6B2082ED4DB01208A
:10A9300000F004F8012000F02BF870BD10B50446BB
:10A94000002C04D08121032009F00EFB03E08021BC
:10A95000032009F009FB10BD10B50446002C04D0FB
:10A960008121042009F000FB03E08021042009F08C
:10A97000FBFA10BD10B50446002C04D08121022042
:10A9800009F0F2FA03E08021022009F0EDFA10BD8F
:10A9900010B50446002C04D08121044809F0E4FAE3
:10A9A00003E08021014809F0DFFA10BD0107000033
:10A9B00010B50446002C05D081210720000209F0C3
:10A9C000D3FA04E080210720000209F0CDFA10BD7F
:10A9D00010B50446002C04D08121044809F0C4FAC3
:10A9E00003E08021014809F0BFFA10BD0207000012
:10A9F00010B5F920FFF70AFF8820FFF707FF902026
:10AA0000FFF704FF9820FFF701FF08210846FFF732
:10AA100045FFE820FFF7FAFE12210846FFF73EFF48
:10AA2000A020FFF7F3FE70210846FFF737FFA820AC
:10AA3000FFF7ECFE70210846FFF730FFB020FFF76C
:10AA4000E5FE70210846FFF729FFB820FFF7DEFE7C
:10AA500000210846FFF722FFC020FFF7D7FE0021A4
:10AA60000846FFF71BFFC820FFF7D0FE002108466D
:10AA7000FFF714FFD020FFF7C9FE2F210846FFF78C
:10AA80000DFFD820FFF7C2FE2F210846FFF706FF73
:10AA9000E020FFF7BBFE2F210846FFF7FFFE402016
:10AAA000FFF7B4FE00210846FFF7F8FE0A20FFF783
:10AAB000ADFE002405E000210846FFF7EFFE601C14
:10AAC000C4B25A2CF7DB00240AE000200B490855D9
:10AAD0000B4908550B4908550B490855601CC4B271
:10AAE0005A2CF2DB8120FFF791FE00200749087005
:10AAF0008870C8700871487010BD0000E81400200C
:10AB0000421500209C150020F61500207D00002035
:10AB100010B58020FFF77AFE10BD00000020044928
:10AB20000870012003490870002048707047000039
:10AB3000820000207D00002010B5484800780028E1
:10AB40007AD046488078030010F03EFD0604434A60
:10AB5000535A687E414800794149085C3F49097968
:10AB6000404A515C884209D13C4800793E49085C22
:10AB70003A4909793D4A515C88421BD037480079EF
:10AB80003749085C35490979364A505433480079C9
:10AB90003549085C31490979344A50542F48C07806
:10ABA000002803D004202D49887011E001202B4992
:10ABB00088700DE000202949C87008460079401CC3
:10ABC0000871084600795A2802DB002008710870D5
:10ABD00041E04020FFF71AFE0220204988703AE049
:10ABE0001E4A11791079FFF759FE03201B4988701E
:10ABF00031E00A20FFF70AFE0420184988702AE095
:10AC0000164A1279194B995C144A1279154B985CC3
:10AC1000FFF744FE0520114988701CE00F480079B9
:10AC2000401C0E490871084600795A2805DB0020AF
:10AC300008710870C87003E00EE001200749C87071
:10AC400000200649887006E00020044908708870DA
:10AC5000C870087100BF00BF10BD00007D0000205B
:10AC6000E8140020421500209C150020F615002055
:10AC700010B50DF01FFF012811D10E4800780528EE
:10AC800006D1FF22A532002101200FF093FB0FE037
:10AC90004B22D200002101200FF08CFB08E00020A5
:10ACA0000549888048800022114601200FF082FB70
:10ACB00010BD0000CA0000201A00002058221152C6
:10ACC000704710B504460121022000F071FA0021FE
:10ACD000022000F06DFA10BD014600205322525CA4
:10ACE00010231A40002A08D05322525C0C231A4029
:10ACF0009210032A18D1032016E05422525A01233D
:10AD0000DB031A40002A0ED05322525C0C231A4057
:10AD10009210032A05D05322525C9207920F032A05
:10AD200001D1022000E00120704702460020582394
:10AD30009B5A0B40002B01D0012000E000207047FF
:10AD4000014600226020405AFF231B0218400005E4
:10AD5000020F1001014BC01870470000005504405D
:10AD600010B5002A0AD056231B5A0C02234356243E
:10AD7000235256231B5A8B43235209E056231B5A56
:10AD80000C02A3435624235256231B5A0B4323522F
:10AD900010BD0000F8B504460D46012700263448D2
:10ADA000844203D10121022000F002FA2878401EDB
:10ADB000A0702088FF2101310843208020884008AE
:10ADC00040002080A878401EC1B25A200155687901
:10ADD0000007000CE97909020843A97908435C21BE
:10ADE0000853288981B240200153A868C000C10CD3
:10ADF00042200153A88981B244200153E868C00071
:10AE0000C10C46200153288A81B248200153286989
:10AE1000C000C10C4A200153A88A81B24C200153C2
:10AE20006869C000C10C4E2001535020005B297995
:10AE300009020843502108535020005B29798843B8
:10AE40005021085300E0761C5020005B4007400F63
:10AE50002979884202D007488642F4D15020005B0D
:10AE60004007400F2979884200D000273846F8BDB6
:10AE700000540440FFFF000030B5034600201C8949
:10AE80008C4209DD082A05D218244C431D682C1970
:10AE9000A05C02E0002000E0002030BD10B50246BA
:10AEA00013898B4205DD18234B431468E318987C03
:10AEB00000E0002010BD0146FF22C889C007C00F76
:10AEC00000280AD00120C88100E0521EC889C007AE
:10AED000C00F002801D0002AF7D1C889C007C00FD1
:10AEE00000280FD10220C8810420C881487A400878
:10AEF00040004872487A38239843487200204872CC
:10AF0000012070470020FCE70246507A01231843D5
:10AF10005072507A0B78DB0018435072087A01287F
:10AF200008D1888850814868000C0123DB0318434E
:10AF3000908108E0087A002805D150814868800097
:10AF40001A4B18409081487A012804D1507A402346
:10AF50001843507206E0487A002803D1507A402303
:10AF6000984350720878002811D1C87A1072087B73
:10AF70001070487B5070887B9070CB7BD370087CBE
:10AF800010714B7C5371887C9071CB7CD371887A23
:10AF9000002803D00120C002D08101E00820D08128
:10AFA000FF200130D081012070470000FC1F00000D
:10AFB000002904D0427A80231A43427203E0427A85
:10AFC00080239A434272704730B5024600200F4BEF
:10AFD0005024A45A0D022C435025AC525024A45A9C
:10AFE0008C43AC5200E05B1E5024A45A6407640FEB
:10AFF0008C4201D0002BF6D15024A45A6407640F70
:10B00000002C01D0002000E0012030BDFFFF000037
:10B01000827A80231A40802A00D081727047000013
:10B0200070B5044600250023002D02D001266020C3
:10B0300006530420C88188890126F6033040002881
:10B0400008D0012010728889C004C0084E8930439E
:10B05000506006E00020107288890F4E304080104A
:10B060005060087AD072002304E0CE5C10460C30A9
:10B07000C6545B1CD07A9842F7DCC889042630405D
:10B08000002804D1C889F6023040002801D00020F1
:10B0900070BDD07AFCE70000FC1F0000027C80231A
:10B0A0001A40802A00D00174704710B50246FF2371
:10B0B000D089C007C00F00280AD00120D08100E04D
:10B0C0005B1ED089C007C00F002801D0002BF7D12C
:10B0D000D089C007C00F002801D0002010BD507AD1
:10B0E000012420435072507A3824A0435072C87A09
:10B0F0001072487A00280FD1087B1070487B50707E
:10B10000887B9070CC7BD470087C10714C7C54711F
:10B11000887C9071CC7CD471FF200130D0814000BC
:10B12000D081107ADAE70000F8B504460D46002019
:10B13000002C00D100BF002A00D100BF012C01D19A
:10B1400041263043012A01D112263043022C01D17D
:10B15000C0263043022A01D130263043134E3070CE
:10B1600076788027BE43114F7E70012C08D1FF21D5
:10B1700000BF0E4EB3781E460E4033468B42F8D1C8
:10B180000A4E76784027BE43084F7E70012A0BD1C5
:10B190000026009603E000BF009E761C0096FF2765
:10B1A0006937009EBE42F6D9F8BD00000004024097
:10B1B000002905D0054A12780243044B1A7004E0B6
:10B1C000024A12788243014B1A70704720040240F1
:10B1D000002905D0054A927E0243044B9A7604E08A
:10B1E000024A927E8243014B9A76704700080240E1
:10B1F00001200649087000BF0448007880210840FB
:10B200000028F9D00120024908707047000C024064
:10B210000C01002070B5034614460020002B01D11C
:10B22000C0B202E005468035E8B2012902D1051D11
:10B23000E8B206E0022903D105460835E8B200E08D
:10B24000C0B2012C02D1851CE8B200E0C0B2084DAA
:10B25000A870AD7801263543054EB570002201E097
:10B2600000BF521C7D252D01AA42F9D970BD0000F6
:10B27000000C024070B500242448007920210840C9
:10B28000002801D0224D3FE000F046F80546214855
:10B29000007880210840002836D01E488078084079
:10B2A000002801D01A4D02E000F036F80546194892
:10B2B00080780007840F022C01DBAD0804E0012C2C
:10B2C00001D16D0800E000BF124880788007C00FF0
:10B2D000002801D02D0101E00C2045430D480078E5
:10B2E0004007840F002C02D1601CC4B207E0032C7D
:10B2F00003D1601C4006040E01E06006040E2146E6
:10B300002846FCF71DFF0546284670BD0004024094
:10B3100000127A00000C024000B5C0229178F82299
:10B3200011401C4A12781143EA2923D00ADC0A464C
:10B33000E03A130010F048F90A181C20242A2A2A9F
:10B340002A161A2AED291FD004DCEB2916D0EC2985
:10B350001CD117E0F02903D0F82917D10E4817E0C7
:10B360000E4815E00E4813E00E4811E00E480FE0BD
:10B370000E480DE00E480BE00E4809E00E4807E0CD
:10B380000E4805E00E4803E00E4801E00D4800BFFE
:10B3900000BF00BD201C02400090D003006CDC0206
:10B3A0000048E80100366E010024F400001BB700DD
:10B3B00000127A00808D5B0000093D00C0C62D00A0
:10B3C00080841E0040420F0010B50446204600F065
:10B3D0001DFD002010BD000010B590211348FCF7A2
:10B3E0005FFF124812490860124848600620088131
:10B3F0000020887206220F490D4800F04BFA002108
:10B400000B48FFF705FE80210B48FCF749FF0A486F
:10B410000A4948600A4B04220A49084800F08AFB9E
:10B4200055210648FFF73AFE10BD0000E407002052
:10B43000C4070020E4C2010074080020D0070020E7
:10B44000C9B3000074C201000C4A127812060B4BFB
:10B450005B781B041A43094B9B781B021A43074B6A
:10B46000DB781A43104642084240D20083085A4013
:10B470001146034A5140034A116070478306002079
:10B480000102000088060020F8B504460F46A07AA5
:10B490004006400E002874D10025ACE01820684317
:10B4A00021680818407C01283CD1012118206843FC
:10B4B00022681018017400260CE0182068432168E7
:10B4C00008180830815D18206843226810188155DB
:10B4D000701CC6B2082EF0D30021182068432268E1
:10B4E000101801741820684322681018417418203D
:10B4F00068432268101841611820684322681018B8
:10B5000081742C20684361680818406A002809D0BB
:10B5100018236B432268D0182C236B436268D2181F
:10B52000516A884718206843216808184069FF213C
:10B53000C94388425DD818206843216808184069CB
:10B54000C119182068432268101841611820684307
:10B550002168081841692C206843626810188069C6
:10B56000814246D31820684321680818807C5528FA
:10B570003FD0552118206843226810188174002696
:10B5800024E03CE01820684321680818805D2C21E5
:10B590006943626851181031895D08401821694378
:10B5A0002268511888551820684321680818805D62
:10B5B0002C216943626851180831895D08431821BC
:10B5C0006943226851188855701CC6B2082ED9D319
:10B5D0002C20684361680818806A002809D0182365
:10B5E0006B432268D0182C236B436268D218916A8F
:10B5F0008847681C85B22089A84200DD4EE7F8BD67
:10B6000010B50446002010F021FB022841D121484A
:10B610000078002802D101201E4908701D480078DA
:10B6200001281FD11B484078401C1A494870214608
:10B630005A20FCF785FD17494978884229D800200F
:10B640001449487008468078401C88700846807805
:10B650000A2803D30020887002200870002010F010
:10B6600025FB16E00B480078022812D109484078E3
:10B67000401C0849487021467D20C000FCF760FD51
:10B6800004494978884204D800200249487010F0E3
:10B690000DFB10BD6800002000B587B00021684692
:10B6A0000171042141710C480290411003910B4932
:10B6B000049105910A480690FFF78EFE01A810F04C
:10B6C00059FB00F0EDFA00F00FF80021054808F0F2
:10B6D000B7FC07B000BD0000FFFF1F00FFFFFF1F0A
:10B6E0001DB900000205000010B5FF2002306549B9
:10B6F0004860002008720120087000204872012074
:10B7000088726148FFF7D7FB5E495F48FFF7FCFB93
:10B7100001215D48FFF74CFC5C485A494860002015
:10B720000872012008700020487201208872564873
:10B730001030FFF7C0FB534953481030FFF7E4FBCC
:10B74000012151481030FFF733FC5048401E4D494D
:10B750004860002008720120087000204872012013
:10B76000887249485030FFF7A6FB4649464850309A
:10B77000FFF7CAFB012144485030FFF719FC43484A
:10B78000C13840494860002008720120087000203C
:10B790004872012088723C484030FFF78CFB3949E1
:10B7A00039484030FFF7B0FB012137484030FFF700
:10B7B000FFFBFF201230334948600020087201204F
:10B7C000087000204872012088722F486030FFF70F
:10B7D00072FB2C492C486030FFF796FB01212A4868
:10B7E0006030FFF7E5FBFF2021302649486000204C
:10B7F00008720120087000204872012088722248D7
:10B80000A030FFF758FB1F491F48A030FFF77CFB13
:10B8100001211D48A030FFF7CBFB3F204001194913
:10B820004860002008720120087000204872012042
:10B83000887215482030FFF73EFB1249124820302D
:10B84000FFF762FB012110482030FFF7B1FB1048E1
:10B850000C494860002008720120087000204872DE
:10B860000120887208483030FFF725FB054906485B
:10B870003030FFF749FB012103483030FFF798FBD8
:10B8800010BD00008C180020105504400204000078
:10B89000DF070000F0B50B46144643600481002129
:10B8A00036E0002216E02C254D4346687519AD5C44
:10B8B00018274F430668F619B5542C254D434668A2
:10B8C0007519AD5C18274F430668F6190836B5544C
:10B8D000551CEAB2082AE6D3002518274F4306680C
:10B8E000F619357418274F430668F619757418272A
:10B8F0004F430668F619B57418274F430668F619C2
:10B90000F57418274F430668F61975614D1CA9B2E6
:10B9100005898D42C5DC00258572F0BD70B50446F1
:10B92000606800F0BBFD0546E27A23460C332946E9
:10B93000094800F07BFD09496068884203D0491C32
:10B940006068884206D1E17AA28890B222460C3221
:10B9500002F000FD70BD0000C4070020DF070000FA
:10B96000F8B5054600262C46002C07D000BF03E0A2
:10B97000FF20A055701CC6B2082EF9D304F01AFBA4
:10B98000C0000821084007462068884338432060EB
:10B99000F8BDF8B5054600262C46002C07D000BFA0
:10B9A00003E0FF20A055701CC6B2082EF9D304F0A6
:10B9B00071FB07462068000C00043843206004F047
:10B9C00027FC0004070C3F04208880B23843206025
:10B9D000F8BDF8B505460026002704F01FFB0A2134
:10B9E0000090FCF7C3FB87B22C46002C07D000BFA9
:10B9F00003E0FF20A055701CC6B2082EF9D3072122
:10BA000009062068884339120906072212061140E8
:10BA1000084320606068000A0002F9B208436060D1
:10BA200001F0AAFC0002000A0002009020790099AF
:10BA30000843606004F0B2FAC007C00FC00700906E
:10BA400020684000400800990843206003F0C2FDD0
:10BA50000007000F009020680009000100990843CA
:10BA6000206003F0B1FD022806D1012109072068FA
:10BA700088434018206004E00121090720688843BA
:10BA8000206004F057FA0001F0210840009020687F
:10BA9000884300990843206004F002FBFF2806DD7C
:10BAA000FF21090420688843401820600BE004F05F
:10BAB000F7FA0004FF210904084000902068884339
:10BAC000009908432060F8BDF8B50546002600201F
:10BAD000009004F07BFA07466421FCF747FB80B234
:10BAE00000902C46002C07D000BF03E0FF20A0559B
:10BAF000701CC6B2082EF9D32068000A0002009913
:10BB0000C9B208432060002001F048FC0004070C83
:10BB10003F04208880B23843206003F061FD283064
:10BB20000002FF2109020840074620688843384385
:10BB30002060F8BDFFB581B004460F460025002601
:10BB4000002000902760039820810498E060002086
:10BB5000207400BF9DE01C206843216808586A01DA
:10BB6000616888501C2068432168081880686A0151
:10BB70006168891848601C2068432168081840687B
:10BB80006A016168891888601C2068432168081868
:10BB9000C0686A0161688918C8601C206843216810
:10BBA0000818007C6A016168891808741C206843C1
:10BBB00021680818407C6A016168891848741C2053
:10BBC000684321680818807C6A0161688918888345
:10BBD0001C20684321680818C07C6A0161688918C4
:10BBE000887400206A0161688918C8741C20684341
:10BBF000216808184068002813D01C206843216879
:10BC00000818C07C002805D1401E6A0161688918A7
:10BC1000C8831AE00020C0436A0161688918C8839C
:10BC200013E01C20684321680818C07C002805D058
:10BC300000206A0161688918C88306E000206A0153
:10BC400061688918C88301200090002607E0002160
:10BC50006A016068801814308155701CC6B2690191
:10BC600060684018808BB042F1DC1C20684321687A
:10BC70000818406900280AD06B016268D218104683
:10BC800014301C236B432268D21851698847681C02
:10BC9000C5B22089A84200DD5DE7009805B0F0BD7F
:10BCA00000B58BB056480790002108A8017068467F
:10BCB000017608A84170002052498872082108A81E
:10BCC000C170002004E0002209A90A54411CC8B236
:10BCD00008A9C9788142F6DC4B48FFF7ECF806A9C1
:10BCE0004948FFF711F94648401C0790002108A871
:10BCF00001706846017608A84170002041498872A9
:10BD0000082108A8C170002004E0002209A90A54F3
:10BD1000411CC8B208A9C9788142F6DC3A484030D3
:10BD2000FFF7C9F806A938484030FFF7EDF845207D
:10BD300000010790002108A801706846017608A854
:10BD4000417000202F498872082108A8C170002086
:10BD500004E0002209A90A54411CC8B208A9C97804
:10BD60008142F6DC28485030FFF7A5F806A926489E
:10BD70005030FFF7C9F8112040010790002108A8B2
:10BD800001706846017608A8417000201D4988723C
:10BD9000082108A8C170002004E0002209A90A5463
:10BDA000411CC8B208A9C9788142F6DC1648203087
:10BDB000FFF781F806A914482030FFF7A5F8FD2009
:10BDC000C0000290002168460173017141738173C4
:10BDD0000821C173002004E0002204A90A54411C78
:10BDE000C8B26946C97B8142F6DC07481030FFF7CC
:10BDF00062F801A904481030FFF786F80BB000BDC7
:10BE0000EE0600008C1800208055044030B585B047
:10BE10000446002520680190A1796846C1726179C5
:10BE2000417200210172017000BF05E02046083018
:10BE3000415D03A841556D1C6846C07AA842F5D8FB
:10BE4000112149010198401A1BD023210901401AF0
:10BE500011D011494018002802D0012817D104E060
:10BE600069460E48FFF721F912E069460B48403059
:10BE7000FFF71BF90CE0694608485030FFF715F949
:10BE800006E0694605482030FFF70FF900E000BFE3
:10BE900000BF05B030BD000062FDFFFF80550440CB
:10BEA000F0B585B004460F4600250026207C4006EC
:10BEB000400E55287ED100BF76E1690160684018C8
:10BEC000807C002877D169016068401840686A0169
:10BED000616889188968884209D2690160684018D8
:10BEE0004068C0196A016168891848605AE16901AF
:10BEF00060684018C068AF49884208D86901606826
:10BF00004018C068401C6A0161688918C8606901EE
:10BF100060684018C07C002821D1002607E000217D
:10BF20006A016068801814308155701CC6B26901BE
:10BF300060684018808BB042F1DC1C2068432168A7
:10BF40000818406900280AD06B016268D2181046B0
:10BF500014301C236B432268D21851698847690149
:10BF6000606840580090690160684018017C68462C
:10BF7000017100214171690160684018017F6846C4
:10BF80008171690160684018417C6846C171002672
:10BF900008E06901606840181430815D02A881558D
:10BFA000701CC6B2690160684018808BB042F0DC3A
:10BFB000E06801E0FCE01DE0002806D06846E1688A
:10BFC00088476A0161688918C87469016068401807
:10BFD000C07C002804D16A01616889184860E1E0EA
:10BFE0006901606840184068C01B6A01616889186F
:10BFF0004860D7E069016068401880680028EED08A
:10C00000690160684018C08B0028E8D06901606849
:10C010004018C08B6A0161688918C968884207D1D5
:10C02000690160684018C08B6249C94388427DD16C
:10C0300069016068401840686A0161688918896808
:10C04000884209D26901606840184068C0196A01D5
:10C05000616889184860A5E000206A016168891854
:10C060004860690160684018C0685249884208D831
:10C07000690160684018C068401C6A0161688918DD
:10C08000C860002607E000216A016068801814304B
:10C090008155701CC6B2690160684018808BB0423F
:10C0A000F1DC1C20684321680818406900280AD088
:10C0B0006B016268D218104614301C236B4322684F
:10C0C000D218516988476901606840580090690139
:10C0D00060684018017C6846017100214171690166
:10C0E00060684018017F6846817169016068401886
:10C0F000417C6846C171002608E06901606840180B
:10C100001430815D02A88155701CC6B26901606857
:10C110004018808BB042F0DCE068002808D0684608
:10C12000E16888476A016168891800E015E0C87411
:10C13000690160684018C07C002804D16A01616808
:10C14000891848602EE06901606840184068C01B8B
:10C150006A0161688918486024E01C2068432168EE
:10C160000818406800280FD00020C0436A016168A9
:10C170008918C8831C2068432168081840686A0130
:10C1800061688918886008E000206A016168891880
:10C19000C8836A0161688918886000206A01616843
:10C1A0008918C860681CC5B22089A84200DD84E6F1
:10C1B00005B0F0BD0000FFFF7CB500BF1921264887
:10C1C0000078FBF7BDFF044624486043244A8118E9
:10C1D0000022012009F006FE20460A225043643066
:10C1E000001981B2002201200BF036FB01200A2247
:10C1F00062431219D1B20A22624312190090D0B2DE
:10C2000001231A4608F050F80120009001900B20FD
:10C21000604382B20B20604381B2002301200AF008
:10C2200093FE6F20604381B201200BF065FD002575
:10C2300005E00121284609F00FFD681CC5B20F2D4D
:10C24000F7DB21460B2251436431C8B20BF020FFCB
:10C250000BF008FF7CBD000063000020672B00008E
:10C26000A0860100002005490870054908700549AD
:10C27000087005490870054908707047640000207F
:10C2800065000020630000206200002061000020A3
:10C29000F0B589B000BF00BF00BF00BF00BF00BF46
:10C2A00000BF00BF00BF052153480078FBF748FFDF
:10C2B0000446E1B2012009F079FB03214E480078E1
:10C2C000FBF754FF0B214843643080B20690E1B283
:10C2D00001231846069A08F0C1FA474909788A00EE
:10C2E00088180621FBF742FFFF21F531484380B251
:10C2F00007900798FBF73AFFC7B23946012008F0CC
:10C3000091FF03213C480078FBF730FF0B214843A5
:10C31000643080B208900022012008990BF09CFA4A
:10C32000032135480078FBF721FF3449484334495D
:10C330004018039000220120039909F053FD0321C6
:10C340002D480078FBF712FF0B21484380B2049080
:10C35000032129480078FBF709FF0B21484386B2E7
:10C360000120F1B20090049AD0B201231A4607F0DE
:10C370009BFF032120480078FBF7F8FE0B21484380
:10C3800085B20120009000232A46294601900AF038
:10C39000DBFD032118480078FBF7E8FE6F214843D6
:10C3A00080B20590012005990BF0A6FC1548007895
:10C3B0003C2805DA13480078401C1249087002E056
:10C3C0003C20104908700F4800781E2805DC0A48F8
:10C3D0000078401C084908700BE0074800780028E6
:10C3E00002D10549087004E003480078401E024964
:10C3F000087009B0F0BD000064000020672B000049
:10C40000A086010065000020002000BF06E000219A
:10C41000044A1154044A1154411CC8B25A28F6DB8C
:10C4200070470000E81400209C150020FFB581B083
:10C4300004460F463D462089A8422DDD182068435A
:10C4400021680818007C002826D1002609E00498FD
:10C45000815D182068432268101808308155701CCF
:10C46000C6B2082EF3D301211820684322681018A1
:10C4700041742C20684361680818006A00280BD0BA
:10C4800018236B432268D218104608302C236B43C4
:10C490006268D218116A884705B0F0BD01460620CF
:10C4A000104BCA1A99420FD008DCCA1FFA3A002A68
:10C4B00012D0102A0AD01F2A10D10BE0C02A07D0B0
:10C4C000C12A0BD100200BE0012009E0022007E087
:10C4D000032005E0042003E0052001E0062000BF62
:10C4E00000BF70474103000010B504467D21C9001C
:10C4F00061430846322103F071FB10BD014800681A
:10C5000070470000440000200148006870470000A8
:10C510004000002010B505490988652251430846AE
:10C520006421FBF723FE80B210BD00004E00002006
:10C53000014800787047000053000020014800784F
:10C54000704700004C00002010B50CF0B3FA012831
:10C550002ED100F065F8012000F068F803F09CFB94
:10C5600084B2204600F044F803F036FD84B2204641
:10C5700000F04AF803F06EFE012805D100F03EF805
:10C58000012000F047F805E0002000F037F8002017
:10C5900000F040F800201349086013480068134970
:10C5A00088421ED210480068801C0F49086018E0BD
:10C5B00000200D4908600B4800680C49884204D2ED
:10C5C00008480068801C07490860002000F028F82F
:10C5D000012000F02BF8002000F00AF8002000F005
:10C5E00013F810BD4400002040000020FFFFFF7F33
:10C5F00001490880704700004E0000200149087082
:10C600007047000053000020014908807047000077
:10C6100050000020014908707047000054000020BD
:10C6200001490870704700004C0000200149087063
:10C6300070470000520000200021014A117170472C
:10C6400000600040002201494A75704700600040C8
:10C65000002201494A767047006000400021014AEB
:10C6600011727047006000400021014A1173704749
:10C67000006000400021014A1174704700600040D2
:10C680000021014A11757047006000400021014AF5
:10C690001176704700600040002201494A737047DC
:10C6A00000600040002201494A7470470060004069
:10C6B00010B51C4C1C49206888421ED106221B491B
:10C6C000201DFBF7F8FD002817D10D221849204640
:10C6D0000A30FBF7F0FD00280FD10622154920464D
:10C6E0001730FBF7E8FD002807D106221249204643
:10C6F0001D30FBF7E0FD00280DD000F073FE0A4866
:10C700000E49086007480FF0C0FB0C4A2421054879
:10C710000FF0E6FB04E0242221460848FBF7A7FDC2
:10C7200010BD0000000250007AA7A55A990600200B
:10C730009F060020930600208D0600208C1C002000
:10C74000002008490870084908700120074908704E
:10C75000002007490870074807490860002007497A
:10C76000087070477B0600207A0600207D060020B6
:10C770008206002025060000AC0600208C06002062
:10C7800010B504469120604384B20A212046FBF78D
:10C79000EDFC84B205212046FBF7E8FC052901DB0E
:10C7A000601D84B2204610BD70B5A8B005460024B7
:10C7B0000026A0216846FBF773FD00F093FC1E499C
:10C7C0000A6814216943505000211B480268142054
:10C7D0006843101841601848026814206843101814
:10C7E000816015484068002824D000BF17E060062B
:10C7F000060E282E00D316E00F480168142060436F
:10C800000858B1006A4650500B4801681420604334
:10C8100008184168701C80001150601CC4B20648A2
:10C82000007AA042E3DC00BF620003486946436827
:10C830000220984728B070BDDC1C002030B5A9B09C
:10C8400000240025A02101A8FBF72AFD00BF25E058
:10C850006006050E00F046FC1F490A68142161437A
:10C86000505000211C480268142060431018416099
:10C87000194802681420604310188160282D0BD2DB
:10C8800015480168142060430858A90001AA5050B7
:10C890000021681C80001150601CC4B20E48007A50
:10C8A000A042D5DC0C484068002813D00A48007A22
:10C8B0004000282806D30848282201A943680220FE
:10C8C000984707E00448007A4200034801A94368FA
:10C8D0000220984729B030BDDC1C002010B50CF0B8
:10C8E000E9F801287ED1FFF70FFE4F49884216D2A2
:10C8F0000F204E494871887108468078002801D180
:10C900000520487049488078052802D10020474911
:10C910004870002045490872487208702AE0FA20E1
:10C920004249487188714249088803F085FA4048B5
:10C93000807800280CD13D49087008464079C870BD
:10C94000084680790871002088704870487211E0AC
:10C950000120364908700846407A00280AD1012093
:10C96000487208464078887008464079C870084682
:10C97000807908712D4880782C494978884213DDE8
:10C9800000202A49C87008460079401C08710846F2
:10C9900000798979884220DB002024490871084603
:10C9A0008078401E887018E0204880781F494978B8
:10C9B000884212DA00201D4908710846C078401CE0
:10C9C000C8700846C0784979884206DB00201749BC
:10C9D000C87008468078401C887015488078002808
:10C9E00005D100E013E00120104908721BE0104857
:10C9F0000088732803DB02200C49087213E00C48FE
:10CA0000008870280FDC0020084908720BE0002025
:10CA10000649087008464079C87008468079087150
:10CA200000200872487210BDB80B0000F408002006
:10CA30006C0000200020044988704870C87008719C
:10CA40000872487270470000F40800200020064970
:10CA500008808870054988704870FA20C87008718D
:10CA600000200872487270476C000020F408002013
:10CA700070B503F03BF9044603F04AF905460CF0A3
:10CA800019F801282ED105211A48FEF707FA552872
:10CA900004D1002018498870088027E0012D04D1B6
:10CAA000002015498870088020E001201249887014
:10CAB0001248844202DB201A84B200E000240A21DA
:10CAC0002046FBF753FB052901DB601D84B20C48AF
:10CAD000844200DD04460A212046FBF747FB064955
:10CAE000088003E00020044988700880FFF7F6FE04
:10CAF00070BD0000C40700206C000020AA0A0000DE
:10CB0000C60700001CB500200090019000F0EAFA72
:10CB10000B49086000200B49096808600A48006852
:10CB200000280CD00749096808680A21FBF708FBB0
:10CB30000090012269460520034B1B6898471CBDE5
:10CB40007C0700207007002078070020002008499B
:10CB50004880084908800849088008490870084941
:10CB600088720849088048800120087170470000D9
:10CB70002C000020200000202200002024000020A3
:10CB8000A807002026000020F8B503F091F807461A
:10CB900003F0A0F80090FFF7D1FC012860D1052137
:10CBA000C548FEF77BF9552802D00098012807D127
:10CBB0000020C2490870C2490880C249887256E004
:10CBC000BE480078002810D10120BC4908703D46BD
:10CBD0002846E917890F091889030D0CBA488542C0
:10CBE00000DD0546B648058041E0B648807A400041
:10CBF000B4490F520846867A0EE07000B1490D5ACA
:10CC0000701E4000085A7100AE4A5052701E40001B
:10CC100011460D52701EC6B2002E08DD7000A949E3
:10CC2000095A701E4000A74A105A8142E5DBA54808
:10CC3000807A401CA34988720846807A052816DB52
:10CC4000002088720846C5882846E917890F091808
:10CC50008D109D48854200DD05469948058006E017
:10CC60000020964908709649088096498872944831
:10CC7000058896480088A84257DA94480088281A00
:10CC800084B292480079012827D190484088A04278
:10CC90000BDA8E4840880A308C4948800846408824
:10CCA000A04204DD0846448001E08848448087486B
:10CCB00044882046E117890F09188C100A2C00DAE5
:10CCC0000A248248008800198049088008460088A4
:10CCD000A84201DD08460580CDE07C484088142844
:10CCE00005DD7A48408814387849488002E0002001
:10CCF00076494880754844882046E117890F09180D
:10CD00008C100A2C03DA012070490871B3E06F48D7
:10CD10000088A04205DD6D480088001B6B49088033
:10CD2000A9E0002069490880A5E068480088A84279
:10CD300059DD66480088401B84B2644800790128A8
:10CD400027D162484088142805DD6048408814389F
:10CD50005E49488002E000205C4948805B48448886
:10CD60002046E117890F09188C100A2C03DA0220DB
:10CD7000564908717FE055480088001953490880DA
:10CD8000084600885049884275DD08464F490880AA
:10CD900071E04E484088A0420BDA4C4840880A3087
:10CDA0004A49488008464088A04204DD084644803D
:10CDB00001E046484480454844882046E117890FF1
:10CDC00009188C100A2C00DA0A2440480088291916
:10CDD000884202DA3D4805804DE03C480088001B4F
:10CDE0003A49088047E0394844882046E117890FCE
:10CDF00009188C100A2C3EDD34484088142805DDC3
:10CE00003248408814383149488002E000202F49D8
:10CE100048802E4844882046E117890F09188C1055
:10CE20002A480079012813D10A2C03DA0220274965
:10CE3000087120E025480088001924490880084628
:10CE400000882149884216DD08462049088012E002
:10CE50000A2C03DA01201D4908710CE01B480088E8
:10CE6000A04205DD19480088001B1849088002E02F
:10CE700000201649088016480088502804DC134812
:10CE800000881349088016E0104800881049098876
:10CE9000884204DD0D4800880D4908800BE00B48EE
:10CEA00000880B490988081A84B2502C03DB074814
:10CEB000008807490880F8BDC4070020240000202E
:10CEC00020000020A8070020E02E000026000020FF
:10CED0002200002010B5044664204443A1212046CE
:10CEE000FBF72EF90446204610BD00007CB5002457
:10CEF00000200190009000F03FFA05460A21FBF760
:10CF00001FF9044601226946042000F063FC0098E2
:10CF1000401C002814D17D20C00020181149086051
:10CF2000084600680190012201A9032000F090FC4E
:10CF30000120009001226946042000F089FC0FE0E6
:10CF4000009801280CD17D200001201805490860B7
:10CF5000084600680190012201A9032000F078FC36
:10CF60007CBD0000D400002010B501200F490870DE
:10CF700000200F49096808600D49096848600C499C
:10CF80000968886000F07EF9FFF7BCFDFFF756FCEA
:10CF900008480068002807D00122054801680831C8
:10CFA0000020044B1B68984710BD000015070020A7
:10CFB000100700200C07002010B518480068184919
:10CFC000884229D117480068002804D01548006815
:10CFD00080471549087015480068002804D0134898
:10CFE000006880471249087012480068002804D081
:10CFF00010480068804710490880104800680028E1
:10D0000005D00E48006880470D49088002E00D48B1
:10D010000B49088000F078F810BD000020070020C0
:10D0200078563412FC060020140700200007002068
:10D03000160700200407002018070020080700201A
:10D040001A0700201027000010B50023174C23609A
:10D05000174C2370174C2370174C2370174C2380E8
:10D06000174C2380174C2370174C13682360174C00
:10D0700053682360164C93682360164CD368236072
:10D08000154C1369236000280CD0144B1860134C06
:10D090000B682468A3600023104C246823600F4CA5
:10D0A000246863600E4B014C236010BD20070020F4
:10D0B0001C07002014070020160700201807002076
:10D0C0001A07002015070020FC060020000700209A
:10D0D00004070020080700200C070020100700208C
:10D0E00078563412054800680549884203D105483E
:10D0F0000068806870470020C043FBE720070020DD
:10D10000785634121007002070B500240025002640
:10D110003048007801285CD12F480078002858D189
:10D120002E480078012854D12D4805882D490988BA
:10D13000694308462C49FBF703F885B2E12000015A
:10D14000854207D81921694308460921FAF7F8FFF3
:10D15000044600E0244C2548006800680019234973
:10D160000968086021480068006820490968496822
:10D17000884207D31D48006800681C49096849684F
:10D18000461A0AE01948006840680021C943081A95
:10D190001649096809684018461C1548864218D384
:10D1A000344601462046FAF7CBFF04460F48006894
:10D1B00041680F48604308180C490968486001201D
:10D1C0000C49087009480068806800190749096817
:10D1D000886070BD14070020150700201607002086
:10D1E000180700201A070020102700001007002051
:10D1F000A08601001C07002000220C4B1A600C4B7B
:10D200000A681A600B4B4A681A600B4B8A681A60EE
:10D210000A4BCA681A600A4B0A691A60002801D0D2
:10D22000084A1060084A014B1A6070472007002026
:10D23000FC0600200007002004070020080700204B
:10D240000C070020100700207856341210B50A4849
:10D25000006800280ED00948007801280AD1002073
:10D260000649087001220648016808310020024B77
:10D270001B68984710BD00000C0700201C07002009
:10D28000100700201CB50020009001900024FFF73B
:10D2900029FF04460E480068046000200C49096814
:10D2A00048600B49096888600A48006800280DD06A
:10D2B00007480068006800900548006840680190D1
:10D2C000022269460120034B1B6898471CBD0000E1
:10D2D0002407002028070020F8B505460C4616460E
:10D2E0000027002D17D00E480560FFF7FBFE07460C
:10D2F0002068B84203D90A480068076003E008497B
:10D30000206809680860064960680968486004493F
:10D31000A0680968C8600348066000F005F8F8BD19
:10D32000240700202807002070B500240025FFF7FF
:10D33000D9FE04460F4800680068A04200D903E007
:10D340000C4800680068251A0A48006840684019BF
:10D3500008490968886007480068806805490968C5
:10D36000C968884205D903480068C068014909684E
:10D37000886070BD240700200148006880687047FD
:10D3800024070020002801D0024A1060024A1160E0
:10D39000704700002407002028070020014610489D
:10D3A000026814204843101882680D48036814204E
:10D3B00048431818C06882420BD9094802681420F3
:10D3C00048431018C26806480368142048431818D8
:10D3D0008260034802681420484310188068704730
:10D3E000DC1C0020002005E019490A5C19490A5498
:10D3F000411CC8B20628F7DB002006E016490A5C8B
:10D400001449891D0A54411CC8B20D28F6DB0020BE
:10D4100006E012490A5C0F4913310A54411CC8B294
:10D420000628F6DB002006E00D490A5C094919319F
:10D430000A54411CC8B20628F6DB002005E0002291
:10D4400004491F310A54411CC8B20128F7DB704758
:10D4500099060020901C00209F06002093060020C3
:10D460008D06002010B5002005490880488008710D
:10D470004871887102F0A4FD0149C87110BD000017
:10D480007000002070B50024002502F099FD61496C
:10D49000C87102F081FC044602F088FC0546FFF7E3
:10D4A0004DF8012870D101215B48FDF7F7FC5528A4
:10D4B00007D1002057490871487108804880887159
:10D4C000A7E0FF2C01D0FF2D5FD1FF2C28D1FF2D2D
:10D4D00026D000204F490871012048716320088040
:10D4E000FF2014306843488048880A21FAF73EFE3E
:10D4F0004849488008464088632801DD6320488009
:10D5000044484088112803DB42484088192803DD3D
:10D510000120404988717CE000203E49887178E014
:10D52000FF2C01D1FF2D26D101203A49087100209E
:10D53000487163204880FF201430604308800888C9
:10D540000A21FAF713FE3349088008460088632849
:10D5500001DD632008802F480088112803DB2D4857
:10D560000088172803DD01202A49887151E0002036
:10D57000284988714DE063202649088048800020B2
:10D5800088710871487144E03CE00120214908712C
:10D590004871FF2014306043088008880A21FAF798
:10D5A000E5FD1C49088008460088632801DD6320EA
:10D5B0000880FF20143068431649488048880A21B3
:10D5C000FAF7D4FD1349488008464088632801DDF6
:10D5D000632048800F48008811280BDB0D48008825
:10D5E000172807DC0B484088112803DB09484088CE
:10D5F000192803DD0120074988710AE00020054948
:10D60000887106E00020034908714871088048804D
:10D61000887170BD70000020C4070020FFB583B082
:10D6200006460D46174600240020029000BF142035
:10D63000784380190190002E57D00198002854D0CB
:10D640002B4806602A49069848600846077200BFC2
:10D6500045E0FFF747FD02902001295802988142DA
:10D6600004D820012858401C002806D120490298DF
:10D670000A6814216143505006E0200129581C48D3
:10D680000268142060431150200140194068401C7A
:10D69000002807D1002116480268142060431018A2
:10D6A000416008E0200140194168114802681420D7
:10D6B0006043101841602001401981680C480268DD
:10D6C000142060431018C16020014019017B0848F4
:10D6D00002681420604310180161601CC4B2044841
:10D6E000007AA042B5DC00F005F807B0F0BD0000FC
:10D6F000DC1C002070B5002400250026FFF7F2FC9A
:10D70000054600BF4EE02A480168142060430858CF
:10D71000A84239D8264801681420604308582E1AB8
:10D720002348016814206043081840688119204884
:10D73000026814206043101881601D48016814209D
:10D740006043081881681A48026814206043101862
:10D75000C068814224D91648016814206043081823
:10D760000069002803D02046FFF71EF818E0104893
:10D770000168142060430818C1680D48026814202D
:10D780006043101881600BE0094801681420604371
:10D790000818406806490A681421614351188860D6
:10D7A000601CC4B20248007AA042ACDC70BD00002C
:10D7B000DC1C002010B500BF14244C4323180028A3
:10D7C00005D0002B03D0024C20606260217210BD96
:10D7D000DC1C0020F8B505460E4614462B000DF063
:10D7E000F3FE0504121920272E001748FBF7C0F896
:10D7F000164908701448FAF76BFD07466421FAF7DA
:10D800009FFC30601CE0A004020C31461020FBF7A6
:10D81000A9F915E0A004020C31463020FBF7A2F96B
:10D820000EE0A004020C31465020FBF79BF907E004
:10D83000A004020C31467020FBF794F900E000BF11
:10D8400000BF0020F8BD0000CA160020850000209F
:10D8500070B505460E4614462B000DF0B5FE0504C6
:10D860001C232A3138003068002802D1FAF71EFF45
:10D8700010E064223168514308461649FAF732FD38
:10D88000002015490870012264211248FBF7D8F9DD
:10D89000114908701CE0A004020C31461020FBF76F
:10D8A0001FFB15E0A004020C31463020FBF718FBEB
:10D8B0000EE0A004020C31465020FBF711FB07E0FC
:10D8C000A004020C31467020FBF70AFB00E000BF09
:10D8D00000BF70BDBC1600208400002000B5AFB0B2
:10D8E00050211BA8FAF7DCFC00201A90142115A87F
:10D8F000FAF7D6FC0020129013901490119040215A
:10D9000001A8FAF7CDFC00203F49086001221BA9BD
:10D91000FFF760FF1B98401C002801D11A9001E01E
:10D920001B981A9039481590394816903948179025
:10D93000002018903848199015AA1AA93748FFF7FF
:10D9400083FB02221CA90120FFF744FF1C98401C06
:10D95000002801D1129001E01C9812901C98401CE4
:10D96000002801D1139001E01D9813902C481490C9
:10D9700012A92C48199AFFF7AFFC08221EA9022011
:10D98000FFF728FF1E98401C002801D1019001E0FC
:10D990001E9801901F980290234803900120694629
:10D9A0000874801E059021490791012101A8017783
:10D9B000881E09901D490B91012109A80173881E39
:10D9C0000D901A490F9101210DA80173042201A99C
:10D9D0001748199BFFF722FE01221BA90320FFF71E
:10D9E000F9FE14491B9808601B98401C002806D1BA
:10D9F000FF20F530086001220320FFF729FF0E48C1
:10DA0000014908602FB000BD880000203DC500001E
:10DA100031C5000015C5000051D800005016002087
:10DA200076841E005C1600200F2700009F860100F0
:10DA30006C160020D4000020A33AA55A00B585B08A
:10DA400014216846FAF72CFC00200F4908600F48A3
:10DA500000900F4801900F480290002003900E485C
:10DA6000049069460D48FFF7C7FB0D480499FFF77E
:10DA700089FC04210B48049AFFF79CFE0A480249DE
:10DA8000086005B000BD0000880000203DC5000012
:10DA900031C5000015C5000051D800005016002007
:10DAA0005C1600206C160020A33AA55A00200B49F2
:10DAB00008800B4908800B49088001200A4908703A
:10DAC00000200A4908730A4908804880012008712B
:10DAD000002006494880088070470000320000207E
:10DAE000340000203600002038000020B407002059
:10DAF0003A000020FEB502F015F9009002F01CF982
:10DB00000190FEF71BFD01286BD10521D548FDF7DB
:10DB1000C5F9552807D10020D3490870D34908809A
:10DB2000D349888067E00198012807D10020CE49B9
:10DB30000870CE490880CE4988805CE0CA480078E9
:10DB4000002808D10120C8490870009D0A206843B8
:10DB5000C64908804FE0009881B2C548007B42006A
:10DB6000C348801D8152801F067B11E07100C048B0
:10DB7000801D455A701E4100BD48801D415A7200EB
:10DB80008152701E4100BA48801D4552701EC6B2B7
:10DB9000002E0ADD7100B648801D415A701E4200F9
:10DBA000B348801D805A8142E0DBB148007B401CB5
:10DBB000AF4908730846007B032807DB0020087381
:10DBC000084605890A206843A84908800020A8491A
:10DBD00008804880A548008888800120A2490870F4
:10DBE00009E00020A0490870A0490880A0490880E9
:10DBF0004880087388809D4805889E480088A84210
:10DC000056D29C480088281A84B29A480079012884
:10DC100026D198484088A0420BDA96484088801C5C
:10DC20009449488008464088A04204DD0846448064
:10DC300001E0904844808F48448803212046FAF749
:10DC400095FA84B2022C00DA02248A48008800196E
:10DC50008849088008460088A84200D90D80CDE098
:10DC600084484088062805DD82484088801F814915
:10DC7000488002E000207F4948807E484488032194
:10DC80002046FAF773FA84B2022C03DA01207949AC
:10DC90000871B3E077480088A04205DD7548008828
:10DCA000001B74490880A9E0002072490880A5E0A3
:10DCB00070480088A84259D96E480088401B84B239
:10DCC0006C480079012827D16A484088062805DD7C
:10DCD00068484088801F6749488002E00020654905
:10DCE00048806448448803212046FAF73FFA84B20A
:10DCF000022C03DA02205F4908717FE05D4800884A
:10DD000000195C490880084600885B49884275DD37
:10DD100008465849088071E056484088A0420BDA0E
:10DD200054484088801C5349488008464088A04297
:10DD300004DD0846448001E04E4844804D48448854
:10DD400003212046FAF712FA84B2022C00DA0224E8
:10DD5000484800882919884202D246490D804DE082
:10DD600044480088001B4349088047E041484488F4
:10DD700003212046FAF7FAF984B2022C3EDD3D4831
:10DD80004088062805DD3B484088801F3949488087
:10DD900002E0002037494880364844880321204665
:10DDA000FAF7E4F984B233480079012813D1022C40
:10DDB00003DA02202F49087120E02E48008800195C
:10DDC0002C490880084600882B49884216DD084601
:10DDD0002849088012E0022C03DA01202549087145
:10DDE0000CE024480088A04205DD22480088001B82
:10DDF0002049088002E000201E4908801D48008854
:10DE00001E490988884203DA1A4800880F2804DA74
:10DE100018480088194908800AE016480088174900
:10DE20000988081A0F2803DB124800881349088064
:10DE3000124807880C48007800280ED06B20474312
:10DE400064213846FAF77CF907460A370A488742C0
:10DE500000D907460A490F8002E0002008490880DF
:10DE6000FEBD0000C4070020380000203200002062
:10DE7000B40700203A000020C6070000360000204A
:10DE8000340000200020074908800749088007491E
:10DE900008804880012008710020054948800880DA
:10DEA0007047000034000020360000203A000020B7
:10DEB000B40700200020024908700249087070472A
:10DEC0007B0000207C00002010B5FEF737FB012806
:10DED00013D103210C48FCF7E1FF552805D10020A0
:10DEE0000A4908700A4908700CE001F069FF074907
:10DEF000087001200649087004E0002003490870FA
:10DF00000349087010BD0000C40700207B000020FA
:10DF10007C000020F0B5A9B004460E46002500277D
:10DF200000202890A0216846FAF7BAF9FFF7DAF83E
:10DF300026490A681421614350502448016814207E
:10DF400060430818C068B0420CD220480168142011
:10DF500060430818C1681D48026814206043101807
:10DF6000416005E0194801681420604308184660C4
:10DF700016484068002826D0002517E06806070EDE
:10DF8000282F00D316E01148016814206843085870
:10DF9000B9006A4650500D480168142068430818BB
:10DFA0004168781C80001150681CC5B20748007A8F
:10DFB000A842E3DC00BF6A000448694643680220C7
:10DFC000984701202890289829B0F0BDDC1C00203B
:10DFD00010B500F0EDFD00F0D7F80CF085FB00F077
:10DFE0000DFB00F001F810BD70B541480078912894
:10DFF00000D070BD00F0BEF8012876D13D48008801
:10E000003D49088008468078F021884320303A490D
:10E01000887008468078000900013549097A0907A7
:10E02000090F0843344988703148807A401E3049CE
:10E03000887208460089401C088108460089C98802
:10E04000884216DA08202C49887200240EE02848FD
:10E0500041882848001D415C2748C01C01552448C0
:10E060004088401C22494880601CC4B2072CEEDB6B
:10E070002DE01F4800891E49C98888421CD11C48D0
:10E0800000791B498978401AC5B2681C1A49887200
:10E0900000240EE0164841881648001D415C1648D1
:10E0A000C01C015512484088401C11494880601C22
:10E0B000C4B2AC42EEDB0AE000F006FD00200C49E1
:10E0C00008700C490888092100F0B8F991E701208F
:10E0D00000F0BCFC084A917A1088921C00F070F99C
:10E0E00005490888002100F0C1F800BF81E7000061
:10E0F000401A0020DC1900206C1900201B49097E01
:10E10000002932D01949897E0C225143174A515AAD
:10E11000174A118000200CE01449897E0C225143DB
:10E12000124A8918891C0A5C1149891C0A54411C2D
:10E13000C8B20828F0DB0D49897E0C2251430B4AF6
:10E140008918897A0A4A91720121D1720749097E98
:10E15000491E064A11761146897E491C9176114660
:10E16000897E022901DB0021917670473819002051
:10E17000601900200349487B012802D10021014A8F
:10E1800051737047501A002010B53348406800287A
:10E1900061D13148007B03000DF016FA07590512D2
:10E1A000212E3D4A59002D480078002807D0002034
:10E1B0002A4908702A490888012100F03FF947E000
:10E1C00026480078002809D00020244908702549F5
:10E1D0004A8808880123091D00F040F938E01F48EB
:10E1E0000078002807D000201C4908701C490888C6
:10E1F000022100F023F92BE018480078002809D00C
:10E2000000201649087017494A8808880923091D03
:10E2100000F024F91CE011480078002807D0002005
:10E220000E4908700E490888092100F007F90FE02F
:10E230000A480078002809D00020084908700949D8
:10E240004A8808880323091D00F008F900E000BF90
:10E2500000BF00F039FC10BD501A0020401A002009
:10E26000DC190020781900207047000070B50446C2
:10E270000D4634480088A04263D1002D61D1324858
:10E28000007822284ED004DC20283DD0212856D109
:10E2900041E0902802D0912851D115E02A48C08849
:10E2A00001280AD100202849087000F00DFC2749F8
:10E2B0000888002100F0C2F805E0032000F0C6FB4A
:10E2C000A020214908703BE01F4800891E49C988E9
:10E2D00088420AD100201C49087000F0F5FB1B4958
:10E2E0000888002100F0AAF80DE01748807A00287D
:10E2F00006D000F0E9FB1449087B00F089FB02E03E
:10E30000032000F0A3FB1BE0062000F09FFB112080
:10E310000D49087014E0062000F098FB11200A490E
:10E3200008700DE000200849087000F0CDFB084996
:10E330004A8808880923091D00F090F800E000BF12
:10E3400000BF70BD54190020401A0020DC190020C5
:10E350007819002070B50346184C247E022C00DB8F
:10E3600070BD164C647E0C256C43144D2B5300205D
:10E370000AE0155C114C647E0C2674430F4EA41900
:10E38000A41C2554441CE0B28842F2D30B4C647E9A
:10E390000C267443094EA419A1723446247E641CD1
:10E3A00035462C762C46647E641C6C762C46647E46
:10E3B000022C01DB00246C7600BFD1E73819002065
:10E3C000F0B585B007460D4616461A48078000246A
:10E3D00006E031781748801C0155761C601CC4B2D9
:10E3E000AC42F6DB2C4605E0AA211248801C015500
:10E3F000601CC4B2082CF7DB0E480088019008218D
:10E400006846C1720021417201720170002406E069
:10E410000848801C015D03A80155601CC4B2082C8B
:10E42000F6DB69460448FCF740FE0120014988728A
:10E4300005B0F0BD541900209055044070B5044655
:10E440000D46294620460CF07BF870BD70B5044699
:10E450000D46294620460CF081F870BDF8B50446FB
:10E460000D4616461F463B463246294620460CF0CE
:10E4700076F8F8BDF8B507460E4615465C480078B4
:10E48000002804D009213846FFF7D8FFF8BD002D39
:10E4900001D0602D04DD09213846FFF7CFFFF5E7F5
:10E4A000544807804580002406E031785148001D1B
:10E4B0000155761C601CC4B2AC42F6DB00204C490E
:10E4C000487008468580FF2088727F2008730846C0
:10E4D000808808282EDA0120C88008468088488075
:10E4E0000120088143480088434908800846807815
:10E4F000F02188434049887008468078000900016F
:10E500003B4909790907090F08433B498870384896
:10E510000079401C8872002407E03648001D015D28
:10E520003548C01C0155601CC4B231488088A042E7
:10E53000F3DC4AE00721681CF9F718FE002907D030
:10E54000072128460830F9F711FE2949C88005E05F
:10E550000721681CF9F70AFE2549C88006202449CE
:10E560004880012008812348008823490880084604
:10E570008078F021884310301F49887008468078E1
:10E58000000900011A4989880905090F08431A4939
:10E59000887008464088FF21090288431449898809
:10E5A0000902FF2212021140084313494880082043
:10E5B0008872002407E00F48001D015D0E48001D11
:10E5C0000155601CC4B2062CF5DB012000F03EFAB8
:10E5D000094A917A1088921CFFF7F2FE90200449B4
:10E5E0000870054908880021FFF740FE00BF4DE78D
:10E5F000401A0020DC1900206C19002010B5FFF72C
:10E600007DFD1448C07A002822D012488078000985
:10E61000002806D0012807D002280AD0032810D1EC
:10E620000CE000F09DF90FE000F09EF800F05AFABF
:10E630000AE000F011F800F055FA05E000F000F9EA
:10E6400002E0FFF711FE00BF00BF00200149C872C1
:10E6500010BD00006019002010B540480078112856
:10E6600000D010BD3E4800883F214901884200D0BB
:10E67000F7E73B4880780007000F3849097A090717
:10E68000090F88420CD000203449087000F01CFAB1
:10E6900034494A8808880423091DFFF7DFFEE0E7B4
:10E6A0002E480089401C2D4908810846807A401E6A
:10E6B000887208460089C98888421BDA2848807A0F
:10E6C000082800D0CDE700240EE02548C01C015DDD
:10E6D000224842882348001D815420484088401C1D
:10E6E0001E494880601CC4B2072CEEDB062000F0F7
:10E6F000ADF930E01948808818494988401A18490E
:10E70000897A884203DA1648807A082800D0A8E778
:10E7100000240EE01248C01C015D104842881148D8
:10E72000001D8154601CC4B20C484088401C0B4939
:10E7300048800A484088094989888842EADB0020E5
:10E740000649087000F0C0F906494A880888002385
:10E75000091DFFF783FE00BF83E70000401A002079
:10E76000601900207819002070B5324800788021A7
:10E770000840802800D170BD2F4800883F21490102
:10E78000884200D0F7E72C48807A082800D0F2E7CA
:10E790002948807805072D0F2D0227484088000A58
:10E7A0000543082D00DAE6E70020224948700620DC
:10E7B0004880084685800120088108208872002052
:10E7C000C8728988481C0721F9F7D0FC002909D0B4
:10E7D00018498988084608300721F9F7C7FC154908
:10E7E000C88007E013498988481C0721F9F7BEFC57
:10E7F0001049C880104800881049088008464580A4
:10E80000002407E00C48001D015D0C48001D015567
:10E81000601CC4B2062CF5DB042000F017F91020B0
:10E8200004490870054A51881088FFF70FFE00BFA1
:10E83000A1E70000401A002060190020781900208C
:10E8400010B544480078A02808D0424800789128A4
:10E8500004D040480078A12800D010BD3E48008870
:10E860003F21490188420AD03C4908880921FFF725
:10E87000E5FD00F029F9002036490870EDE736483B
:10E88000807A08280AD0354908880921FFF7D6FD83
:10E8900000F01AF900202F490870DEE72E48807832
:10E8A0000007000F002804D0012825D0022843D1FA
:10E8B0002EE028484078002800D048E02648C0785C
:10E8C000002803D101202349487003E02248C07882
:10E8D000204988721F480078912803D01E4800798B
:10E8E0001C49087391201B49087000F0EDF8194984
:10E8F000087B00F08DF82AE016484078002800D008
:10E9000025E0A12013490870032000F09FF81EE0C5
:10E9100010484078002800D019E00E480078A02860
:10E9200009D10E4908880821FFF788FD00F0CCF8CE
:10E930000020084908700AE0084908880521FFF707
:10E940007DFD00F0C1F800200249087000BF00BF43
:10E9500000BF82E7401A002060190020DC19002067
:10E9600010B52848007880210840802800D110BDCB
:10E9700024480078002806D0234800883F21490118
:10E98000884200D0F3E72048807A1F498978090738
:10E99000090F884203DD1C48807A082800D0E6E78A
:10E9A000194880780007000F002805D016488078A5
:10E9B0000007000F072800DDD9E713480088134936
:10E9C0000880114880780007000F4880002407E085
:10E9D0000D48C01C015D0D48001D0155601CC4B2EE
:10E9E0000A484088A042F3DC00200649087000F085
:10E9F0006BF806494A8808880023091DFFF72EFD99
:10EA000000BFB4E7401A00206019002078190020E8
:10EA10007F2805DC7D21C90041430A4A91600DE051
:10EA2000F12808DBF92806DC0107090F64225143AD
:10EA3000044A916002E00449024A91600221014ABD
:10EA400051737047501A002018F0010000B5030000
:10EA50000CF0BAFD0729050B11171D232900012110
:10EA6000144A11731449516022E00221114A1173B2
:10EA7000114951601CE003210E4A11730F49516086
:10EA800016E004210B4A11730D49516010E0052175
:10EA9000084A1173002151600AE00621054A1173EA
:10EAA0000849516004E00021024A1173516000BF1F
:10EAB00000BF00BD501A0020A8610000F82401002A
:10EAC00028230000F0490200002001490873704724
:10EAD000501A0020024909880918014A118070471C
:10EAE000501A002010B52F480078102818D12E4851
:10EAF000408860280ADD2D48807800090001801CCC
:10EB00002A49887022202749087025E02748807804
:10EB100000090001254988702020224908701BE067
:10EB200020480078112816D11E48807A002800D08D
:10EB300010BD1C484078002800D0F9E7082019498A
:10EB400088721A48807800090001184988702020CE
:10EB50001449087000E0EBE7FD20C000134908806D
:10EB600008468078F0218843303010498870084684
:10EB7000C0780020C870084600791420087103206E
:10EB800088720220FFF762FF084A917A1088921C6F
:10EB9000FFF716FC054908880021FFF767FB00BF57
:10EBA000C6E70000401A0020781900206C190020E8
:10EBB000244A118852888A4242D0224A52888A4284
:10EBC00004DA204A52888A1A90B207E01D4A528815
:10EBD0000023DB439A1A521C521890B2194A5180F2
:10EBE000127B002A10D0174A5268002A0CD0154A0E
:10EBF0005268824205D9134A5268121A114B5A6060
:10EC000002E000220F4B5A600E4A527B022A17D1B3
:10EC10000C4A9268002A0CD00A4A9268824205D9AE
:10EC2000084A9268121A074B9A6002E00022054BCC
:10EC30009A60044A9268002A02D10122014B5A7359
:10EC400070470000501A0020FEB5002700200290F7
:10EC500001900090002400250026FDF76FFC01289C
:10EC600079D100218A48FCF719F9552808D189483B
:10EC700001788948F9F714FB00208649087006E1FD
:10EC800001F0B2F8074601F0C3F8029001F0B6F8BF
:10EC9000019001F0C7F8009001F09CF87F490870DE
:10ECA000F020384000110A2805DBF0203840001120
:10ECB000C01C044303E0F020384000110443240248
:10ECC0003807000F0A2804DB3807000FC01C044374
:10ECD00002E03807000F04432402F02102980840A4
:10ECE00000110A2805DB029808400011C01C0443EB
:10ECF00004E0F02102980840001104432402029825
:10ED00000007000F0A2805DB02980007000FC01C4F
:10ED1000044303E002980007000F0443F021019828
:10ED2000084000110A2805DB019808400011C01CAA
:10ED3000054304E0F02101980840001105432D022D
:10ED400001980007000F0A2806DB01980007000F52
:10ED5000C01C054304E092E001980007000F054342
:10ED60002D02F0210098084000110A2805DB0098C8
:10ED700008400011C01C054304E0F0210098084041
:10ED8000001105432D0200980007000F0A2805DB3B
:10ED900000980007000FC01C054303E0009800071F
:10EDA000000F05433D480078002808D1002604E004
:10EDB0000020B100384A5050761CFF2EF8D3384856
:10EDC000007836490978884213DA002C11D034488B
:10EDD00002783449204600F0A7F8002809D13048CD
:10EDE000007880002F490C502D480078401C2C4999
:10EDF00008702B48007829490978884213DA002DD9
:10EE000011D0274802782749284600F08DF80028BD
:10EE100009D123480078800022490D50204800780D
:10EE2000401C1F4908701E4800781C490978884218
:10EE30002DD100260AE0B0001A490858B1001A4A3C
:10EE400050500020B100174A5050761C14480078EA
:10EE50008642F0D3114800780E490870002010490E
:10EE60000870002606E0B0000F490858B1000A4AB1
:10EE70005050761C074800788642F4D307E00548D6
:10EE800001780548F9F70CFA002002490870FEBD28
:10EE9000C40700207A000020F01000207800002035
:10EEA00079000020F80C00200009002010B505F0C2
:10EEB000A1F910BD00BF704710B504468020204363
:10EEC00001460320400205F04FF810BD10B5102197
:10EED0000320400205F048F810BD000010B50224E0
:10EEE000024805F091F80446204610BD01060000D6
:10EEF00010B50021014805F037F810BD01060000EB
:10EF000010B50446802020430146024805F02CF845
:10EF100010BD00000106000010B51021014805F0E9
:10EF200023F810BD0106000030B503460C46002151
:10EF3000002000BF06E08D0065599D4200D10120F0
:10EF40004D1CE9B29142F6DB30BD00002E4800783E
:10EF5000401C2D4908702D480078401C2B49087032
:10EF60002B480078401C2A4908702A480068401C39
:10EF70002849086008460068FF219131884202D97B
:10EF800000202449086020480078C82802D90020C1
:10EF90001D4908701D480078842802D900201B49AB
:10EFA00008701B480078502802D9002018490870C2
:10EFB000194818490968405C1849087018481249EE
:10EFC0000978405C17490870174810490978405C77
:10EFD0001649087016480E490978405C15490870B2
:10EFE000154809490978405C1449087014480649D5
:10EFF0000978405C13490870134803490978405C5C
:10F000001249087070470000BB060020BC060020B3
:10F01000BD060020C006002003C80100B406002081
:10F0200093C90100B50600205BCA0100B6060020A6
:10F03000A7CB0100B8060020DFCA0100B7060020F8
:10F04000F7CB0100B9060020BFCC0100BA060020B2
:10F0500010B50446204600F051FA204600F002F8B0
:10F0600010BD000010B50446B148007800287DD1DD
:10F07000B0480088B049884278DAB0480078002863
:10F080004FD0AF480078002803D0AA480088AD4987
:10F090000880AD480078002818D1A6480188A94802
:10F0A00000881930814206D30120A7490870A14881
:10F0B0000088A44908809F480088A249098888429E
:10F0C0001CDA9C4800889F49088017E09D48018809
:10F0D000984800881930814206D300209A49087068
:10F0E0009448008897490880924800889549098883
:10F0F000884203DD8F480088924908809248007852
:10F10000002857D191480078042803D08C48007813
:10F11000002807D087480088822803DA05208B4919
:10F120000870A1E089480078032803D0844800785B
:10F13000002809D07F480088FF211931884203DA6E
:10F140000420824908708FE080480078022803D0AC
:10F150007B48007800280AD076480088FF21AF312C
:10F16000884204DA0320794908707DE0DFE07748BF
:10F170000078012803D072480078002808D06D4834
:10F1800000887349884203DA0220704908706BE0F6
:10F190006E480078002803D069480078002863D0C2
:10F1A000644800883721090188425DDA01206749F7
:10F1B000087059E064480078012855D16348007808
:10F1C000012803D05E480078002809D059480088FB
:10F1D00037210901884203DB00205C49087043E0C5
:10F1E0005A480078022803D055480078002808D0F3
:10F1F000504800885649884203DB01205349087073
:10F2000032E052480078032803D04D4800780028A7
:10F2100009D048480088FF21AF31884203DB022033
:10F220004A49087020E049480078042803D044483F
:10F230000078002809D03F480088FF211931884212
:10F2400003DB0320414908700EE0404800780528A0
:10F2500003D03B480078002806D036480088822832
:10F2600002DB042039490870FDF74EF9394988421C
:10F270005DD3394800880019374908803048007844
:10F28000002808D000202E490870334908802F48F4
:10F2900000783249087000F0FFFC00281FD12E488A
:10F2A00000882F49884239DB00202B4908802B48F1
:10F2B000007826490978884205DA28480078401CF9
:10F2C000264908702AE025480078204909788842B4
:10F2D00024DD22480078401E204908701EE01E48A8
:10F2E00000882049884219DB00201B4908801B4800
:10F2F000007816490978884205DA18480078401CD9
:10F30000164908700AE015480078104909788842C3
:10F3100004DD12480078401E104908700F4800783C
:10F320000A490978884202D100200B49088010BDA3
:10F330000B00002002000020102700001200002017
:10F3400008000020040000200A0000200600002021
:10F3500076020000B80B0000180000200700002013
:10F36000C05D0000407E050000200B4908700B497D
:10F37000087001200A4908700A49087000200A49EB
:10F3800008700A4908700A4908800A4908800A4931
:10F3900008800A4908707047060000200700002016
:10F3A00008000020090000200A0000200B000020B7
:10F3B0000C0000200E000020100000201200002091
:10F3C00000200B4908700B49087001200A49087099
:10F3D0000A49087000200A4908700A4908700A4959
:10F3E00008800A4908800A4908800A49087070475D
:10F3F000060000200700002008000020090000206F
:10F400000A0000200B0000200C0000200E0000204D
:10F410001000002012000020F1B5002631480078CD
:10F42000002804D00320F9F797FF2F4908802F48C0
:10F43000008819284FD300202C4908802C480078D8
:10F44000142831D20320F9F787FF06460A213046F7
:10F45000F8F78CFE052901DB701D86B2002407E059
:10F4600060002449085AB04200DD05E0601CC4B2C7
:10F470001F4800788442F3DB00BF1D48057808E090
:10F48000681E40001B49085A69001A4A5052681EFB
:10F49000C5B2A542F4DC600016490E52144800784B
:10F4A000401C1349087016E00027052405E06000A1
:10F4B0001049085AC719601CC4B20F2CF7D30A218F
:10F4C0003846F8F73DFE08490880002008490870D2
:10F4D0000120094908700548018800980818034967
:10F4E0000880F8BD0900002002000020160000205E
:10F4F0000000002080070020120000202349098816
:10F50000234A91422BDB0021224A1180224A11809A
:10F5100022490988AF221201914207DC204909786B
:10F52000002916D01D490988914212DD02211D4A89
:10F53000117000211C4A117005211C4A1170002114
:10F54000174A117001211A4A11700021194A1170CD
:10F550001AE0124909880918104A118014E00021A4
:10F560000C4A11800D4A11800B490988124A9142B8
:10F5700005DD00210B4A1170094A117004E00649AB
:10F5800009880918044A1180704700000200002011
:10F59000102700000E0000200C00002010000020AA
:10F5A000090000200B0000200600002007000020BA
:10F5B000080000200A000020B80B00000148007875
:10F5C00070470000F40800200148007A70470000EE
:10F5D000F40800200148807870470000F4080020FB
:10F5E00001480088704700006C000020F8B5002337
:10F5F000002500950024002200BF94E001259D40D5
:10F60000ACB20D8825400095009DA5426FD11A46E9
:10F610008D79012D0DD1464D03263602AD192D5C95
:10F62000012696403543424E03273F02F6193554D2
:10F630000CE03F4D03263602AD192D5C01269640A5
:10F64000B5433B4E03273F02F6193554CD78002DC4
:10F650004ED1374D60352D5CCE78002E01D101267C
:10F6600000E000269640B543314E603635548D7823
:10F67000002D2ED12E4D19267601AD192D5C8E78D8
:10F68000002E01D1012600E000269640B543284E09
:10F6900019277F01F61935540D79002D0ED1244D0F
:10F6A00050352D5C0E79002E01D1012600E0002698
:10F6B0009640B5431E4E5036355423E01C4D503510
:10F6C0002D5C0E7996403543EEB2194D50352E54CF
:10F6D00018E0174D19267601AD192D5C8E789640ED
:10F6E0003543134E19277F01F61935540AE018E007
:10F6F0000F4D60352D5CCE7896403543EEB20C4D03
:10F7000060352E544D79012D0AD1094D30352D5CCF
:10F71000012696403543EEB2054D30352E5400E0BB
:10F7200000BF5D1CABB2082B00DA67E7F8BD000034
:10F7300000000440FFB5074615461E460024384623
:10F74000019900F01FF8002802D0012004B0F0BD9C
:10F7500000240CE00A2060430949085CB04204D14F
:10F760002946204600F05EF807E0601C84B20A20BB
:10F7700060430349085C0028ECD100BF0020E5E7A6
:10F78000180100200246002A03D1402901DD012092
:10F790007047032A03D1022901DD0120F8E7042A7A
:10F7A00003D1202901DD0120F2E7052A03D1202918
:10F7B00001DD0120ECE70C2A03D1102901DD012035
:10F7C000E6E70D2A05D1012903DD402901DA0120F0
:10F7D000DEE70E2A03D1202901D10120D8E700203D
:10F7E000D6E7000010B5064A03231B02D218125CAC
:10F7F0008A43034B032424021B191A5410BD000032
:10F800000000044010B5064A03231B02D218125C04
:10F810000A43034B032424021B191A5410BD000091
:10F820000000044070B502460020B1E00A235343B3
:10F830005A4C1B195B1C440004191B199B788B4202
:10F840007DD10A235343554C1B195B1C44000419FA
:10F850001B195B78082B33D10A2353434F4C1B19D8
:10F860005B1C440004191B574D4C4E4D6419E35C5E
:10F87000012423430A245443484D6419641C450061
:10F8800045196457464D474EAD192B550A2353432E
:10F89000424C1B195B1C440004191B57404C354655
:10F8A0006419E35C022423430A2454433B4D641946
:10F8B000641C450045196457394DAD192B5564E05A
:10F8C0000A235343354C1B195B1C440004191B19B4
:10F8D0005B78092B34D10A235343304C1B195B1C32
:10F8E000440004191B572E4C2E4D6419E35C402430
:10F8F00023430A245443294D6419641C45004519C7
:10F900006457274D274EAD192B550A235343234CDB
:10F910001B195B1C440004191B57214C3546641904
:10F92000E35C8024A3430A2454431C4D6419641CE3
:10F930004500451964571A4DAD192B5525E025E0B2
:10F940000A235343154C1B195B1C440004191B5715
:10F95000134C144D6419E35C0A2454430F4D64198D
:10F96000641C45004519641965780124AC402343A3
:10F97000DCB20A235343094D5B195B1C4500451952
:10F980005B57074D074EAD19EC5404E0431CD8B249
:10F99000032800DA4AE700BF70BD0000180100200C
:10F9A0000000044075080000F8B50024FCF7C6FD0F
:10F9B000012861D100F0C4FA044664220721002026
:10F9C00002F0CAFD012C21D100F038FB00280ED036
:10F9D00000F0EAFA054600F0DBFA0646012003468D
:10F9E000024629460090304604F05EFC50E000F0EC
:10F9F000DBFA054600F0CCFA064601200023024659
:10FA000029460090304604F04FFC41E0022C21D101
:10FA100000F014FB00280ED000F0C6FA054600F0F6
:10FA2000B7FA0646012003460246294600903046B2
:10FA300004F03AFC2CE000F0B7FA054600F0A8FA12
:10FA40000646002001231A4629460090304604F05D
:10FA50002BFC1DE000F0F2FA054600F0A5FA064680
:10FA600000F096FA0746012003462A4631460090E8
:10FA7000384604F019FC0BE000200346024601461C
:10FA8000009004F011FC00220721104602F064FDF2
:10FA9000F8BD0000FEB547480078012809D1FCF701
:10FAA0004DFD012802D1FCF787FB82E0FCF7ACFC9E
:10FAB0007FE0FCF743FD012879D1FCF725FD3E49A5
:10FAC000884271D33D480088032805DA3B48008806
:10FAD000401C3A49088011E000203849088000F0B5
:10FAE0005DFA054600F078FA06460A21F8F728FB89
:10FAF00004462A462146012007F0AEFE00F08EFBA8
:10FB0000054600F04BFB07460A21F8F719FB0446AF
:10FB100000F044FA06462A46214606F063F9FFF74C
:10FB200043FF00F007FA04462146012005F03EFF9E
:10FB300000F04CFA0546FF21F531F8F717FBC4B287
:10FB40002146012005F06EFBFFF738FD0446FFF764
:10FB500047FD0546FFF73EFD064623462A46314649
:10FB6000012004F07BFE00F09DF8044621460120B0
:10FB700008F0C2F800F02CFB044600F06BFA0546D2
:10FB800000F01EFA064600F029FB074600F068FA6E
:10FB900033463A460146009501940290012007F051
:10FBA000D3F906E003E0FFE7FCF772FB01E0FCF7A6
:10FBB0002BFCFEBDAC000020B80B0000660000204E
:10FBC0000149086070470000E8060020024800680C
:10FBD000401C014908607047E4060020F3B581B07D
:10FBE000064600200E49086000F01EF8044600F0AA
:10FBF0001BF805462F1B3046029903F043FC00908A
:10FC00000AE000F011F805462F1B0648006800289E
:10FC100002D004480068804700988742F1D3FEBDB7
:10FC2000E4060020E8060020014800687047000054
:10FC3000E40600200B490978012901D101200FE0D9
:10FC400008490978022901D1022009E0054909780B
:10FC5000032901D1042003E00121024A117001208F
:10FC6000704700007D06002010B5094B1B8899B233
:10FC70000A12C8B2D3433133064C2370C343233333
:10FC8000637013465633A37003467133E37010BD9F
:10FC9000AC06002083060020014800887047000061
:10FCA0003200002001480078704700007B000020EF
:10FCB00010B5002205210648FBF7DEF804020122F8
:10FCC00005210348FBF7D8F8201880B210BD0000CA
:10FCD000C407002010B5062205210348FBF7CCF825
:10FCE000C006C00F10BD0000C407002010B50422DC
:10FCF00005210648FBF7C0F8040205221146034817
:10FD0000FBF7BAF8201880B210BD0000C40700202D
:10FD100010B5062205210248FBF7AEF8C01110BD50
:10FD2000C407002010B5022205210248FBF7A4F801
:10FD300010BD0000C407002010B5062205210348AD
:10FD4000FBF79AF88006C00F10BD0000C407002022
:10FD500010B5042202210348FBF78EF8C007C00F3C
:10FD600010BD0000C407002010B505220221034881
:10FD7000FBF782F8C007C00F10BD0000C4070020C9
:10FD800010B5002204210348FBF776F84006400F27
:10FD900010BD0000C407002010B500220121024858
:10FDA000FBF76AF810BD0000C407002010B501225F
:10FDB00011460248FBF760F810BD0000C4070020A0
:10FDC00010B5022203210248FBF756F810BD0000CF
:10FDD000C407002010B5032200210248FBF74CF8AD
:10FDE00010BD0000C407002010B5002211460248D3
:10FDF000FBF742F810BD0000C407002010B5042234
:10FE000000210248FBF738F810BD0000C4070020AD
:10FE100010B5012200210248FBF72EF810BD0000AA
:10FE2000C407002010B5052200210248FBF724F882
:10FE300010BD0000C4070020322815DA3C4989783B
:10FE4000012903DD01213A4A517070E0384989786F
:10FE5000002905DD2F286ADC0021354A517066E053
:10FE60000021334A517062E03E2817DA322815DB50
:10FE70002F498978022903DD02212D4A517056E06D
:10FE80002B498978012905DD3B2850DC0121284ACE
:10FE900051704CE00121264A517048E0502817DA91
:10FEA0003E2815DB22498978032903DD0321204AF6
:10FEB00051703CE01E498978022905DD4D2836DC69
:10FEC00002211B4A517032E00221194A51702EE082
:10FED000622817DA502815DB15498978042903DDD3
:10FEE0000421134A517022E011498978032905DD64
:10FEF0005F281CDC03210E4A517018E003210C4AD4
:10FF0000517014E073280FDA62280DDB08498978F4
:10FF1000042905DD70280ADC0421054A517006E039
:10FF20000421034A517002E00521014A51707047D3
:10FF3000F408002001480078704700000700002006
:10FF400001480078704700009B000020F8B50026AB
:10FF500000240025FDF710FA07460A21F8F7F0F80B
:10FF6000054609480068854200D303E0064800685A
:10FF7000461B34467D200001844200D304460348DA
:10FF800004600068F8BD0000D4000020D00000200C
:10FF90000148007870470000A40000200148007963
:10FFA000704700009400002001484078704700002E
:10FFB000A4000020014880797047000094000020D0
:10FFC00001484079704700009400002001480088F3
:10FFD000704700002200002010B50024FFF7DEFF6C
:10FFE00000280AD10A4800880A49884202DB0846EC
:10FFF000074908800648048808E005480088FCF79F
:020000040001F9
:1000000069FF84B20448844200DB0446204610BDE8
:1000100034000020C6070000CE040000002005497F
:100020000988054A914202DB1146024A11800149C2
:100030000888704734000020C60700000148007897
:1000400070470000B50600200148007870470000A6
:10005000B7060020014800797047000070000020BA
:1000600070B500240A48C07901280CD108490888D5
:10007000FCF786FB05460A21F8F778F884B2632C72
:1000800003DD632401E002480488204670BD0000BF
:1000900070000020014800887047000070000020B8
:1000A00010B500240A2103480088F8F75FF884B2ED
:1000B000204610BD02000020014800787047000073
:1000C0000B00002010B50024044803F09DFF002819
:1000D00001D0012400E00024204610BD03070000E9
:1000E00010B50024054803F08FFF002802D001203E
:1000F000044601E00020044610BD00000507000092
:1001000010B50024054803F07FFF002802D001202D
:10011000044601E00020044610BD0000070700006F
:1001200010B50024062003F06FFF002801D0012441
:1001300000E00024204610BD10B50024054803F05F
:1001400063FF002802D00120044601E0002004469D
:1001500010BD00000607000010B50024044803F09D
:1001600053FF002801D0012400E00024204610BDE8
:100170000305000010B50024044803F045FF0028E3
:1001800001D0012400E00024204610BD0405000039
:1001900001488079704700007000002070B500248D
:1001A000FFF7FCFE002803D1FDF7E6F804460DE05A
:1001B000FFF7F4FE012806D1FDF7DEF80546FCF74F
:1001C00089FE044602E0FDF7D7F80446204670BDDC
:1001D00001484079704700007000002070B500248D
:1001E0000A48C07901280CD108494888FCF7C8FAA8
:1001F00005460A21F7F7BAFF84B2632C03DD6324B6
:1002000001E002484488204670BD000070000020D4
:1002100001484088704700007000002070B500243D
:10022000FFF7BCFE002803D1FDF7B8F804460FE045
:10023000FFF7B4FE012807D10020FDF7AFF805460F
:10024000FCF748FE044603E00020FDF7A7F804464B
:10025000204670BD0148007870470000380000203B
:1002600070B505460024032D00D170BD002D01D0CE
:10027000012D1BD181210320800203F075FE802116
:10028000134803F071FE32211248FFF7A7FC002447
:1002900009E0A200104BD2189178A200985A03F0FE
:1002A00063FE601CC4B23B2CF3DB0FE0022D0DD1CA
:1002B000002409E0A200094BD2189178A200985AB4
:1002C00003F052FE601CC4B23B2CF3DB00BFCCE752
:1002D00002060000A08601009CC0010088C1010048
:1002E000F8B5002100240023002200BF0AE0012508
:1002F0008D40ABB205881D402C469C4200D10A4679
:100300004D1CA9B21029F2DB0588FF2D1FDC284DFA
:100310006D7E0688B543264E757635462D7E068859
:10032000B543234E357635466D7E8678F607F60F53
:10033000964035431E4E757635462D7E86780227CB
:100340003E40760896403543194E357622E0184DEA
:10035000ED7E0688B543164EF5763546AD7E0688A9
:10036000B543134EB5768578ED07ED0F1646083E7A
:10037000B5400F4EF67E35430D4EF5768578022654
:1003800035406D081646083EB540094EB67E3543E9
:10039000074EB5760025009505E000BF6D462D7827
:1003A0006D1CEEB200966D462D78012DF5D9F8BD85
:1003B000206B0440C107C90F002905D00021394A2C
:1003C0001171002238490A7102210140002905D02B
:1003D0000021344A1172002233490A72042101407B
:1003E000002905D000212F4A117300222E490A73DB
:1003F00008210140002905D000212A4A1174002259
:1004000029490A7410210140002905D00021254AFC
:100410001175002224490A7520210140002905D0C8
:100420000021204A117600221F490A76402101400E
:10043000002904D000221B494A711B494A718021BE
:100440000140002904D0002216494A7216494A7216
:10045000FF2101310140002904D0002211494A73D3
:1004600011494A73012149020140002904D00022A8
:100470000C494A740C494A7401218902014000293F
:1004800004D0002207494A7507494A750121C9026B
:100490000140002904D0002202494A7602494A76E6
:1004A000704700000060004000610040C107C90FB4
:1004B000002905D001223C490A7100213B4A1171F3
:1004C00002210140002905D0012237490A7200218A
:1004D000364A117204210140002905D00122324917
:1004E0000A730021314A117308210140002905D007
:1004F00001222D490A7400212C4A11741021014057
:10050000002905D0012228490A750021274A1175C2
:1005100020210140002905D0012223490A7600212B
:10052000224A117640210140002905D001221E49AE
:100530004A7100221D494A7180210140002905D0DD
:10054000012219494A72002218494A72FF210131D9
:100550000140002905D0012213494A7300221349A2
:100560004A73012149020140002905D001220E49A8
:100570004A7400220D494A74012189020140002970
:1005800005D0012208494A75002208494A7501210F
:10059000C9020140002905D0012203494A76002200
:1005A00002494A7670470000006100400060004048
:1005B00010B50C480078002803D00B4A50689168A9
:1005C000884708484078002803D0084A5068916856
:1005D000884704488078002803D0054A506891680D
:1005E000884710BD0060004068020020E80300203A
:1005F0006805002010B508480079002803D0074A94
:1006000010695169884704484079002803D0044A9A
:1006100050689168884710BD006000406802002063
:10062000F403002010B50848007A002803D0074AD8
:10063000D069116A88470448407A002803D0044AE8
:1006400050689168884710BD006000406802002033
:100650000004002010B50848007B002803D0074A9A
:10066000906AD16A88470448407B002803D0044A36
:1006700050689168884710BD006000406802002003
:100680000C04002010B50848007C002803D0074A5D
:10069000506B916B88470448407C002803D0044A83
:1006A00050689168884710BD0060004068020020D3
:1006B0001804002010B50848007D002803D0074A20
:1006C000106C516C88470448407D002803D0044AD0
:1006D00050689168884710BD0060004068020020A3
:1006E0002404002010B50848007E002803D0074AE3
:1006F000D06C116D88470448407E002803D0044A1E
:1007000050689168884710BD006000406802002072
:100710003004002010B50848407F002803D0074A65
:100720005068916888470448007F002803D0044A35
:10073000906DD16D884710BD006000403C040020E2
:100740006802002010B508484078002803D0074A06
:1007500050689168884704480078002803D0044A0C
:10076000506E916E884710BD206000404804002004
:100770006802002010B509480079002803D0084A13
:10078000106F516F88470548001D4078002803D03E
:10079000044A50689168884710BD000020600040FE
:1007A000680200205404002010B5034AD06F78324C
:1007B0009168884710BD00006802002010B5024A09
:1007C00050689168884710BDEC02002010B50948B8
:1007D000007C002803D0084A506891688847054883
:1007E00010304078002803D0044A50689168884748
:1007F00010BD000020600040F802002078040020B6
:1008000010B5024A50689168884710BD0403002063
:1008100010B5024A50689168884710BD1003002047
:1008200010B50948007F002803D0084A5068916835
:10083000884705481C304078002803D0044A506897
:100840009168884710BD0000206000401C03002014
:100850009C04002010B50C480078002803D00B4AF7
:1008600050689168884708484078002803D0084AB3
:1008700050689168884704488078002803D0054A6A
:1008800050689168884710BD4060004028030020F0
:10089000A80400202806002010B50D480079002883
:1008A00003D00C4A5068916888470948001D407879
:1008B000002803D0084A5068916888470448001D02
:1008C0008078002803D0054A50689168884710BD99
:1008D0004060004034030020B404002034060020AF
:1008E00010B50D48007A002803D00C4A5068916872
:1008F0008847094808304078002803D0084A5068E3
:1009000091688847044808308078002803D0054A59
:1009100050689168884710BD406000404003002047
:10092000C00400204006002010B50D48007B0028C0
:1009300003D00C4A50689168884709480C304078C9
:10094000002803D0084A50689168884704480C3052
:100950008078002803D0054A50689168884710BD08
:10096000406000404C030020CC0400204C060020D6
:1009700010B50D48007C002803D00C4A50689168DF
:100980008847094810304078002803D0084A50684A
:1009900091688847044810308078002803D0054AC1
:1009A00050689168884710BD40600040580300209F
:1009B000D80400205806002010B5024A50689168FB
:1009C000884710BD6403002010B50948007E002848
:1009D00003D0084A50689168884705481830407825
:1009E000002803D0044A50689168884710BD000071
:1009F0004060004070030020F004002010B509485A
:100A0000007F002803D0084A50689168884705484D
:100A10001C304078002803D0044A50689168884709
:100A200010BD0000406000407C030020FC0400205A
:100A300010B508480078002803D0074A506891682C
:100A4000884704484078002803D0044A50689168D9
:100A5000884710BD60600040880300200805002022
:100A600010B509480079002803D0084A50689168F9
:100A700088470548001D4078002803D0044A506884
:100A80009168884710BD000060600040940300201A
:100A90001405002010B50948007A002803D0084A40
:100AA000506891688847054808304078002803D08E
:100AB000044A50689168884710BD0000606000409B
:100AC000A00300202005002010B5024A506891685C
:100AD000884710BDAC03002010B5024A50689168E9
:100AE000884710BDB803002010B50948007D0028D4
:100AF00003D0084A50689168884705481430407808
:100B0000002803D0044A50689168884710BD00004F
:100B100060600040C40300204405002010B509486F
:100B2000007E002803D0084A50689168884705482D
:100B300018304078002803D0044A506891688847EC
:100B400010BD000060600040D00300205005002070
:100B500010B50948007F002803D0084A5068916802
:100B6000884705481C304078002803D0044A506864
:100B70009168884710BD000060600040DC030020E1
:100B80005C05002010B5FE4800688079002806D07A
:100B900001286ED002286DD003286CD104E2F848F9
:100BA0000068407903000AF00FFD0A0614BC2BBC54
:100BB00047BC67BC9BBC07F05FFB0020F04909689D
:100BC000C873EF4800684079401CED4909684871D6
:100BD000AEE0EC490969EA4A1268D27A885C07F00B
:100BE000C3FBE74800684079401CE5490968487143
:100BF000E34800684079401CE1490968487197E082
:100C000001F012FE002810D107F0AEFBDC480068AE
:100C10004079401CDA4909684871D9480068407930
:100C2000401CD7490968487105E007F04FFB0020D8
:100C3000D349096848717BE001F0F6FD002811D125
:100C4000012007F091FBCE4800684079401CCC4958
:100C500009684871CA4800684079401CC849096859
:100C6000487105E007F032FB0020C549096848716A
:100C70005EE05FE0FEE0A3E101F0D6FD002828D1B0
:100C8000BF490968C97A24225143BF4A12688918AA
:100C9000BB4A1268D27B885C07F066FBB8480068E4
:100CA000C07B401CB6490968C873B5480068C07B62
:100CB000242814D3B24800684079401CB049096820
:100CC0004871AF4800684079401CAD4909684871D7
:100CD00005E007F0FBFA0020A9490968487127E000
:100CE00001F0A2FD002815D1A5480068C07A401C7B
:100CF000A3490968C872A2480068C07AA149097866
:100D0000884207DB00209E490968C87201209C497F
:100D10000968887107F0DAFA002099490968487172
:100D200006E007F0D3FA002095490968487100BF32
:100D300000BF4FE192480068407903000AF044FC8C
:100D4000080513912A914791709107F095FA0020B8
:100D50008B490968C8738A4800684079401C8849F3
:100D60000968487184E087490969854A1268D27A1E
:100D7000885C07F0F9FA824800684079401C804995
:100D8000096848717E4800684079401C7C490968C0
:100D900048716DE001F048FD002811D1262007F0D0
:100DA000E3FA774800684079401C75490968487142
:100DB000734800684079401C71490968487105E032
:100DC00007F084FA00206E490968487150E001F08C
:100DD0002BFD00281DD1012007F0C6FA68480068E5
:100DE000C07B401C66490968C87365480068C07BC1
:100DF000242814D3624800684079401C604909687F
:100E000048715F4800684079401C5D490968487135
:100E100005E007F05BFA002059490968487127E0AE
:100E200001F002FD002815D155480068C07A401C29
:100E300053490968C87252480068C07A5149097814
:100E4000884207DB00204E490968C87202204C49DD
:100E50000968887107F03AFA002049490968487121
:100E600006E007F033FA002045490968487100BFE1
:100E700000BFAFE042480068407903000AF0A4FBDD
:100E80000805138B2A8B478B638B07F0F5F900203D
:100E90003B490968C8733A4800684079401C3849A2
:100EA000096848717EE037490969354A1268D27A83
:100EB000885C07F059FA324800684079401C304994
:100EC000096848712E4800684079401C2C4909681F
:100ED000487167E001F0A8FC002811D1252007F037
:100EE00043FA274800684079401C25490968487141
:100EF000234800684079401C21490968487105E091
:100F000007F0E4F900201E49096848714AE001F041
:100F10008BFC002810D107F027FA194800684079A7
:100F2000401C174909684871154800684079401C01
:100F300013490968487105E007F0C8F90020104915
:100F4000096848712EE001F06FFC002815D10C48AB
:100F50000068C07A401C0A490968C87208480068DD
:100F6000C07A08490978884207DB002004490968EB
:100F7000C872032002490968887107F0A7F905E0E3
:100F80006C070020681D002068070020002012491F
:100F90000968487106E007F099F900200E490968D0
:100FA000487100BF00BF15E000200B490968887137
:100FB000094909684871062007490968C87009E0AD
:100FC00007F084F90020044909684871024909685A
:100FD000887100BF00BF10BD6C07002010B56A48C3
:100FE0000068407903000AF0EFFA090610C627C628
:100FF00044C6608EC60007F03FF963480068407938
:10100000401C614909684871BCE0604909695E4A51
:101010001268D27A885C07F0A7F95B4800684079CB
:10102000401C594909684871574800684079401C7C
:10103000554909684871A5E001F0F6FB002811D177
:101040004F2007F091F9504800684079401C4E4904
:10105000096848714C4800684079401C4A49096851
:10106000487105E007F032F90020474909684871E6
:1010700088E001F0D9FB002810D107F075F942484B
:1010800000684079401C4049096848713E48006842
:101090004079401C3C490968487105E007F016F9A1
:1010A00000203949096848716CE001F0BDFB002857
:1010B00022D135480068C07A401C33490968C8729B
:1010C00031480068C07A3149097888420FDB002036
:1010D0002D490968C8722C4800684079401C2A498B
:1010E00009684871002028490968486208E0002022
:1010F00025490968487103E00020234909684871BF
:1011000007F0E4F83EE020480068407C002816D054
:101110001E48C068002803D01C48C16819208847B1
:101120000020194909684862174909684871164939
:1011300009688871052014490968C8701AE01248C6
:101140000068406A282807D20F480068406A401C9F
:101150000D49096848620DE000200B4909684862A2
:1011600009490968487108490968887105200649D4
:101170000968C87006E007F0A9F80020024909686C
:10118000487100BF00BF10BD6C070020681D002023
:1011900010B50024F7480068807A01287ED1F54810
:1011A0000068C07900287AD0F24800688079002869
:1011B00004D0012874D0022873D191E1ED48006871
:1011C000007B24286ED2EB480068C07901287AD1D0
:1011D000002475E0E7480068C07A24214843E649C6
:1011E00009684018E3490968097B415CE1480068E7
:1011F000C07A24225043E14A12688018DD4A1268FE
:10120000127B805C814229D0DA480068C07A2421B0
:101210004843DA4909684018D6490968097B415CA6
:10122000D4480068C07A24225043D34A12688018F8
:10123000D04A1268127B8154CE480068407B242833
:1012400005D3CC480068007BCA4909684873C9487F
:101250000068007BC7490968887308E0C5480068D2
:10126000407B242803D20120C24909688871C14803
:101270000068007B401CBF4909680873BD480068CE
:10128000007B242808D3BB480068407B242803D275
:101290000120B84909688871B64805E0D3E1CDE17D
:1012A00069E0BAE138E00EE00068007B242804D24F
:1012B000B04800688079012800D103E0601CC4B206
:1012C000242C87D356E0002413E0AA480068C07A93
:1012D00024214843A94909684018015DA5480068D0
:1012E000C07A24225043A44A126880180155601C19
:1012F000C4B2242CE9D300209E49096848732320F6
:101300009C490968887301209A49096888712420DA
:101310009849096808732DE0002096490968087308
:1013200094480068C07A401C92490968C872914884
:101330000068C07A92490978884217DB8D480068B6
:10134000007C012804D102208A490968887106E0DE
:10135000002088490968887186490968C871002099
:1013600084490968C8728349096808740020814962
:101370000968487161E17F480068407903000AF01C
:1013800023F9080513A62AA651A68EA6012079499D
:101390000968087406F070FF764800684079401CC0
:1013A00074490968487199E075490969714A126878
:1013B000D27A885C06F0D8FF6E4800684079401CFD
:1013C0006C49096848716B4800684079401C69495C
:1013D0000968487182E001F027FA00281BD16549AD
:1013E0000968497B491CC8B206F0BEFF6148006825
:1013F000407B60490968C8735E4800684079401CBA
:101400005C49096848715B4800684079401C59494B
:101410000968487105E006F059FF00205549096840
:1014200048715BE001F000FA00282BD151490968AE
:10143000C97A24225143504A126889184D4A1268C9
:10144000D27B885C06F090FF4A480068C07B401C55
:1014500048490968C87347480068C07B454909681E
:10146000897B88421ADD434800684079401C414925
:10147000096848713F4800684079401C3D49096847
:1014800048710BE006F022FF3A480068407B39497A
:101490000968C87300203749096848711EE001F0E7
:1014A000C3F900280CD133490968887124203149D7
:1014B0000968C8732F49096848732E4909688873F9
:1014C00006F004FF00202B490968487106E006F089
:1014D000FDFE002027490968487100BF00BFACE04D
:1014E00024480068407903000AF06EF808050F8E62
:1014F000268E4C8E688E06F0BFFE1E48006840792E
:10150000401C1C490968487185E01D490969194A50
:101510001268D27A885C06F027FF16480068407986
:10152000401C144909684871124800684079401C01
:101530001049096848716EE001F076F9002811D170
:10154000252006F011FF0B4800684079401C09492E
:1015500009684871074800684079401C05490968D6
:10156000487105E006F0B2FE0020024909684871A2
:1015700051E000006C07002068070020640700208D
:10158000681D002001F050F9002810D106F0ECFE93
:10159000644800684079401C6249096848716148A4
:1015A00000684079401C5F490968487105E006F011
:1015B0008DFE00205B49096848712CE001F034F988
:1015C00000281AD157480068C07A401C554909685C
:1015D000C87254480068C07A5349097888420CDBC5
:1015E000002050490968C8724E49096888714D4900
:1015F000096848714B490968C87106F067FE002008
:1016000048490968487106E006F060FE0020454937
:101610000968487100BF00BF0FE006F057FE0020C8
:101620004049096848713F49096888713D4909681E
:1016300008733C490968C87200BF71E0002039494D
:10164000096888726CE037480068807A022867D1A0
:1016500034480068007A00285ED03248006840793B
:10166000002804D001280CD0032846D11BE006F046
:1016700003FE2C4800684079401C2A4909684871DB
:1016800049E0002006F070FE264800684079401CC2
:10169000244909684871234800684079401C214961
:1016A0000968487137E006F0B1FD002812D11D48E5
:1016B00000684078401C1B49096848701948006858
:1016C0004078032812D301F04FF90020154909682A
:1016D00048700BE00020134909680872AA201149DC
:1016E0000968887000200F490968487006F0EEFD0F
:1016F00000200C49096848710DE006F0E7FD002064
:10170000084909684871074909684870AA200549CD
:101710000968887000BF03E00020024909688872E8
:1017200010BD00006C070020681D0020F8B50446BD
:101730000D4600260C2060431D49085C002801D09E
:101740000120F8BD0C2060431949401885600C2029
:10175000604340188068002801D10120F1E7012191
:101760000C206043124A115400222046E317DB0E7E
:101770001B185B115B01E31A9B000E4FDB19E71787
:10178000FF0E3F197F11DA5509F050FF0022204665
:10179000E317DB0E1B185B115B01E31A9F00064B7E
:1017A000FB18E717FF0E3F197F11DA553046C8E7DF
:1017B00068020020006000400061004000BFFEE7BA
:1017C00009480088401C08490880084600880749E5
:1017D000884208DD06480078062804D008460249F9
:1017E000088001208870704790000020DC05000010
:1017F0009B00002010B50B488078012810D10A48C2
:101800000078012802D1094802F0D6F9064800788C
:10181000022802D1054802F0CFF9002002490870E1
:1018200010BD0000900000209B000020A4000020BC
:101830007047000010B500F0A5FD012803D100207D
:1018400001490880887010BD90000020F0B5054661
:101850000E46174600243A463146284600F0A0FDC1
:1018600000BF42E000202101394A12685052210194
:10187000374A12688918488000212001344A1268CA
:10188000801881802001324A12688018C1802001AE
:101890002F4A12688018017220012D4A12688018A0
:1018A000417220012A4A1268801881722001284A58
:1018B00012688018C17200202101254A1268891817
:1018C000087300212001224A126880184173002009
:1018D00021011F4A126889188873002120011C4ABF
:1018E00012688018C173601CC4B21A484078A042C4
:1018F000B8DC64201849096808807D20C0001649BA
:101900000968488015481449096888807D200001CD
:1019100011490968C88010490968088110480E49B2
:10192000096848810F480C490968888140000A49C4
:101930000968C8813220084909680882FF20F5300B
:10194000054909684882044909688882F0BD000099
:10195000F8060020EC060020F40600204C040000ED
:10196000102700003075000038B5002404E0002086
:101970000D490855601C84B2282CF8D30121684613
:10198000417001706A4609490748FFF75FFF7D21F2
:10199000C900322000F0F4F80549064800F00EF9BD
:1019A000054800F0DDF838BDD81600200CC4010051
:1019B00028230000B80B00001027000010B51E48B7
:1019C0000078002803D101201B4908701EE01A4846
:1019D0000078012803D102201749087016E0164844
:1019E0000078022803D10320134908700EE0124842
:1019F0000078032803D104200F49087006E00E4840
:101A00000078042802D100200B4908700A480078A9
:101A100007280AD1FEF7CEFA002803D10120074992
:101A2000887102E000200549887103480078052884
:101A300001D1FAF703FF10BD9B00002094000020A5
:101A4000F8B500240025002631480078002803D18D
:101A500005202F49087016E02D480078052803D18D
:101A600006202B4908700EE029480078062803D18B
:101A700007202749087006E025480078072802D18A
:101A80000020234908702248007801280BD1012446
:101A9000172500261F48012332462946009020467C
:101AA00001F016FD33E01A48007802280CD1012419
:101AB0003B2500261748401C01233246294600904A
:101AC000204601F005FD22E01148007803280DD1E1
:101AD000FEF764FA002803D101200F49087102E0E3
:101AE00000200D49087109F041FD10E00848007818
:101AF00004280CD1FEF764FA002803D1012006491E
:101B0000487102E000200449487109F02FFDF8BD3A
:101B10009B000020A40000209400002010B5044683
:101B2000230009F051FD091606090C0D0E0F1415BE
:101B30001900FFF785FF10E0FFF740FF0DE00CE014
:101B40000BE00AE001F0ACFC08F012F805E004E05C
:101B500003E0FFF735FE00E000BF00BF10BD00004E
:101B600001460020054A126892898A4201DB012061
:101B700002E0024A1268D18170470000F40600209A
:101B8000024600200C4B1B681B8A934201DD01209A
:101B900010E08A4201DB01200CE0074B1B689B88A8
:101BA0008B4201DC012005E0034B1B681A80024BCD
:101BB0001B68598070470000F40600200246002090
:101BC0000C4B1B681B8A934201DD012010E08A4206
:101BD00001DB01200CE0074B1B685B88934201DBB3
:101BE000012005E0034B1B689A80024B1B68D980DB
:101BF00070470000F406002070B5044600250C2054
:101C00006043FE49096840184068002807D00C214D
:101C10006143FA4A126889184868804705460C20D3
:101C20006043F6490968085C002873D10C206043C2
:101C3000F249096840188068002874D02001F049F2
:101C400009684018C07A02280AD1032D08D10C2057
:101C50006043EA4A1268801881680120884762E080
:101C60002001E74909684018C07A02280AD1042DEA
:101C700008D10C206043E14A126880188168022074
:101C8000884750E02001DE4909684018C07A0228E0
:101C90000AD1052D08D10C206043D84A126880185B
:101CA0008168032088473EE02001D5490968401833
:101CB000C07A02280AD1062D08D10C206043CF4AF1
:101CC000126880188168042088472CE02001CC49E4
:101CD00009684018C07A02280AD1072D08D10C20C3
:101CE0006043C64A126880188168052088471AE058
:101CF0002001C34909684018C07A02280BD1082D79
:101D000009D10C206043BD4A126880188168062002
:101D1000884708E00DE00C206043B84A126880183C
:101D20008168002088472001B54909684018C572BC
:101D30000CE30C206043B1490968085C012873D1A9
:101D40000C206043AD49096840188068002874D0B1
:101D50002001AB4909684018C07A03280AD1022D36
:101D600008D10C206043A54A1268801881680120C0
:101D7000884762E02001A24909684018C07A042817
:101D80000AD1022D08D10C2060439C4A12688018A9
:101D900081680220884750E020019949096840186D
:101DA000C07A05280AD1022D08D10C206043934A3D
:101DB000126880188168032088473EE0200190491E
:101DC00009684018C07A06280AD1022D08D10C20D3
:101DD00060438A4A126880188168042088472CE092
:101DE0002001874909684018C07A07280AD1022DC6
:101DF00008D10C206043814A126880188168052050
:101E000088471AE020017E4909684018C07A0828EE
:101E10000BD1022D09D10C206043784A126880183A
:101E200081680620884708E00DE00C206043734A73
:101E3000126880188168002088472001704909686D
:101E40004018C57282E20C2060436C490968085C46
:101E50000228F7D1002D7DD1200169490968085A6F
:101E600068490968098A884275DA20016449096865
:101E7000085A0A3081B22001614A126811522001C9
:101E80005F490968085A5F490968098A884231DB55
:101E900020015B490968401840885A490968098847
:101EA000884227DB20015649096840184088554977
:101EB0000968498888421DDC00202101504A1268C7
:101EC0008918488020014E4909684018807A002806
:101ED000B8D10C206043494909684018806800283F
:101EE000B0D00C206043454A1268801881680120F8
:101EF00088472BE2200142490968085A414909688C
:101F0000098A88429EDB20013D49096840184088C3
:101F10003C4909688988884294DB2001384909686E
:101F20004018408837490968C98888428ADC0020FF
:101F30002101334A12688918488020013049096814
:101F40004018807A0028D4D10C2060432B490968BE
:101F5000401801E063E00BE080680028C9D00C2045
:101F60006043264A12688018816802208847EDE1A4
:101F700000202101224A1268891848802101204A44
:101F800012688918C872002120011D4A1268801841
:101F9000C18020011A4A1268801841722001184A33
:101FA000126880188172184801782001144A12685A
:101FB0008018017200202101114A12688918888056
:101FC00021010F4A12688918087321010C4A12680E
:101FD0008918487321010A4A1268891888730021F8
:101FE0002001074A12688018C1730C20604303491E
:101FF0000968401880680028B9D007E0F006002082
:10200000F8060020F4060020EC0600200C206043B7
:10201000CF4A1268801881680020884796E1012D18
:10202000A5D12001CB4909684018C07AA84225D023
:1020300000212001C74A1268801841800020210138
:10204000C44A12688918C8802001C249096840182A
:10205000C572C14800782101BE4A126889184872C9
:1020600000202101BB4A126889188880BA4801788B
:102070002001B84A12688018017267E12001B54951
:1020800009684018007AB4490978884220D0B248DB
:1020900000782101AF4A1268891808722001AD4901
:1020A00009684018407AAC490978884209D0200173
:1020B000A8490968401880882101A64A1268891831
:1020C000C88000212001A34A12688018818012E094
:1020D0002001A049096840188088A04988420AD296
:1020E00020019C490968401880880A302101994ADA
:1020F000126889188880200196490968401840882C
:10210000964988420AD220019249096840184088BD
:102110000A3021018F4A12688918488020018D49B0
:1021200009684018407A8C490978884205D0012016
:102130002101884A12688918887220018549096836
:1021400040184088864909680988884204DB0021D4
:102150002001804A1268115220017E490968401806
:10216000807A00287ED10C206043794909684018A4
:102170008068002877D02001764909684018408897
:10218000774909680989884214DB20017149096887
:102190004018007B00280DD10C2060436C4A126867
:1021A000801881680320884701202101694A12684C
:1021B00089180873200167490968401840886849F0
:1021C00009684989884214DB20016249096840187E
:1021D000407B00280DD10C2060435D4A12688018B6
:1021E000816804208847012021015A4A1268891811
:1021F00048732001574909684018408858490968C0
:102200008989884214DB2001524909684018807B83
:1022100000280DD10C2060434D4A12688018816857
:1022200005208847012021014A4A126889188873CD
:102230002001484909684018408849490968C98906
:10224000884210DB2001434909684018C07B002800
:102250007CD10C2060433E4A1268801881680620B9
:10226000884701E007E03BE001202101394A12687C
:102270008918C8736AE02001364909684018407A15
:1022800001282ED13448007802282AD12001314972
:1022900009684018C08832490968498A884255DB74
:1022A00020012C490968401880882D490968898ACD
:1022B00088424BDB0C206043254909684018806840
:1022C000002843D00C206043214A1268801881689E
:1022D00007208847002021011E4A12688918487289
:1022E00034E020011B4909684018407A02282DD1AA
:1022F00019480078012829D1200116490968401899
:10230000C08817490968898A88421FDB2001114962
:1023100009684018808812490968498A884215DB93
:102320000C2060430A4909684018806800280DD0D5
:102330000C206043064A126880188168082088478C
:1023400000202101034A12688918487270BD0000FC
:10235000F0060020F8060020EC060020F0FF000048
:10236000F406002010B5002400BF04E02046FFF76B
:1023700043FC601CC4B202484078A042F6DC10BDA9
:10238000EC06002010B50024044801F03DFE0028B2
:1023900000D000E00124204610BD0000030400002E
:1023A00010B5074B14781C7054785C70054B19609D
:1023B000054B186003461833044C236010BD000021
:1023C000EC060020F0060020F4060020F8060020AD
:1023D00010B50446012C09D164220C21002000F024
:1023E000BBF80121022003F037FC08E000220C2199
:1023F000104600F0B1F80021022003F02DFC10BDC2
:1024000010B50024042000F0BDFF002800D000E03B
:102410000124204610BD10B50446012C09D16422C8
:102420001C21002000F098F80121062003F014FC84
:1024300008E000221C21104600F08EF80021062042
:1024400003F00AFC10BD10B50024062000F09AFF2E
:10245000002801D0012400E00024204610BD10B562
:102460000446012C09D164221721002000F074F8E1
:102470000121042003F0F0FB08E0002217211046A0
:1024800000F06AF80021042003F0E6FB10BD0020F4
:1024900000BF704710B50446022C1CD100220D214C
:1024A000104600F059F8FDF7C9FD002809D0642254
:1024B0000B21002000F050F801210D2003F0CCFB8F
:1024C00038E000220B21104600F046F800210D20D4
:1024D00003F0C2FB2EE0032C1CD100220B2110467E
:1024E00000F03AF8FDF7AAFD002809D064220D217A
:1024F000002000F031F801210D2003F0ADFB19E0C0
:1025000000220D21104600F027F800210D2003F0D5
:10251000A3FB0FE0002C0DD164220D21002000F060
:102520001BF800220B21104600F016F801210D20A7
:1025300003F092FB10BD10B50024FDF745F802280A
:1025400001D1022406E0FDF73FF8012801D1032460
:1025500000E00024204610BD10B5064B1B788342D6
:1025600007DD242905D224234343034C24681B1987
:102570005A5410BD681D00206407002010B574482F
:1025800000684079030009F01FF80B0711D325D329
:102590005A6D77D38DA8D30005F06EFE6C480068A5
:1025A0004079401C6A4909684871CFE06949496926
:1025B000087805F0D9FE664800684079401C6449F7
:1025C00009684871624800684079401C60490968A0
:1025D0004871BBE000F028F9002811D17F2005F0F8
:1025E000C3FE5B4800684079401C5949096848713E
:1025F000574800684079401C5549096848711DE0FA
:10260000534800684078401C514909684870504858
:102610000068407803280BD300204D4909684870B2
:10262000AA204B4909688870032049490968C87085
:1026300005F04CFE002046490968487186E000F02C
:10264000F3F8002807D1424800684079401C40490F
:102650000968487103E000203D490968487105F0A8
:1026600035FE73E005F008FE394800684079401CEB
:1026700037490968487169E0364949690978491C50
:10268000C8B205F071FE324800684079401C3049FC
:10269000096848712E4800684079401C2C49096837
:1026A000487153E000F0C0F800280FD105F0B6FDE6
:1026B000274909688870012005F02AFE244800682F
:1026C0004079401C22490968487105E005F0FEFD8B
:1026D00000201F490968487138E01D48006880786B
:1026E00018280CD102201A490968087000201849DE
:1026F00009684870042016490968C87011E0144838
:1027000000684078401C1249096848701048006809
:102710004078032805D300F027F900200C49096808
:10272000487005F0D3FD00200949096848710DE0A3
:1027300005F0CCFD00200649096848710449096884
:102740004870AA2002490968887000BF00BF10BD08
:102750006C070020681D002010B5314800684079E2
:10276000002804D001280CD0032848D11DE005F032
:1027700083FD2B4800684079401C2949096848714D
:102780004BE028490969087805F0EEFD2448006807
:102790004079401C22490968487121480068407905
:1027A000401C1F490968487137E000F03DF80028D7
:1027B0000CD101201A4909680870002018490968DD
:1027C0004870042016490968C87011E01448006870
:1027D0004078401C124909684870114800684078E8
:1027E000032805D300F0C0F800200D49096848709F
:1027F00005F06CFD00200A49096848710DE005F0FC
:1028000065FD002006490968487105490968487056
:10281000AA2003490968887000BF00BF10BD0000EE
:102820006C070020681D002010B505F0EFFC044681
:102830001F4800680078002838D01D480068C0781C
:10284000042833D3002C09D1002119480068C07A2C
:102850008200174800681430815027E0144800684F
:10286000C07A8100124800681430405811498842EB
:1028700011D20F480068C07A81000D4800681430FA
:102880004058401C0A490968C97A8A000849096801
:10289000143188500AE000F067F80021044800680D
:1028A000C07A82000248006814308150204610BD72
:1028B0006C070020B80B000000B587B00120694606
:1028C0000871084802900848039008480490084896
:1028D00005900848069001A9074800F00FF807B0D6
:1028E00000BD0000212C0100F541010055B7010099
:1028F0006DC401006CC4010038170020F8B506460D
:102900000F46002400253946304600F0EFF900BF9D
:1029100014E000250EE00021242060430B4A1268D9
:102920008018415524206043094A12688018415597
:10293000681CC5B2242DEED3601CC4B205480078D3
:10294000A042E6DC00F010F8F8BD000064070020AB
:1029500068070020681D00200120024909680871ED
:10296000704700006C07002010B500F073F90020DC
:1029700003490968087002490968C87010BD000061
:102980006C07002007480068C078062808D1054871
:102990000068C079002803D1012002490968C87184
:1029A000704700006C07002010B555480068C078DB
:1029B000030008F009FE08671D1A1714110E0566BA
:1029C00050484068002803D04E484168002088479E
:1029D00093E000F0E5F890E000F0C6F88DE000F03C
:1029E000D1F88AE0FFF7B8FE87E0FFF7C7FD84E083
:1029F00044484068002803D0424841680120884785
:102A00003F480068407C00281AD03E48C068002833
:102A100003D03C48C168C82088470020384909686D
:102A20004862374800680078002804D00420344900
:102A30000968C87024E0022031490968C8701FE0A5
:102A40002F480068406A401C2D49096848622C489C
:102A50000068406A7D21C900884211D300202849BE
:102A600009684862264800680078002804D00420DD
:102A700023490968C87003E0022021490968C87029
:102A80003BE000BF1F484068002803D01D48416854
:102A9000002088471A480068407C002813D0194855
:102AA000C068002803D01748C168C82088470020A4
:102AB00013490968486212480068C078401C1049F0
:102AC0000968C87018E00E480068406A401C0C494C
:102AD000096848620A480068406A7D21C900884246
:102AE0000AD3002006490968486205480068C07892
:102AF000401C03490968C87000BF00BF10BD00003A
:102B00006C070020681D002010B515480068C078CB
:102B1000072824D0012012490968487408E01148A8
:102B20008068002802D00F4988688047FFF73CFF83
:102B30000B480068C0780628F1D109480068007A7F
:102B40000028ECD106480068C0790028E7D1044885
:102B50000068807A0028E2D101490968487410BDF4
:102B60006C070020681D002010B50548006800783B
:102B7000012802D1FEF706F801E0F6F7C3FC10BD0C
:102B80006C07002010B5054800680078012802D1C4
:102B9000FEF724FA01E0F7F793F810BD6C07002068
:102BA00010B51D480068807A002829D11A480068AD
:102BB000007A002803D00220174909688872164855
:102BC0000068C079002803D0012013490968887281
:102BD000114800680079012812D100200E490968C7
:102BE00008710D490968887207200B490968C87087
:102BF0000A484068002803D00848416800208847F8
:102C0000054800680078012802D1FEF7C1FA01E00A
:102C1000F7F730F910BD00006C070020681D002098
:102C200010B504462146084801F00AFA0748007822
:102C3000002805D1002C03D032210548FCF7CEFF37
:102C40000248047010BD000001030000AD00002028
:102C500050C300000020244909684870AA20224976
:102C60000968887000202049096848621E4909687F
:102C700008711D49096848711B49096888711A491A
:102C80000968C87118490968087217490968887283
:102C900015490968C8721449096808732420124943
:102CA000096848731049096888730F490968C8732F
:102CB00000200D49096808740B49096848740A49DD
:102CC0000968887408490968C8740749096848612F
:102CD000002105480068816103480068C16102481D
:102CE00000680162704700006C07002010B50A7888
:102CF0000D4B1860034628330C4C236024235343A8
:102D0000044628341B190A4C23600A4C4B68636044
:102D10008B68A360CB68E3604B6963610B692361D7
:102D20000B78237010BD00006C07002064070020A2
:102D300068070020681D002007480068C078062842
:102D400008D105480068007A002803D10120024913
:102D500009680872704700006C07002010B504462F
:102D6000012C09D1642220210020FFF7F5FB01216D
:102D7000084602F071FF08E0002220211046FFF70C
:102D8000EBFB0021012002F067FF10BD10B500240D
:102D9000032000F0F7FA002801D0012400E000240D
:102DA000204610BD10B50446032C0ED16422152117
:102DB0000020FFF7D1FB002214211046FFF7CCFBC7
:102DC00001210E2002F048FF39E0022C1CD1FDF752
:102DD00035F9002809D0642214210020FFF7BCFB3C
:102DE00001210E2002F038FF08E0002214211046D5
:102DF000FFF7B2FB00210E2002F02EFF002215216A
:102E00001046FFF7A9FB1AE0012C0ED16422142111
:102E10000020FFF7A1FB01210E2002F01DFF002280
:102E200015211046FFF798FB09E0002215211046F6
:102E3000FFF792FB002214211046FFF78DFB10BD17
:102E400010B50024F9F760FB094988420DD3FDF75E
:102E500033F9002807D1FDF76DF8012801DD0324BF
:102E600004E0022402E0022400E00124204610BD18
:102E7000B80B000010B50446012C09D164221D21B5
:102E80000020FFF769FB0121002002F0E5FE08E0C9
:102E900000221D211046FFF75FFB0021084602F0CB
:102EA000DBFE10BD10B50024022000F06BFA0028F4
:102EB00010D0012410480078052805DA0E48007863
:102EC000401C0D49087015E005200B4908700020D2
:102ED00048700FE0002408484078052805DA0648C5
:102EE0004078401C0449487004E0052002494870BD
:102EF00000200870204610BDCA00002010B504460E
:102F0000012C09D164221E210020FFF725FB01219D
:102F1000092002F0A1FE08E000221E211046FFF762
:102F20001BFB0021092002F097FE10BD70B50024A4
:102F300000250026FCF70CFF0546FCF715FF0646AA
:102F400002210848F7F7AAFF552800D108E0012E12
:102F500001D1002404E0012D01D1012400E000246E
:102F6000204670BDC407002010B50446012C09D1CD
:102F700064221F210020FFF7EFFA0121082002F050
:102F80006BFE08E000221F211046FFF7E5FA002142
:102F9000082002F061FE10BD70B500250024FCF78A
:102FA0000FFF044603210C48F7F778FF552803D19B
:102FB00001200A4908800AE0762C03DA012007493B
:102FC000088004E0782C02DB0020044908800348D4
:102FD0000588284670BD0000C4070020CC000020F2
:102FE00010B50446012C09D1642221210020FFF7ED
:102FF000B3FA0121072002F02FFE08E00022212170
:103000001046FFF7A9FA0021072002F025FE10BDA7
:1030100010B50024FCF79AFF002801D1012400E03C
:103020000024204610BD70470020704710B50446AC
:10303000012C09D1642216210020FFF78DFA01210D
:10304000032002F009FE08E0002216211046FFF7D7
:1030500083FA0021032002F0FFFD10BD10B500240B
:10306000052000F08FF9002801D0012400E00024A1
:10307000204610BD10B50446012C09D16422192147
:103080000020FFF769FA0121052002F0E5FD3CE090
:10309000022C17D1FCF7D2FF002809D06422192195
:1030A0000020FFF759FA0121052002F0D5FD2CE0A0
:1030B000002219211046FFF74FFA0021052002F0E7
:1030C000CBFD22E0032C17D1FCF7BEFF002809D06E
:1030D000642219210020FFF73FFA0121052002F0A8
:1030E000BBFD12E0002219211046FFF735FA00213E
:1030F000052002F0B1FD08E0002219211046FFF77B
:103100002BFA0021052002F0A7FD10BD10B5002408
:1031100004211B48F7F7C2FE552801D101242CE0F9
:10312000FCF748FF012827D1FCF72AFE01280BD025
:10313000FCF726FE022807D0FCF722FE032803D066
:10314000FCF71EFE052801D1012416E0FCF718FE4D
:10315000042801D1022410E0FCF712FE062801D158
:1031600003240AE0FCF70CFE002803D0FCF708FE5D
:10317000072802D1002400E00024204610BD0000F2
:10318000C407002010B50446012C0ED164221B2177
:103190000020FFF7E1F900221A211046FFF7DCF9C1
:1031A00001210A2002F058FD0DE064221A210020BE
:1031B000FFF7D2F900221B211046FFF7CDF90121BC
:1031C0000A2002F049FD10BD10B50024FCF7E0FF15
:1031D000012801D1012400E00024204610BD10B5D3
:1031E000F9F7ACF90446204610BD000010B5034BBA
:1031F00007220349034800F013F910BDDF31010035
:1032000018C401000017002070B506465C488068AD
:10321000002804D05A4988688047054600E0002508
:103220000024A6E0564841680C20604308184088F6
:10323000A84207D0524841680C20604308184088D3
:1032400002287DD14E4841680C20604308188068F0
:1032500000280CD04A494A680C21614351188868FB
:10326000804747490968E2008918487009E04448E6
:1032700041680C206043095C41480068E200801806
:1032800041703F480068E100401840783C490968B7
:10329000E200895C88420FD039480068E10040189C
:1032A000417837480068E2008154002034490968B9
:1032B000E200891848605AE031480068E10040188F
:1032C00041782F4842680C206043101840788142B2
:1032D0001FD12B480068E100401841682848426827
:1032E0000C2060431018808881420BD82448006865
:1032F000E10040184068801921490968E2008918F6
:10330000486034E001201E490968E20089184880BD
:103310002DE01B480068E1004018416818484268E9
:103320000C2060431018C08881420DD814480068F2
:10333000E10040184068811911480068E20000E08F
:1033400009E08018416012E000200D490968E200A0
:10335000891848800BE0002009490968E2008918B3
:103360004880002106480068E20080184160601C27
:1033700084B203488089A04200DD53E770BD00009D
:10338000CC1C00200146064A92898A4205DD044A87
:103390001268CB00D218508800E00020704700006F
:1033A000CC1C0020002000BF14E00D494A680C210D
:1033B00041435118498801290AD10021084A12685D
:1033C000C300D2185180064A1268C300D218516057
:1033D000411C88B2024989898142E6DC70470000BD
:1033E000CC1C0020002000BF13E00C494A680C21CF
:1033F000414351184988002909D1084A1268C3007D
:10340000D2185180054A1268C300D2185160411C7D
:1034100088B2024989898142E7DC7047CC1C0020D0
:10342000F0B504460020164DAB6069602C60AA819F
:1034300000BF1FE0124D6E680C254543755D104EB0
:103440003668C700F61975700D4D6E680C2545433A
:10345000755D0B4E3668C700F5550025084E366879
:10346000C700F6197580064E3668C700F6197560F4
:10347000451CA8B2024DAD898542DBDCF0BD0000E1
:10348000CC1C002070B505460E46002E05D03146F6
:103490002846F4F755FE044600E02C46204670BD51
:1034A00010B5FCF753FD002801D1F9F71FFD10BD41
:1034B00001200149887170479400002000200349D1
:1034C0000871487101208871704700009400002045
:1034D00070B5049C2578914216DD01280AD18D42F1
:1034E00006DAFF26F61AAE420ED3EE18F5B20BE05E
:1034F000154609E0022807D1954204DD9D4203DB11
:10350000EE1AF5B200E00D46257070BD0D4A416817
:10351000516081699161C168D160416A5162016AFB
:103520001162016811604169516181689160C169EE
:10353000D16101691161816A91620021024A1170B1
:10354000704700003C1D00206207002010B5FFF707
:1035500029FFF8F787FE10BD10B500200949087053
:10356000F8F780FEFFF73EFF06F048FD06F0E4FDA9
:10357000FBF7FAFEFAF79EFCFFF79AFFF9F75AFA03
:1035800010BD0000AC0000201CB5002032490870BE
:1035900004F022FE0020FCF763FE08F03DFBF8F784
:1035A0007BF8F9F785F8F6F7A3FFF7F721FA04F0AF
:1035B000E3FFF8F757FEFAF779FAF9F7C7FAF9F7E0
:1035C00045FAFFF713FEFEF7CFF9FFF775F9FAF7A3
:1035D00085F9FBF7F5FEFAF76DFC204AFF219131E2
:1035E000002006F071FE1D4AFF219131012006F0F6
:1035F0006BFE00221146104606F0AAFD00220121B2
:10360000104606F0A5FD00220221104606F0A0FD9E
:1036100000221146012006F09BFD06F0D5FC06F0C5
:103620008BFDFFF74BFFF9F71DFF00200C49887158
:1036300048710871012088704870142008700722B2
:103640006846F4F714FE0199009800F049FD022144
:10365000012000F025FC1CBDAC0000200090D00330
:10366000BE0000207047000010B50446552C03D161
:1036700005494869804702E00349086880470020FF
:103680000249087010BD00003C1D002062070020A8
:1036900010B546480078030007F096FF0A06111B94
:1036A00026303B465051738141484068002802D083
:1036B0003F494868804701203C49087000BF3C48AA
:1036C0008068002804D03A498868804737490870E4
:1036D00069E03748C068002802D03549C86880478B
:1036E00003203249087000BF31480069002804D027
:1036F0002F49086980472D49087054E02C484069DB
:10370000002802D02A4948698047002027490870CC
:1037100049E027488069002802D025498869804708
:1037200006202249087000BF2148C069002804D043
:103730001F49C86980471D49087034E000BF1B4815
:10374000007807280AD11A48006A002802D01849D0
:10375000086A804709201549087011E0134800786D
:1037600008280AD11248406A002802D01049486A45
:10377000804709200D49087002E000200B490870BD
:1037800000BF0A480078002808D00948806A00284D
:1037900004D00749886A80470449087003E0002084
:1037A0000249087000BF00BF10BD00006207002082
:1037B0003C1D00207047000010B50022FF21913110
:1037C000104606F081FD0022FF219131012006F014
:1037D0007BFD002008F0BAFA05F01CFD05F070FD35
:1037E00005F086FD00F056FAF7F792F90220FCF793
:1037F00037FD002006490870FFF786F9FFF7ACF89F
:10380000FFF7D2F8F6F7E4FF00F03EFB10BD000032
:103810000401002010B5012405F04CF9012801D164
:10382000052407E0F8F76AFE0349884201D2012423
:1038300000E00224204610BD204E000010B50624F2
:1038400005F038F9002800D1002405F039F90128E5
:1038500003D005F035F9072800D90924204610BD0A
:1038600010B5F7F755F900221146012006F0A2FD28
:1038700000213A48F7F712FC002400BF00F0BAFC20
:1038800032217D200001FCF7A9F90020344908709D
:103890000AE00022324801781046FEF75DFE30480B
:1038A0000078401C2E4908702D4800782428F0DB51
:1038B00000202C49087009E000212A48007806F011
:1038C0008BF928480078401C264908702548007864
:1038D0000E28F1DBFFF768F8F6F750FE05F03CF82C
:1038E00021480078401C20490870084600780528C7
:1038F00012D300200870FFF745F81C4800780A280A
:1039000005D3002019490870FFF716FA04E017489C
:103910000078401C1549087005F0D2F80128ADD98F
:1039200005F0CEF80728A9D200200E49087008E05B
:103930000C48007806F06AF90A480078401C0949EA
:103940000870084800780E28F2DBF7F751F8552187
:103950000248F7F7A3FB204610BD0000D007002067
:10396000C7000020C5000020C6000020C8000020BD
:1039700010B5032408E000F03DFC012000F044FBFA
:10398000002801D0042400E0F5E700BF204610BD68
:1039900010B500202749086004F01EFC0120FCF748
:1039A0005FFCF7F779FE08F037F9F6F7A1FDFAF7B3
:1039B00045F8F7F71DF804F0DFFFFAF777F8FAF7A4
:1039C00061FAF9F7C3F8FFF711FCFDF7CDFFFFF738
:1039D00009FDFFF76DFDFEF76FFFFBF7F1FCFAF74E
:1039E00069FA154AFF219131002006F06DFC124A58
:1039F000FF219131012006F067FC0022114610469C
:103A000006F0A6FB00220121104606F0A1FB0022D1
:103A10000221104606F09CFB00221146012006F010
:103A200097FB06F0D1FA06F087FB0221012000F097
:103A300037FA10BD440000200090D00310B50248B2
:103A4000FFF764FD10BD0000F4C401000021014A2D
:103A50001175704740600040014600BFF0200840EB
:103A600000110A23584302460807000F8018C0B20D
:103A700070470146002204E0501CC2B208460A38D2
:103A8000C1B20A29F8DA1007000E08437047000097
:103A900010B5044601218020F7F78AFB607A0128DF
:103AA00005D14248C078102108434049C870607A67
:103AB000A22805D13E48007F802108433C49087771
:103AC000607A3B49087700203A4948770846407FAA
:103AD0002178084337494877E07B002805D008461D
:103AE000407F20210843334948773248407FC0084F
:103AF000C000A17A08432F4948770846807FF72104
:103B000008402C498877E078FFF7B3FF294988748B
:103B1000A078FFF7AEFF2749C8746078FFF7A9FFC8
:103B2000244908752078002805D10846007D2179B0
:103B3000084320490875E079FFF79BFF1D49887508
:103B40006079FFF796FF1B494875A079FFF791FF51
:103B50001849C875207AFFF78CFF16490876084681
:103B6000807F4006400E8877E07A002806D008461D
:103B7000807F402108430F49887703E00D48807F0C
:103B80000C498877A07BFFF774FF0A498876607B31
:103B9000FFF76FFF0749C876207B08770846807FCC
:103BA000102188430349887710BD0000200402409B
:103BB00060040440404F044010B504461B48807F19
:103BC00001210843194988772078FFF752FF1749E8
:103BD00008756078FFF74DFF1449C874A078FFF7A7
:103BE00048FF1249887420780C2806DD0846407F7B
:103BF000082108430D49487709E00C48407F0B49EC
:103C000048770846007DE178084308490875074869
:103C1000807F400840000549887700BF0348807FC7
:103C2000022108400028F9D110BD0000404F044097
:103C300010B5002014490876162007F0EBFC00218F
:103C4000124801761248407F802108431049487786
:103C50000846807F012108430D49887700BF0C4842
:103C6000807F022108400028F9D00948807F400861
:103C700040000749887700BF0548807F022108403F
:103C80000028F9D110BD00004060004040610040B4
:103C9000404F044010B50020074908700021202043
:103CA000F7F786FA012105480175002004490875D7
:103CB000152007F097FC10BD005004404061004003
:103CC0004060004070B504460D46002C14D0002D15
:103CD00012D0042D10D800F013F800280CD10026C3
:103CE00008E00649885D22460121F5F749FAA41C3F
:103CF000701CC6B2AE42F4DB70BD0000EC000020C8
:103D000000200549897DC907C90F002901D001207C
:103D100000E00020704700000050044030B585B03E
:103D200005460C46002003900490009001900290FC
:103D3000072C0BDC0120A04081B268468181012163
:103D4000C17303A90220FBF751FC3EE0082C01D00F
:103D5000092C0BD10120A04081B26846818101214C
:103D6000C17303A90120FBF741FC2EE00A2C03D00C
:103D70000B2C01D00D2C0BD10120A04081B2684644
:103D800081810121C17303A90020FBF72FFC1CE0F6
:103D90000C2C01D00F2C0BD10120A04081B2684621
:103DA00081810121C17303A90E20FBF71FFC0CE0E8
:103DB0000E2C0AD10120A04081B2684681810121E8
:103DC000C17303A90C20FBF711FC002168460170A8
:103DD000C17041700121817000210171C1720D21FA
:103DE0008172FF21017200214172F5F729FA03491E
:103DF0001520FDF79BFC05B030BD00004D3A0100D9
:103E000010B5002010490875152007F0EBFB0021C4
:103E10000E4801751520002809DB00BF00BFC2064F
:103E2000D20E012191400A4A116000BF00BF00BFBD
:103E3000084880798011032805D006480078802141
:103E400008430449087010BD4060004040610040D4
:103E500000E100E00050044010B5F5F7EBFA10BDAA
:103E600010B501231A4600211846F7F75DF9012223
:103E700011461046F7F7CEF9F7F7BAF9014807F0FF
:103E8000BDFE10BD0090D00300BF044800690421AE
:103E900008430249086130BF00BF704700ED00E0F1
:103EA000F3B585B00546002003900490EEB22804D7
:103EB000070E0F2F54DA082E52DA002009E00C21E9
:103EC0004143284A515AA94201D1044603E0411C0A
:103ED000C8B21728F3D300BF0120B04086B20C202F
:103EE000604320494018C3780C2060434018827812
:103EF000F8B231460190FBF71DFC6846868101212E
:103F000081730021C17302214174F8B203A9FBF748
:103F10006DFB0C216143134A8918C888FCF7C6FA67
:103F20000C2060430F494018C188684601816946EA
:103F30000698887202A8FCF7D3F90C226243094B59
:103F4000D21891680C226243D21804201056FDF753
:103F5000EDFB0C216143034A8918C888FCF72AFA53
:103F600007B0F0BDA0C60100FEB505460C46002016
:103F7000C0430290EFB22804060E0F2E42DA082F3B
:103F800040DA0120B840694608808020204000289F
:103F900016D101208870A007800F022801D1487136
:103FA00009E0A007800F012802D16946487102E0AC
:103FB000002069464871F0B26946FBF717FB1FE025
:103FC0000020694688700E202040002800D000BFE5
:103FD00010202040002802D16946087102E001202B
:103FE00069460871E007C00F002802D16946887150
:103FF00002E0012069468871F0B26946FBF7F6FAE3
:10400000002002900298FEBD30B50146CAB20C04F1
:10401000230E00200F2B0FDA082A0DDA012494401A
:10402000A2B2064C03252D026419E45C1440002C56
:1040300001D0012000E0002030BD0000000004405D
:10404000F8B504460F460020C0430090E6B22004B5
:10405000050E0F2D11DA082E0FDA0120B04086B2BE
:10406000002F04D1E8B23146FBF7BCFB03E0E8B215
:104070003146FBF7C7FB002000900098F8BD000018
:104080001649897F01221143144A917700BF1349D1
:10409000897F022211400029F9D01049897C817062
:1040A0000E49C97C41700D49097D01700B498A7D1B
:1040B0008271497D01710949CA7D42710A7EC271CE
:1040C000897F49084900054A917700BF0349897FE4
:1040D000022211400029F9D170470000404F0440EE
:1040E00003B585B000200190029003900490002158
:1040F00068464173817E01A8C1706846417E01A86F
:1041000081706846017E4171002101A8017108217A
:1041100068460171817D01A8C1716846C17D417207
:10412000417D01A881716846017D01A801720021CD
:1041300068468173C17301A881730C2141734121C9
:10414000684601740021C17401A8FFF7A1FC1A2080
:104150000449888204491620FDF7E8FA00F006F8C1
:1041600007B000BD204F044005BD010010B5FFF7AA
:104170005FFD10BD70B504460D46601E0D498842B6
:1041800000D90124002C00D1012440200A490870E4
:10419000084600786043094948610321081F07F079
:1041A00051FA00200549886107200861044805602C
:1041B00070BD0000FFFFFF00DC00002000E000E019
:1041C000D80000200020C043002809DBC206D20E20
:1041D00001219140054A1160BFF34F8FBFF36F8FEC
:1041E00000BF0020024908618861704780E100E05B
:1041F00000E000E010B507F0CBF910BD1A20084927
:1042000008722B2048723C2088724D20C8727F2093
:10421000044909680860AC200349487070470000F1
:1042200000040240E00000200010024000B51848E1
:104230000078012812D117480078642809DB022091
:10424000154948710871002012490870104908701A
:1042500004E010480078401C0E4908700F480078B0
:10426000012814D10E480078012804D100200C49FF
:1042700008700C4908700B480078322802DBF8F708
:104280005FFA04E007480078401C0649087000BD4A
:104290008106002080060020700600207A0600209B
:1042A0007C0600207B060020FFB581B00E46174635
:1042B000012F07D1F748407D00090001C01DF549D5
:1042C000487505E0F348407D00090001F149487553
:1042D000049801287ED10A210198F3F731FF0546A1
:1042E000ED48445DE007C00F002807D0E948007C96
:1042F00000090001C01DE749087405E0E548007C9D
:1043000000090001E349087402202040002807D07A
:10431000E048C07BF02188437030DE49C87305E077
:10432000DC48C07BF0218843DA49C8730420204070
:10433000002807D0D748807C00090001C01DD5495E
:10434000887405E0D348807C00090001D149887455
:1043500008202040002807D0CE48407CF021884328
:104360007030CC49487405E0CA48407CF02188434D
:10437000C849487410202040002807D0C548407C18
:1043800000090001C01DC349487405E0C148407CD4
:1043900000090001BF49487420202040002807D0B0
:1043A000BC48007CF02188437030BA49087405E0AD
:1043B000B848007CF0218843B6490874402020406A
:1043C000002808D0B348807CF02188437030B14980
:1043D000887406E08BE0AF48807CF0218843AD49CB
:1043E00088740A210198F3F7ABFE0D46AA48445D94
:1043F000E007C00F002807D0A648807BF021884343
:104400007030A449887305E0A248807BF02188437E
:10441000A049887302202040002807D09D48807B57
:1044200000090001C01D9B49887305E09948807B05
:10443000000900019749887304202040002807D014
:104440009448007DF021884370309249087505E05A
:104450009048007DF02188438E490875082020404F
:10446000002807D08B48007D00090001C01D894944
:10447000087505E08748007D000900018549087539
:1044800010202040002807D08248C07CF0218843BB
:1044900070308049C87405E07E48C07CF0218843B4
:1044A0007C49C87420202040002807D07948C07B70
:1044B00000090001C01D7749C87305E07548C07B3D
:1044C000000900017349C87340202040002807D02C
:1044D0007048C07C00090001C01D6E49C87454E0DA
:1044E0006C48C07C000900016A49C8744DE0694805
:1044F000007C00090001674908740846C07BF02170
:1045000088436449C8730846807C000900018874A8
:104510000846407CF02188435E4948740846407C48
:104520000009000148740846007CF021884359497D
:1045300008740846807CF0218843564988740846F0
:10454000807BF0218843534988730846807B0009AB
:10455000000188730846007DF02188434D490875A5
:104560000846007D0009000108750846C07CF0215E
:1045700088434849C8740846C07B00090001C873D5
:104580000846C07C00090001C8740A9801287DD142
:104590000A213046F3F7D4FD05463F48445DE00765
:1045A000C00F002807D03B48407B00090001C01D18
:1045B0003849487305E03748407B00090001354918
:1045C000487302202040002807D03248007BF021A9
:1045D000884370302F49087305E02E48007BF02196
:1045E00088432C49087304202040002807D029481C
:1045F000807DF021884370302649887505E0254884
:10460000807DF021884323498875082020400028B8
:1046100007D02048807D00090001C01D1D49887514
:1046200005E01C48807D000900011A4988751020AA
:104630002040002807D01748407DF0218843703083
:104640001449487505E01348407DF021884311491D
:10465000487520202040002807D00E48407BF021DC
:10466000884370300B49487305E00A48407BF021CD
:104670008843084948734020204000280ED0054850
:10468000C07D00090001C01D024900E092E0C8752C
:104690000AE00000E8140020ECC301006D48C07D72
:1046A000000900016B49C8750A213046F3F748FD3F
:1046B0000D466948445DE007C00F002807D06548F3
:1046C000C07AF021884370306249C87205E06148C1
:1046D000C07AF02188435F49C87202202040002838
:1046E00007D05C48C07A00090001C01D5949C87252
:1046F00005E05848C07A000900015649C8720420F4
:104700002040002807D05348407E00090001C01D0A
:104710005049487605E04F48407E000900014D4968
:10472000487608202040002807D04A48007EF02123
:10473000884370304749087605E04648007EF021FE
:1047400088434449087610202040002807D041487B
:10475000007E00090001C01D3E49087605E03D4885
:10476000007E000900013B490876202020400028F7
:1047700007D03848007B00090001C01D3549087387
:1047800005E03448007B00090001324908734020ED
:104790002040002807D02F48C07DF021884370308A
:1047A0002C49C87554E02B48C07DF0218843294925
:1047B000C8754DE02748407B000900012549487332
:1047C0000846007BF0218843224908730846807D13
:1047D000F02188431F4988750846807D0009000143
:1047E00088750846407DF02188431A494875084677
:1047F000407BF0218843174948730846C07D000973
:104800000001C8750846C07AF02188431149C87272
:104810000846C07A00090001C8720846407E0009B7
:10482000000148760846007EF02188430949087651
:104830000846007E0009000108760846007B000952
:10484000000108730846C07DF02188430149C875FE
:1048500005B0F0BDE8140020ECC30100FFB581B045
:104860000E461746019801287ED10498002828D1C9
:10487000FB480078012824D0F7F746FEF949884222
:104880001FD3FBF7DBFB00280DD0F748807DF0211C
:1048900088437030F44988750846C07C00090001DF
:1048A000C01DC8741AE0F048807DF02188431030A4
:1048B000ED4988750846C07C00090001401CC87499
:1048C0000CE0E948807DF02188437030E649887526
:1048D0000846C07C00090001C01DC874E248C07CC5
:1048E000F02188437030E049C8740846007EF0210A
:1048F00088437030DC4908760846807D0009000155
:10490000401C88750846407DF02188431030D64908
:1049100048750846407D00090001401C487508465E
:10492000007DF02188431030CF4908750846007D8E
:1049300000090001401C0875330006F045FE062EF4
:10494000261E140C042FC848007D00090001C01D5C
:10495000C549087500BFC448007DF0218843703008
:10496000C149087500BF00E0AFE1BF48407D0009C4
:104970000001C01DBC49487500BFBB48407DF02107
:1049800088437030B849487500BFB748807D00093A
:104990000001C01DB449887500BF00E000BF00BF22
:1049A000049800285ED1AE48007801285AD0F7F765
:1049B000ABFDAC49884255D3AB48C07FF02188435A
:1049C000A949C8770846807F000900018877084612
:1049D000407FF0218843A44948770846007FF021B2
:1049E0008843A14908770846C07DF02188439E4945
:1049F000C8750846C07F00090001C8770846807F57
:104A0000F0218843984988770846407F00090001D3
:104A1000C01D48770846807EF021884392498876F9
:104A20000846807E0009000188760846407E00091D
:104A3000000148760846007E000900010876084615
:104A4000007F0009000108770846C07EF0218843F6
:104A50008549C8760846407EF021884370308249F7
:104A60004876B8E164213846F3F76AFB0546012D24
:104A700007D17D48C07FF021884370307A49C877DC
:104A800005E07948C07FF02188437749C8770A213B
:104A90003846F3F755FB0A210090F3F751FB0D461A
:104AA000642F02D37148445D01E07148445DE00722
:104AB000C00F002807D06C48807F00090001C01D8E
:104AC0006949887705E06848807F000900016649E8
:104AD000887702202040002807D06348407FF021DB
:104AE000884370306049487705E05F48407FF02197
:104AF00088435D49487704202040002807D05A4861
:104B0000007FF021884370305749087705E0564808
:104B1000007FF0218843544908770820204000286E
:104B200007D05148C07DF021884370304E49C87588
:104B300005E04D48C07DF02188434B49C8751020E1
:104B40002040002807D04848C07F00090001C01D50
:104B50004549C87705E04448C07F00090001424943
:104B6000C87720202040002807D03F48807FF021D0
:104B7000884370303C49887705E03B48807FF021CE
:104B800088433949887740202040002807D036489C
:104B9000407F00090001C01D3349487705E03248D5
:104BA000407F00090001304948770A213846F3F771
:104BB000C7FA0D462D48445DE007C00F002807D016
:104BC0002948807EF021884370302749887605E0A7
:104BD0002548807EF02188432349887602202040A2
:104BE000002807D02048807E00090001C01D1E4912
:104BF000887605E01C48807E000900011A49887605
:104C000004202040002807D01748407E00090001FA
:104C1000C01D1549487605E01348407E0009000193
:104C20001149487608202040002807D00E48007E11
:104C300000090001C01D0C49087605E00A48007E05
:104C4000000900010849087610202040002811D0F2
:104C50000548007F00090001C01D034908770FE0E7
:104C6000AC000020B80B0000BC150020ECC3010014
:104C7000FFC301005948007F000900015749087728
:104C800020202040002807D05448C07EF0218843CF
:104C900070305249C87605E05048C07EF021884304
:104CA0004E49C87640202040002807D04B48407E1F
:104CB000F02188437030494948768CE04748407E6F
:104CC000F02188434549487685E04448807D0009C5
:104CD0000001424988750846407DF02188433F49DC
:104CE00048750846407D0009000148750846007D6A
:104CF000F0218843394908750846007D0009000104
:104D000008750846C07C00090001C8740846807D0B
:104D1000F0218843314988750846C07CF0218843DA
:104D20002E49C8740846007EF02188432B49087636
:104D30000846C07FF02188432849C8770846807F0D
:104D40000009000188770846407FF0218843234905
:104D500048770846007FF0218843204908770846B5
:104D6000C07DF02188431D49C8750846C07F0009F1
:104D70000001C8770846807FF0218843174988776B
:104D80000846407F0009000148770846807EF021F0
:104D90008843124988760846807E0009000188769B
:104DA0000846407E0009000148760846007E00095A
:104DB000000108760846007F0009000108770846D0
:104DC000C07EF02188430549C8760846407EF02120
:104DD00088430249487605B0F0BD0000BC150020AC
:104DE00010B50146002200200A0EFE4B985CC30756
:104DF000DB0F002B07D0FC4BDB7FF024A343703389
:104E0000F94CE37705E0F84BDB7FF024A343F64C45
:104E1000E37702230340002B07D0F34BDB7F1B0912
:104E20001B01DB1DF04CE37705E0EF4BDB7F1B093B
:104E30001B01ED4CE37704230340002B07D0EA4B22
:104E40009B7F1B091B01DB1DE74CA37705E0E64BAD
:104E50009B7F1B091B01E44CA37708230340002B15
:104E600009D0E14B20335B781B091B01DB1DDE4CB5
:104E70002034637007E0DC4B20335B781B091B0197
:104E8000D94C2034637010230340002B09D0D64B3B
:104E900020331B78F024A3437033D34C2034237089
:104EA00007E0D14B20331B78F024A343CE4C2034B1
:104EB000237020230340002B09D0CB4B20331B78D9
:104EC0001B091B01DB1DC84C2034237007E0C64BB7
:104ED00020331B781B091B01C34C20342370402353
:104EE0000340002B07D0C04B9B7FF024A3437033BB
:104EF000BD4CA37705E0BC4B9B7FF024A343BA4C89
:104F0000A377FF231B040B401A0CB64B985CC30716
:104F1000DB0F002B07D0B44B1B7F1B091B01DB1DD4
:104F2000B14C237705E0B04B1B7F1B091B01AE4C36
:104F3000237702230340002B07D0AB4BDB7EF0240A
:104F4000A3437033A84CE37605E0A74BDB7EF02447
:104F5000A343A54CE37604230340002B07D0A24BC8
:104F60009B7EF024A34370339F4CA37605E09E4BB9
:104F70009B7EF024A3439C4CA37608230340002B84
:104F800007D0994B5B7FF024A3437033964C637733
:104F900005E0954B5B7FF024A343934C637710238C
:104FA0000340002B07D0904B5B7F1B091B01DB1DCF
:104FB0008D4C637705E08C4B5B7F1B091B018A4C92
:104FC000637720230340002B07D0874B1B7FF024FF
:104FD000A3437033844C237705E0834B1B7FF0247D
:104FE000A343814C237740230340002B07D07E4B03
:104FF000DB7E1B091B01DB1D7B4CE37605E07A4B56
:10500000DB7E1B091B01784CE376FF231B020B4060
:105010001A0A744B985CC307DB0F002B07D0724B46
:105020001B7EF024A34370336F4C237605E06E4B58
:105030001B7EF024A3436C4C237602230340002BF9
:1050400007D0694B1B7E1B091B01DB1D664C2376B9
:1050500005E0654B1B7E1B091B01634C2376042373
:105060000340002B07D0604BDB7D1B091B01DB1DC0
:105070005D4CE37505E05C4BDB7D1B091B015A4C65
:10508000E37508230340002B07D0574B9B7E1B0979
:105090001B01DB1D544CA37605E0534B9B7E1B0983
:1050A0001B01514CA37610230340002B07D04E4B1D
:1050B0005B7EF024A34370334B4C637605E04A4B90
:1050C0005B7EF024A343484C637620230340002BEF
:1050D00007D0454B5B7E1B091B01DB1D424C6376F1
:1050E00005E0414B5B7E1B091B013F4C637640236F
:1050F0000340002B07D03C4BDB7DF024A3437033EF
:10510000394CE37505E0384BDB7DF024A343364C86
:10511000E375CAB2334B985CC307DB0F002B07D093
:10512000314B1B7DF024A34370332F4C237505E0D6
:105130002D4B1B7DF024A3432B4C237502230340EE
:10514000002B07D0284B1B7D1B091B01DB1D264CA8
:10515000237505E0244B1B7D1B091B01224C237585
:1051600004230340002B07D01F4BDB7C1B091B01D2
:10517000DB1D1D4CE37405E01B4BDB7C1B091B0195
:10518000194CE37408230340002B07D0164B9B7C7B
:10519000F024A3437033144CA37405E0124B9B7CA2
:1051A000F024A343104CA37410230340002B07D01A
:1051B0000D4B5B7DF024A34370330B4C637505E00E
:1051C000094B5B7DF024A343074C63752023034008
:1051D000002B0BD0044B5B7D1B091B01DB1D024C1C
:1051E000637509E0ECC301009C1500200C4B5B7D4E
:1051F0001B091B010A4C637540230340002B07D099
:10520000074BDB7CF024A3437033054CE37405E0CB
:10521000034BDB7CF024A343014CE37410BD00007E
:105220009C15002000B501287ED1FE4AD278F023DB
:105230009A437032FB4BDA701A4612791209120146
:10524000D21D1A711A461279F0239A437032F54B27
:105250001A711A46527912091201D21D5A711A4650
:105260005279F0239A437032EE4B5A711A46D27932
:1052700012091201D21DDA711A46D279F0239A432B
:105280007032E84BDA711A46527A12091201D21DB5
:105290005A721A46527AF0239A437032E14B5A728C
:1052A0001A46927AF0239A437032DE4B9A721A466B
:1052B0009278F0239A437032DA4B9A701A46D27A77
:1052C00012091201D21DDA721A465278120912011D
:1052D000D21D5A701A46D27AF0239A437032D14BBB
:1052E000DA721A46203AD27FF0239A437032CD4BBD
:1052F000203BDA77CB4A127B12091201D21D2033F0
:105300001A731A46203A927F12091201D21D203BCD
:105310009A77C44A127BF0239A437032C14B1A73B6
:105320001A46203A127F00E0F2E1F0239A437032ED
:10533000BC4B203B1A77BB4A527B12091201D21D8B
:1053400020335A731A46203AD27E12091201D21D16
:10535000203BDA76B44AD278F0239A437032B24BCB
:10536000DA701A46127B12091201D21D1A731A46FC
:10537000127912091201D21D1A711A46927AF0237B
:105380009A437032A84B9A721A461279F0239A43C4
:105390007032A54B1A711A46527912091201D21DA8
:1053A0005A711A46927912091201D21D9A711A463F
:1053B000127A12091201D21D1A721A46127AF023B9
:1053C0009A437032984B1A721A46527A1209120195
:1053D000D21D5A72934A927912091201521C914BB2
:1053E0009A711A469279F0239A4310328D4B9A7132
:1053F0001A46127A12091201521C1A721A46127AAD
:10540000F0239A431032874B1A721A46927A120985
:105410001201521C9A721A46D27812091201521CB9
:10542000DA701A46927812091201521C9A701A46C2
:105430005278F0239A4310327A4B5A701A461278F7
:10544000F0239A431032774B1A701A4612781209D9
:105450001201521C1A701A46203AD27F1209120108
:10546000521C203BDA771A46927FF0239A4310327F
:105470006C4B203B9A771A46527FF0239A431032A6
:10548000684B203B5A771A46527F12091201521C70
:105490005A771A46127F12091201521C1A771A46BD
:1054A000D27EF0239A4310325E4B203BDA761A46C6
:1054B000927EF0239A4310325A4B203B9A765A4AF6
:1054C000127BF0239A431032574B1A731A46D27A42
:1054D000F0239A431032544BDA721A46D27A1209E8
:1054E0001201521CDA721A46927A12091201521CE7
:1054F0009A721A46527AF0239A4310324A4B5A72E1
:105500001A465279F0239A431032474B5A711A4681
:10551000D279F0239A431032434BDA710B0006F034
:1055200053F819F3E9DFD5CBC1B7ADA3998F8778CD
:105530006E645A50463E362E261E160EF5003A4A26
:10554000D279F0239A437032374BDA7100BF364A72
:105550005279F0239A437032334B5A7100BF324A6A
:10556000527AF0239A4370322F4B5A7200BF2E4A60
:10557000927A12091201D21D2B4B9A7200BF2A4A4D
:10558000D27A12091201D21D274BDA7200BF264AC5
:10559000D27AF0239A437032234BDA7200BF224A48
:1055A000127BF0239A4370321F4B1A7300BF1D4ABF
:1055B000203A927EF0239A4370321A4B203B9A761F
:1055C00000BF184A203AD27EF0239A437032154B1E
:1055D000203BDA7600BF134A203A127F12091201EB
:1055E000D21D104B203B1A7700BF0E4A203A527F43
:1055F00012091201D21D0B4B203B5A7700BF094AFA
:10560000203A527FF0239A437032064B203B5A7760
:1056100000BF044A203A927FF0239A437032014B34
:10562000203B03E008150020DC1500209A7700BF1E
:10563000DC4AD27F12091201D21DDA4BDA7700BFA1
:10564000D84A2032127812091201D21DD54B2033CC
:105650001A7000BFD34A20321278F0239A43703276
:10566000D04B20331A7000BFCE4A20325278F0233C
:105670009A437032CB4B20335A7000BFC94A203254
:10568000927812091201D21DC64B20339A7000BFC6
:10569000C44A2032D27812091201D21DC14B2033E4
:1056A000DA7000BFBF4A2032927A12091201D21D6D
:1056B000BC4B20339A7200BFBA4A2032127AF023D0
:1056C0009A437032B74B20331A7200BFB54A20326A
:1056D000127A12091201D21DB24B20331A7200BF86
:1056E000B04A20329279F0239A437032AD4B203386
:1056F0009A7100BFAB4A2032927912091201D21D71
:10570000A84B20339A7100BF01E0FFE700BF47E1DB
:10571000A44A2032D278F0239A43A24B2033DA7085
:105720001A461279120912011A711A461279F023D7
:105730009A439C4B20331A711A465279120912016E
:105740005A711A465279F0239A43964B20335A7174
:105750001A46D27912091201DA711A46D279F02367
:105760009A43904B2033DA711A46527A1209120189
:105770005A721A46527AF0239A438A4B20335A724D
:105780001A46927AF0239A43864B20339A721A462D
:105790009278F0239A43834B20339A701A46D27A38
:1057A00012091201DA721A465278120912015A705D
:1057B0001A46D27AF0239A437A4B2033DA72794A26
:1057C000D27FF0239A43774BDA771A462032127B46
:1057D0001209120120331A73724A927F12091201C0
:1057E000203B9A771A462032127BF0239A436D4B66
:1057F00020331A736B4A127FF0239A43694B1A774E
:105800001A462032527B1209120120335A73654A1C
:10581000D27E12091201203BDA76634AD278F02355
:105820009A43614BDA701A46127B120912011A73FD
:105830001A461279120912011A711A46927AF02345
:105840009A43594B9A721A461279F0239A43564B4F
:105850001A711A465279120912015A711A4692792E
:10586000120912019A711A46127A120912011A7259
:105870001A46127AF0239A434B4B1A721A46527AFE
:10588000120912015A72474A203292791209120102
:10589000444B20339A711A469279F0239A43414B34
:1058A00020339A711A46127A120912011A721A4694
:1058B000127AF0239A433B4B20331A721A46927A9B
:1058C000120912019A721A46D27812091201DA707C
:1058D0001A469278120912019A701A465278F023E9
:1058E0009A43304B20335A701A461278F0239A4369
:1058F0002C4B20331A701A461278120912011A70B2
:10590000284AD27F12091201203BDA771A46927F89
:10591000F0239A43234B9A771A46527FF0239A43F7
:10592000204B5A771A46527F120912015A771A46AB
:10593000127F120912011A771A46D27EF0239A4377
:10594000184BDA761A46927EF0239A43154B9A76D4
:10595000154A127BF0239A43134B1A731A46D27AD4
:10596000F0239A43104BDA721A46D27A12091201C6
:10597000DA721A46927A120912019A721A46527A09
:10598000F0239A43084B5A721A465279F0239A43ED
:10599000054B5A711A46D279F0239A43024BDA71B9
:1059A00000BD0000E8140020DC15002070B505469D
:1059B0000C46012D7ED1A548407D00090001C01D87
:1059C000A24948750846007DF021884310309F4960
:1059D00008750846007D00090001401C087508464E
:1059E000C07CF021884310309849C8740846807CF8
:1059F000F02188431030954988740846807C00095E
:105A00000001401C8874FAF757FB022869D19048BE
:105A10000078012865D0FAF711FB00282FD08B48B9
:105A2000007DF02188437030884908750846007D64
:105A300000090001C01D08750846C07CF02188439C
:105A400070308249C8740846807CF02188437030E9
:105A50007E4988740846807C00090001C01D887456
:105A60000846407DF02188437030784948750846E3
:105A7000407CF0218843703074494874E4E07348F6
:105A8000007DF02188431030704908750846007D7C
:105A900000090001401C08750846C07CF0218843BD
:105AA00010306A49C8740846807CF0218843103061
:105AB000664900E09BE088740846807C000900018C
:105AC000401C88740846407DF021884310305F49AF
:105AD00048750846407CF021884310305B49487483
:105AE000B2E0FAF727FA002820D1FAF7A7FA00283F
:105AF0000ED05648407DF021884370305349487598
:105B00000846407CF02188437030504948740DE0CD
:105B10004E48407DF021884310304C494875084676
:105B2000407CF0218843103048494874FAF702FA63
:105B300001282AD146480078012826D0F6F7E4FC4F
:105B40004449884221D34148407DF0218843703048
:105B50003E4948750846407CF021884370303B49F7
:105B60004874FAF76BFA002807D03848007DF02116
:105B7000884370303549087566E03448007DF0216F
:105B800088431030314908755EE0230005F01CFDA4
:105B9000062C241C140C042D2C48807C00090001C8
:105BA000C01D2A49887400BF2848807CF0218843A2
:105BB00070302649887400BF2448C07CF021884397
:105BC00070302249C87400BF2048007D00090001E0
:105BD000C01D1E49087500BF1C48007DF021884388
:105BE00070301A49087500BF00E000BF2CE017486C
:105BF000407DF0218843154948750846007DF02115
:105C00008843124908750846007D0009000108759F
:105C10000846C07CF02188430C49C8740846807C43
:105C2000F0218843094988740846807C00090001F6
:105C300088740846407D0009000148750846407C8C
:105C4000F02188430149487470BD00000815002008
:105C5000AC000020B80B000030B50246002901D18D
:105C6000002000E00720130005F0AEFC0F09141F10
:105C70002B3743505D67727C88929FA9B500574BC4
:105C80005B7EF024A3430401F0252C402343534CB6
:105C90006376A1E0524B9B79F024A3430401F025E5
:105CA0002C4023434E4CA37196E04D4B2033DB79BF
:105CB0001B091B010407240F2343494C2034E371C3
:105CC0008AE0464B2033DB7C1B091B010407240FB1
:105CD0002343424C2034E3747EE0404B40331B7836
:105CE0001B091B010407240F23433C4C4034237041
:105CF00072E03A4B2033DB7FF024A3430401F0250C
:105D00002C402343354C2034E37765E0334B20337C
:105D10005B7BF024A3430401F0252C4023432F4C4C
:105D20002034637358E02E4B9B791B091B01040739
:105D3000240F23432A4CA3714EE0294B9B7CF02473
:105D4000A3430401F0252C402343254CA37443E0D6
:105D5000234BDB7E1B091B010407240F2343204C2C
:105D6000E37639E01D4B2033DB7F1B091B01040761
:105D7000240F2343194C2034E3772DE0174B9B7EEF
:105D80001B091B010407240F2343144CA37623E0B3
:105D9000134B20339B79F024A3430401F0252C40BE
:105DA00023430F4C2034A37116E00D4BDB7D1B0900
:105DB0001B010407240F2343094CE3750CE0074B38
:105DC00020335B7C1B091B010407240F2343034C76
:105DD0002034637400E000BF00BF30BDE814002031
:105DE000BC150020F7B582B00E461746F74800787C
:105DF00001286ED0F6F788FBF549884269D3FAF797
:105E00009FF803281DD1FAF719F900280DD0F148A1
:105E1000407CF02188437030EE4948740846807C0D
:105E200000090001C01D8874D1E0EA48407CF021DF
:105E30008843E84948740846807C0009000188745A
:105E4000C5E0FAF77DF8002803D0FAF779F80528BD
:105E500065D1029800280CD1DE48407CF0218843AF
:105E6000DC4948740846807C00090001C01D887424
:105E70000BE0D848407CF02188437030D549487405
:105E80000846807C000900018874FAF759F8002858
:105E900020D1D0482030C078F02188437030CD49DF
:105EA0002031C870CB48807D0009000120398875F9
:105EB0000846807DF0218843C649887564222321E5
:105EC0000020FCF749FB002222211046FCF744FB8E
:105ED0007DE04EE0FAF734F8052878D1BD4820304F
:105EE000C078F0218843BB492031C870B948807D13
:105EF00000090001C01D203988750846807DF02109
:105F000088437030B3498875002223211046FCF77E
:105F100023FB642222210020FCF71EFB57E0AD4842
:105F2000407CF0218843AB4948740846807C0009D6
:105F30000001887408462030C078F0218843A549C4
:105F40002031C870A348807D000900012039887580
:105F50000846807DF02188439E49887500222321D0
:105F60001046FCF7F9FA002222211046FCF7F4FA59
:105F70002DE09848407CF021884370309549487462
:105F80000846807C00090001C01D88740846203046
:105F9000C078F021884370308E492031C8708D4818
:105FA000807D00090001C01D203988750846807D6C
:105FB000F0218843703087498875642223210020AE
:105FC000FCF7CAFA642222210020FCF7C5FAF9F78F
:105FD000B7FF002808D07D480078012804D0F6F7E4
:105FE00093FA7B49884276D27B48864209D9794820
:105FF00020304079F0218843703076492031487153
:1060000007E0744820304079F021884371492031FD
:10601000487172493046F2F793F80A210190F2F77D
:106020008FF80D466C48401C864202D36C48445D94
:1060300001E06C48445DE007C00F002809D06548C6
:106040002030C07800090001C01D62492031C870AD
:1060500007E060482030C078000900015D49203128
:10606000C87002202040002809D05A48203080788B
:10607000F0218843703057492031887007E0554837
:1060800020308078F02188435249203188700420E4
:106090002040002809D04F4820304078F021884324
:1060A00070304C492031487007E04A482030407831
:1060B000F0218843474920314870082020400028BB
:1060C0000AD044482030407900090001C01D4149F0
:1060D0002031487108E09EE23E48203040790009B6
:1060E00000013C492031487110202040002809D08F
:1060F000384820300079F02188437030354920310C
:10610000087107E0334820300079F0218843314995
:106110002031087120202040002809D02D4820304F
:10612000007900090001C01D2A492031087107E0EB
:1061300028482030007900090001264920310871E3
:1061400040202040002809D02248203080780009D3
:106150000001C01D1F492031887007E01D48203014
:106160008078000900011B49203188707D21C90019
:106170003046F1F7E5FF0A210190F1F7E1FF0D4606
:106180001648864202D31648445D01E01548445D36
:10619000E007C00F002807D00E48C07FF0218843D9
:1061A00070300C49C87705E00A48C07FF021884369
:1061B0000849C87702202040002815D00548C07F34
:1061C00000090001C01D0349C87713E0AC0000209E
:1061D000B80B00009C1500209F86010010270000CE
:1061E000ECC30100FFC30100FB48C07F00090001B0
:1061F000F949C87704202040002807D0F648807F5E
:1062000000090001C01DF449887705E0F248807F4D
:1062100000090001F049887708202040002809D0B3
:10622000ED482030407800090001C01DEA492031C6
:10623000487007E0E8482030407800090001E6494E
:106240002031487010202040002809D0E24820303A
:106250000078F02188437030DF492031087007E072
:10626000DD4820300078F0218843DB492031087078
:1062700020202040002809D0D7482030007800098D
:106280000001C01DD4492031087007E0D2482030F9
:10629000007800090001D0492031087040202040DA
:1062A000002807D0CC48807FF02188437030CA494D
:1062B000887705E0C848807FF0218843C649887701
:1062C00064213046F1F73CFF0A210190F1F738FFD5
:1062D0000D467D20C000864202D3C048445D01E0E7
:1062E000BF48445DE007C00F002807D0BA48007FD0
:1062F00000090001C01DB849087705E0B648007FD5
:1063000000090001B449087702202040002807D086
:10631000B148C07EF02188437030AF49C87605E0AF
:10632000AD48C07EF0218843AB49C87604202040A8
:10633000002807D0A848807EF02188437030A64905
:10634000887605E0A448807EF0218843A2498876BB
:1063500008202040002807D09F48407FF021884334
:1063600070309D49487705E09B48407FF021884385
:106370009949487710202040002807D09648407F50
:1063800000090001C01D9449487705E09248407F0C
:10639000000900019049487720202040002807D0BC
:1063A0008D48007FF021884370308B49087705E0E5
:1063B0008948007FF02188438749087740202040A2
:1063C000002807D08448C07E00090001C01D824912
:1063D000C87605E08048C07E000900017E49C87685
:1063E0000A213046F1F7ACFE0A210190F1F7A8FE30
:1063F0000D46642E02D37948445D01E07848445D3F
:10640000E007C00F002807D07348007EF0218843C2
:1064100070307149087605E06F48007EF0218843AE
:106420006D49087602202040002807D06A48007E87
:1064300000090001C01D6849087605E06648007E35
:10644000000900016449087604202040002807D094
:106450006148C07D00090001C01D5F49C87505E0A5
:106460005D48C07D000900015B49C87508202040D7
:10647000002807D05848807E00090001C01D5649F9
:10648000887605E05448807E0009000152498876EC
:1064900010202040002807D04F48407EF02188433C
:1064A00070304D49487605E04B48407EF0218843E6
:1064B0004949487620202040002807D04648407EA1
:1064C00000090001C01D4449487605E04248407E6D
:1064D000000900014049487640202040002807D0AC
:1064E0003D48C07DF021884370303B49C87505E0C8
:1064F0003948C07DF02188433749C8750A213046A4
:10650000F1F71EFE0D463548445DE007C00F002838
:1065100007D03148007DF021884370302E4908753E
:1065200005E02D48007DF02188432B4908750220A5
:106530002040002807D02848007D00090001C01D28
:106540002549087505E02448007D0009000122491D
:10655000087504202040002807D01F48C07C00098F
:106560000001C01D1C49C87405E01B48C07C00091F
:1065700000011949C87408202040002807D0164897
:10658000807CF021884370301349887405E01248FC
:10659000807CF02188431049887410202040002816
:1065A00007D00D48407DF021884370300A49487576
:1065B00005E00948407DF0218843074948752020BF
:1065C000204000280ED00448407D00090001C01D75
:1065D000014948750CE000009C150020ECC3010047
:1065E000FFC30100FD48407D00090001FB494875DB
:1065F00040202040002807D0F848C07CF021884384
:106600007030F649C87473E2F448C07CF0218843C6
:10661000F249C874F7E7F9F793FC05287CD1EF48F5
:1066200020304079F0218843EC49203148710846F8
:10663000C07800090001C87008468078F0218843BE
:10664000E6492031887008464078F0218843E349C4
:106650002031487008464079000900014871084619
:106660000079F0218843DD4920310871084600791E
:10667000000900010871084680780009000188704F
:106680007D21C9003846F1F75BFD0546D448445DDD
:10669000E007C00F002807D0D048C07FF021884312
:1066A0007030CE49C87705E0CC48C07FF0218843E0
:1066B000CA49C87702202040002807D0C748C07FB9
:1066C00000090001C01DC549C87705E0C348C07F67
:1066D00000090001C149C87704202040002807D0E4
:1066E000BE48807F00090001C01DBC49887705E0D5
:1066F000BA48807F00090001B84988770820204007
:1067000000280AD0B5482030407800090001C01D9B
:10671000B2492031487008E0F2E1B04820304078BA
:1067200000090001AD4920314870102020400028A8
:1067300009D0AA4820300078F02188437030A7495A
:106740002031087007E0A54820300078F021884308
:10675000A2492031087020202040002809D09F48FD
:106760002030007800090001C01D9C4920310870CC
:1067700007E09A482030007800090001974920314D
:10678000087040202040002807D09448807FF021E6
:10679000884370309149887705E09048807FF021E8
:1067A00088438E49887764213846F1F7C9FC0A216D
:1067B0000190F1F7C5FC0D467D20C000874202D351
:1067C0008848445D01E08648445DE007C00F00282A
:1067D00007D08248007F00090001C01D7F4908776B
:1067E00005E07E48007F000900017C49087702200F
:1067F0002040002807D07948C07EF02188437030BF
:106800007649C87605E07548C07EF0218843734913
:10681000C87604202040002807D07048807EF021F0
:10682000884370306D49887605E06C48807EF021A1
:1068300088436A49887608202040002807D06748A6
:10684000407FF021884370306449487705E0634811
:10685000407FF0218843614948771020204000287C
:1068600007D05E48407F00090001C01D5B494877A2
:1068700005E05A48407F0009000158494877202028
:106880002040002807D05548007FF0218843703011
:106890005249087705E05148007FF02188434F496D
:1068A000087740202040002807D04C48C07E0009CF
:1068B0000001C01D4949C87605E04848C07E00096E
:1068C00000014649C8760A213846F1F739FC0A2109
:1068D0000190F1F735FC0D46642F01D2002F02D153
:1068E0004048445D01E03E48445DE007C00F002899
:1068F00007D03A48007EF021884370303749087647
:1069000005E03648007EF0218843344908760220AD
:106910002040002807D03148007E00090001C01D3A
:106920002E49087605E02D48007E000900012B491C
:10693000087604202040002807D02848C07D0009A0
:106940000001C01D2549C87505E02448C07D000927
:1069500000012249C87508202040002807D01F48A0
:10696000807E00090001C01D1C49887605E01B4897
:10697000807E0009000119498876102020400028F7
:1069800007D01648407EF02188437030134948767E
:1069900005E01248407EF0218843104948762020C7
:1069A0002040002807D00D48407E00090001C01D8E
:1069B0000A49487605E00948407E00090001074978
:1069C00048764020204000280ED00448C07DF021A9
:1069D000884370300149C8750CE000009C15002008
:1069E000FFC30100ECC30100FE48C07DF0218843D5
:1069F000FC49C8750A213846F1F7A2FB0D46FA4852
:106A0000445DE007C00F002807D0F648007DF02164
:106A100088437030F349087505E0F248007DF021A5
:106A20008843F049087502202040002807D0ED482F
:106A3000007D00090001C01DEA49087505E0E9482C
:106A4000007D00090001E749087504202040002866
:106A500007D0E448C07C00090001C01DE149C874AA
:106A600005E0E048C07C00090001DE49C874082048
:106A70002040002807D0DB48807CF021884370301C
:106A8000D849887405E0D748807CF0218843D549EF
:106A9000887410202040002807D0D248407DF02183
:106AA00088437030CF49487505E0CE48407DF021DD
:106AB0008843CC49487520202040002807D0C94889
:106AC000407D00090001C01DC649487505E0C54864
:106AD000407D00090001C34948754020204000283E
:106AE00007D0C048C07CF02188437030BD49C874CD
:106AF00026E2BC48C07CF0218843BA49C8741FE232
:106B0000F9F71EFA06287DD1B64820304079F021E9
:106B10008843B449203148710021B448F4F7BEF9E4
:106B2000552830D1B248FEF75BF9AE482030C07826
:106B300000090001AB492031C87008468078F02177
:106B40008843A8492031887008464078F02188435E
:106B5000A449203148700846407900090001487175
:106B600008460079F02188439E4920310871084683
:106B700000790009000108710846807800090001C9
:106B8000C01D8870DCE19B480078401C9949087062
:106B900094482030C07800090001C01D914920317F
:106BA000C87008468078F021884370308D492031C4
:106BB000887008464078F02188438A49203148701F
:106BC0000846407900090001487108460079F02123
:106BD00088437030834920310871084600790009E4
:106BE0000001C01D08710846807800090001C01D21
:106BF000887081480078002809D1FEF7F1F800205C
:106C00007C4900E04DE008707C49086098E17948D3
:106C10000078642824DA7A4800787749097888422D
:106C200004DB75480078401E754908707248027888
:106C3000744972480068F8F777F900282CD1704839
:106C4000007880006F490858002825D06C480078EB
:106C500080000858694908600020664908701BE0F8
:106C600064480078642817DB65480078401C644954
:106C700008700846007860490978884202DB0020E5
:106C80005F4908705E48007880005E4908585B499B
:106C9000086000205749087058480068FEF7A0F8BF
:106CA0004EE1F9F74DF90728B0D14E482030407930
:106CB000F02188434B49203148710846C0780009CB
:106CC0000001C01DC87008468078F02188434549FE
:106CD0002031887008464078F0218843703041495F
:106CE000203148700846407900090001C01D4871F4
:106CF00008460079F02188433A4920310871084656
:106D0000007900090001C01D08710846807800095B
:106D10000001C01D88703348C07FF021884331498D
:106D2000C8770846C07F00090001C8770846807F01
:106D300000090001887708462030407800090001EA
:106D40002031487008460078F021884325492031D9
:106D50000870084600780009000108702148807F0B
:106D6000F02188431F4988770846007F0009000109
:106D7000C01D08770846C07EF0218843703019494D
:106D8000C8760846807EF0218843703015498876A1
:106D90000846407FF0218843703012494877084602
:106DA000407F00090001C01D48770846007FF021A0
:106DB000884370300B4908770846C07E00090001FF
:106DC000C876F9F7F7F8002868D10648007EF02168
:106DD00088437030034908760846007E00090001A8
:106DE000087611E09C150020ECC30100C4070020C8
:106DF0000B0B0B0B600000207A0000205C000020D1
:106E000058000020F01000200846C07D0009000155
:106E1000C8750846807E0009000188760846407ED5
:106E2000F02188437030474948760846407E000983
:106E30000001C01D48760846C07DF02188437030AF
:106E40004049C8750846007DF021884370303D49AF
:106E500008750846007D0009000108750846C07CD9
:106E600000090001C8740846807CF0218843354938
:106E700088740846407DF021884370303149487558
:106E80000846407D00090001C01D48750846C07CC9
:106E9000F021884370302B49C87451E02948007EA6
:106EA000F02188437030274908760846007E0009A3
:106EB0000001C01D08760846C07D00090001C01D04
:106EC000C8750846807E0009000188760846407E25
:106ED000F021884370301B4948760846407E0009FF
:106EE0000001C01D48760846C07DF0218843154941
:106EF000C8750846007DF021884312490875084688
:106F0000007D0009000108750846C07C00090001E9
:106F1000C8740846807CF02188430A498874084672
:106F2000407DF0218843074948750846407D0009A7
:106F3000000148750846C07CF02188430149C874A7
:106F400005B0F0BD9C150020FFB581B005460E468A
:106F5000002000900027002D7ED0FE488079F0218F
:106F600088437030FB49887108462038007FF02143
:106F700088437030F74920390877F74800780128AE
:106F800072D0F5F7C1FAF54988426DD3F8F7D8FF0A
:106F9000042825D1F9F752F8002811D0ED482038FF
:106FA000807D00090001C01DEA4920398875084626
:106FB000807DF02188437030E6492039887573E080
:106FC000E4482038807D00090001E24920398875B5
:106FD0000846807DF0218843DE492039887563E0CA
:106FE000049800281FD1DB482038807D000900016B
:106FF000D849203988750846807DF0218843703053
:10700000D449203988750846807EF0218843703045
:10701000D04920398876CF480079F02188437030F4
:10702000CC49087140E0CB482038807D0009000140
:10703000C01DC849203988750846807DF0218843E5
:10704000C449203988750846807EF0218843C149AB
:1070500020398876BF4801E02DE305E00079F02172
:107060008843BC4908711FE0BA482038807D000978
:107070000001C01DB749203988750846807DF02180
:1070800088437030B349203988750846807EF021E6
:1070900088437030AF4920398876AE480079F021B6
:1070A00088437030AB4908710A9801287ED10A21C3
:1070B0003046F1F745F80090A94900980C5CE007CC
:1070C000C00F002807D0A348C07900090001C01DE7
:1070D000A049C87105E09F48C079000900019D4999
:1070E000C87102202040002807D09A488079000902
:1070F0000001C01D9749887105E096488079000914
:1071000000019449887104202040002807D091484C
:10711000407900090001C01D8E49487105E08D4885
:107120004079000900018B4948710820204000285F
:1071300007D08848007AF02188437030854908726A
:1071400005E08448007AF0218843824908721020C3
:107150002040002807D07F48007A00090001C01DA8
:107160007C49087205E07B48007A000900017949F2
:10717000087220202040002807D07648C079F021EE
:10718000884370307349C87105E07248C079F021B6
:1071900088437049C87140202040002809D06D48BC
:1071A0004079F021884370306A4900E08EE04871F0
:1071B00005E068484079F0218843664948710A2112
:1071C0003046F0F7BDFF0091654900980C5CE00780
:1071D000C00F002807D05F48C07800090001C01D1B
:1071E0005C49C87005E05B48C07800090001594956
:1071F000C87002202040002807D056488078F0212F
:10720000884370305349887005E052488078F021F7
:1072100088435049887004202040002807D04D48FA
:107220004078F021884370304A49487005E0494869
:107230004078F021884347494870082020400028C2
:1072400007D04448407800090001C01D41494870FA
:1072500005E040484078000900013E494870102090
:107260002040002807D03B48007900090001C01DDC
:107270003849087105E037480079000900013549AF
:10728000087120202040002807D03248C078F02123
:10729000884370302F49C87005E02E48C078F0212F
:1072A00088432C49C87040202040002807D0294836
:1072B000807800090001C01D264988705DE02548DE
:1072C0008078000900012349887056E02148407900
:1072D000F021884370301F494871084680780009C2
:1072E0000001C01D88700846C07900090001C871FE
:1072F0000846807900090001887108464079000934
:10730000000148710846007AF0218843114908724B
:107310000846007A0009000108720846C079F02189
:1073200088430C49C8710846C07800090001C8703C
:1073300008468078F02188430649887008464078DE
:10734000F02188430349487008464078000900014D
:10735000487007E028150020AC000020B80B0000A2
:10736000ECC30100084600790009000108710846D5
:10737000C078F0218843FE49C8700B9801287DD160
:107380000A210398F0F7DCFE0746FA48C45DE007DF
:10739000C00F002809D0F6482038407F00090001BE
:1073A000C01DF3492039487707E0F1482038407F75
:1073B00000090001EE4920394877022020400028CA
:1073C00009D0EB482038007F00090001C01DE849C2
:1073D0002039087707E0E6482038007F00090001DF
:1073E000E3492039087704202040002809D0E048EC
:1073F0002038C07E00090001C01DDD492039C87653
:1074000007E0DB482038C07E00090001D849203958
:10741000C87608202040002809D0D5482038807F31
:10742000F02188437030D2492039887707E0D0486E
:107430002038807FF0218843CD492039887710207B
:107440002040002809D0CA482038807F0009000168
:10745000C01DC7492039887707E0C5482038807F9C
:1074600000090001C24920398877202020400028E7
:107470000BD0BF482038407FF02100E0C5E08843B2
:107480007030BB492039487707E0B9482038407F41
:10749000F0218843B6492039487740202040002811
:1074A00009D0B3482038C07EF02188437030B049FD
:1074B0002039C87607E0AE482038C07EF0218843E6
:1074C000AB492039C8760A210398F0F739FE0F46F8
:1074D000A848C45DE007C00F002809D0A4482038A0
:1074E000407E00090001C01DA1492039487607E00F
:1074F0009F482038407E000900019D492039487688
:1075000002202040002809D099482038007EF02130
:107510008843703096492039087607E0944820382F
:10752000007EF021884392492039087604202040CB
:10753000002809D08E482038C07DF0218843703063
:107540008B492039C87507E089482038C07DF02173
:10755000884387492039C87508202040002809D071
:1075600083482038C07D00090001C01D80492039B2
:10757000C87507E07E482038C07D000900017C49BD
:107580002039C87510202040002809D078482038BC
:10759000807E00090001C01D75492039887607E00A
:1075A00073482038807E00090001714920398876AF
:1075B00020202040002809D06D482038407EF0214E
:1075C000884370306A492039487607E06848203897
:1075D000407EF0218843664920394876402020408B
:1075E000002809D062482038007E00090001C01D33
:1075F0005F49203908762AE15D482038007E00097D
:1076000000015B492039087621E159482038C07EC5
:10761000F0218843703056492039C8760846007EEC
:1076200000090001C01D08760846407F00090001DE
:1076300048770846007F0009000108770846C07EA9
:1076400000090001C8760846807FF0218843484938
:10765000203988770846807F00090001887708462E
:10766000407FF02188434249203948770846407ED0
:107670000009000148760846007EF02188433C4915
:10768000203908760846C07DF021884338492039E2
:10769000C8750846C07D00090001C8750846807E8F
:1076A0000009000188760846407EF0218843304971
:1076B00020394876CBE02E482038C07EF021884320
:1076C0002B492039C8760846007E0009000108765B
:1076D0000846407F0009000148770846007F0009FE
:1076E000000108770846C07E00090001C8760846F8
:1076F000807FF02188431E49203988770846807FA3
:107700000009000188770846407FF0218843184926
:10771000203948770846407E00090001487608462F
:10772000007EF02188431249203908760846C07D42
:10773000F02188430E492039C8750846C07D0009EC
:107740000001C8750846807E000900018876084659
:10775000407EF02188430649203948760448407924
:10776000F02188430249487108468078000903E007
:1077700028150020ECC30100000188700846C0797C
:1077800000090001C871084680790009000188716C
:10779000084640790009000148710846007AF02146
:1077A00088432C4908720846007A000900010872D3
:1077B0000846C079F02188432649C8710846C07838
:1077C00000090001C87008468078F02188432149EB
:1077D000887008464078F02188431E494870084662
:1077E000407800090001487008460079000900014E
:1077F00008710846C078F02188431649C8700846C9
:107800002038807D00090001203988750846807D78
:10781000F02188430F49203988750846807EF02181
:1078200088430C49203988760846007FF021884338
:1078300008492039087707480079F021884305492D
:10784000087108468079F02188430249887105B0A3
:10785000F0BD000028150020F7B582B007460E469F
:107860000025012F6FD1FE48007801286DD0F4F774
:107870004BFEFC49884268D3F8F762FB032831D1FC
:10788000F8F7DCFB002817D0F748407BF02188434D
:107890007030F54948730846C07B00090001C01DDF
:1078A000C873642208210020FAF756FE64220921D9
:1078B0000020FAF751FE5FE0EB48407BF02188435F
:1078C000E94948730846C07B00090001C8730022DB
:1078D00008211046FAF740FE002209211046FAF767
:1078E0003BFE49E00498002816D1DF48407BF02198
:1078F0008843DD4948730846C07B00090001C01D6C
:10790000C873642208210020FAF726FE002209210C
:107910001046FAF721FE2FE0D348407BF021884340
:107920007030D14948730846C07B00090001C87314
:10793000002208211046FAF70FFE642209210020D8
:10794000FAF70AFE18E058E1FFE7C748407BF0214C
:1079500088437030C44948730846C07B0009000161
:10796000C01DC873642208210020FAF7F5FD6422C7
:1079700009210020FAF7F0FD64213046F0F7E0FB22
:107980000546012D09D1B8482038807B0009000147
:10799000C01DB5492039887307E0B3482038807B83
:1079A00000090001B049203988730A213046F0F7F8
:1079B000C7FB0A210190F0F7C3FB0D46642E02D3EA
:1079C000AA48445D01E0AA48445DE007C00F0028D2
:1079D00007D0A548407AF02188437030A249487208
:1079E00005E0A148407AF02188439F49487202206F
:1079F0002040002807D09C48407A00090001C01DA3
:107A00009949487205E09848407A00090001964972
:107A1000487204202040002809D093482038007C78
:107A2000F0218843703090492039087407E08E486F
:107A30002038007CF02188438B49203908740820C5
:107A40002040002809D088482038007C0009000127
:107A5000C01D85492039087407E083482038007C20
:107A600000090001804920390874102020400028B6
:107A700009D07D482038C07BF021884370307A4996
:107A80002039C87307E078482038C07BF02188434C
:107A900075492039C87320202040002809D0724839
:107AA0002038807BF021884370306F4920398873FB
:107AB00007E06D482038807BF02188436A492039EF
:107AC000887340202040002809D067482038C07BB8
:107AD00000090001C01D64492039C87307E06248ED
:107AE0002038C07B000900015F492039C8730A2192
:107AF0003046F0F725FB0D465C48445DE007C00FBB
:107B0000002807D05848407B00090001C01D564995
:107B1000487305E05448407B00090001524948730E
:107B200002202040002807D04F48007BF0218843E6
:107B300070304D49087305E04B48007BF0218843C5
:107B40004949087304202040002807D04648007B9C
:107B500000090001C01D4449087305E04248007B4C
:107B6000000900014049087308202040002807D080
:107B70003D48C07AF021884370303B49C87205E027
:107B80003948C07AF02188433749C8721020204014
:107B9000002807D03448C07A00090001C01D3249CE
:107BA000C87205E03048C07A000900012E49C87249
:107BB00020202040002807D02B48807A00090001AF
:107BC000C01D2949887205E02748807A0009000114
:107BD0002549887240202040002807D02248807A1A
:107BE000F021884370302049887281E01E48807AF5
:107BF000F02188431C4988727AE00022082110464F
:107C0000FAF7AAFC002209211046FAF7A5FC16484B
:107C1000407BF0218843144948730846C07B000923
:107C20000001C87308462038807B00090001203914
:107C300088730D48407AF02188430B494872084602
:107C4000407A00090001487208462038007CF02183
:107C500088430549203908740846007C000909E07A
:107C6000AC000020B80B000028150020ECC3010078
:107C7000FFC30100000108740846C07BF02188435F
:107C80001C49C8730846807BF021884319498873D2
:107C90000846C07B00090001C87308462030407BBD
:107CA00000090001203148730846007BF021884319
:107CB0001049203108730846007B00090001087351
:107CC0000846C07AF02188430A492031C872084624
:107CD000C07A00090001C8720846807AF021884302
:107CE0000449203188720846807A000900018872B0
:107CF00005B0F0BD08150020F8B507460D46002672
:107D0000002F7AD0D448C07900090001C01DD249A3
:107D1000C8710846807AF02188437030CE49887255
:107D200064212846F0F722FA86B2CC48845DE00749
:107D3000C00F002807D0C848C07BF02188437030AE
:107D4000C549C87305E0C448C07BF0218843C249D7
:107D5000C87302202040002807D0BF48C07B00091C
:107D60000001C01DBC49C87305E0BB48C07B0009C9
:107D70000001B949C87304202040002807D0B64844
:107D8000807B00090001C01DB349887305E0B2483B
:107D9000807B00090001B04988730820204000283A
:107DA00007D0AD48407C00090001C01DAA494874B5
:107DB00005E0A948407C00090001A749487410204B
:107DC0002040002807D0A448007CF0218843703070
:107DD000A149087405E0A048007CF02188439E4931
:107DE000087420202040002808D09B48007C00090F
:107DF0000001C01D9849087406E02CE19648007CFB
:107E0000000900019449087440202040002807D050
:107E10009148807BF021884370308F49887305E05A
:107E20008D48807BF02188438B4988730A2128463E
:107E3000F0F786F90A210090F0F782F90E46642DDA
:107E400001D2002D02D18648845D01E08348845D23
:107E5000E007C00F002807D07F48007BF02188434F
:107E600070307D49087305E07B48007BF021884332
:107E70007949087302202040002807D07648007B0B
:107E800000090001C01D7449087305E07248007BB9
:107E9000000900017049087304202040002807D021
:107EA0006D48C07A00090001C01D6B49C87205E029
:107EB0006948C07A000900016749C872082020405B
:107EC000002807D06448407CF02188437030624924
:107ED000487405E06048407CF02188435E4948745E
:107EE00010202040002807D05B48407BF0218843C9
:107EF00070305949487305E05748407BF02188436A
:107F00005549487320202040002807D05248407B24
:107F100000090001C01D5049487305E04E48407BF0
:107F2000000900014C49487340202040002807D038
:107F30004948C07AF021884370304749C87205E04B
:107F40004548C07AF02188434349C8720A2128462F
:107F5000F0F7F6F80E464248845DE007C00F0028AF
:107F600007D03D48407A00090001C01D3A494872D7
:107F700005E03948407A000900013749487202207B
:107F80002040002807D03448007AF0218843703020
:107F90003149087205E03048007AF02188432E49C3
:107FA000087204202040002807D02B48C079F02117
:107FB000884370302849C87105E02748C079F0210E
:107FC00088432549C87108202040002807D022484E
:107FD000807C00090001C01D1F49887405E01E480F
:107FE000807C000900011C49887410202040002872
:107FF00007D01948807A00090001C01D164988720F
:1080000005E01548807A0009000113498872202094
:108010002040002807D01048407AF0218843703073
:108020000D49487205E00C48407AF02188430A491E
:10803000487240202040002807D00748007A0009F5
:108040000001C01D0449087205E00348007A0009D8
:10805000000101490872F8BDBC150020FFC30100F2
:10806000ECC3010070B500BF0A2108480078F0F7A2
:108070007DF8FF21F531484384B22046F0F776F8C9
:10808000C5B229460120FDF7CDF870BD6200002081
:1080900070B5044600250A210E480078F0F750F824
:1080A000054629460120FDF781FC01232246294689
:1080B0001846FCF7D3FB074800783B2805DA05484B
:1080C0000078401C0349087002E000200149087054
:1080D00070BD000061000020F0B504460D46264644
:1080E00000210020002A0CDD122007E06F5CB7425F
:1080F00002D10020197003E04F1CF9B29142F5DB68
:1081000001E000271F70F0BD30B504461320002C9D
:1081100008D1002A04D015788D420BDC002009E03C
:10812000132007E0002A04D0D55C8D4202D1002044
:1081300000E0132030BD002000BF704770B504463A
:108140000D4600200021002A0DDD312008E04E0000
:10815000AE5BA64202D10020197003E04E1CF1B2C2
:108160009142F4DB00BF70BD10B502460020535CA5
:10817000002B05D0535C034C2478A34200D033205D
:1081800010BD00008206002030B503460C460025D5
:10819000F7F750FD195D0840002800D17E252846DC
:1081A00030BD10B503460024F7F744FD1840002801
:1081B00000D17F24204610BD10B5F4F7FDFEF5F781
:1081C000B3F8F5F797FA10BD002002E000BF411C9C
:1081D000C8B22828FAD3704710B500210948FBF728
:1081E000C3FEFFF7F1FFFFF7EFFF00210548401C3A
:1081F000FBF7BAFEFFF7E8FFFFF7E6FF02200249B0
:10820000087010BD02060000AE0000200249087888
:108210000221014A11707047AE00002070B50024A1
:1082200000211448FBF7A0FEFFF7CEFFFFF7CCFFBD
:1082300000251BE06006040E00210E48401EFBF7DF
:1082400093FEFFF7C1FFFFF7BFFFFFF7BDFF094830
:10825000FBF7DAFE044380210648401EFBF784FE4C
:10826000FFF7B2FFFFF7B0FF681CC5B2082DE1DBD6
:10827000204670BD0306000010B5022011490870A9
:1082800000211148FBF770FEFFF79EFFFFF79CFFF0
:1082900000210D48401EFBF767FEFFF795FFFFF733
:1082A00093FF80210848FBF75FFEFFF78DFFFFF784
:1082B0008BFF80210448401EFBF756FEFFF784FF2A
:1082C00010BD0000AE0000200306000010B5022023
:1082D0000D49087080210D48FBF746FEFFF774FF3B
:1082E000FFF772FF00210948401EFBF73DFEFFF734
:1082F0006BFFFFF769FF00210448FBF735FEFFF72E
:1083000063FFFFF761FF10BDAE0000200306000011
:1083100010B50446022012490870012C00D910BD86
:10832000002C04D000210F48FBF71EFE03E0802143
:108330000C48FBF719FEFFF747FF00210948401ED4
:10834000FBF712FEFFF740FFFFF73EFF80210548D5
:10835000401EFBF709FEFFF737FF00BFDFE7000015
:10836000AE0000200306000070B504460220244938
:108370000870002524E080202040002804D000213F
:108380002048FBF7F1FD03E080211E48FBF7ECFDE0
:10839000FFF71AFFFFF718FF00211A48401EFBF7EE
:1083A000E3FDFFF711FFFFF70FFF80211548401E87
:1083B000FBF7DAFDFFF708FF6006040E681CC5B284
:1083C000082DD8DB00210F48FBF7CEFDFFF7FCFEA0
:1083D000FFF7FAFE00210B48401EFBF7C5FDFFF733
:1083E000F3FEFFF7F1FE0748FBF70EFE04490870A5
:1083F00080210448401EFBF7B7FDFFF7E5FE70BD86
:10840000AE0000200306000010B5054800680028F3
:1084100002D003480068804700F088F810BD0000D3
:10842000D800002010B51A480078012811D018484B
:10843000007802280DD01748FBF722FE154908786E
:10844000FBF70AFB134908704878FBF705FB114955
:1084500048706420F6F7FCFDF2F70AFCFFF7ACFE6B
:10846000F5F732FDFBF7E2FEF6F7EEFB0A4800787F
:108470000A2807D3002008490870FAF75DFCFAF7CC
:1084800043FB04E004480078401C0349087010BD19
:108490009B000020A40000200401002010B50A2049
:1084A000FAF7B2FEF9F75EFFF4F7D0FE0A20F3F711
:1084B000A7F801F0DDFF0A20F6F7AEFF01F02EFB72
:1084C000F4F7E0FF10BD10B5F9F7B4F9F9F792F938
:1084D000F5F710FBF4F758FBF4F7CAFA10BD0000EB
:1084E00010B5F4F731F87D2109010648F3F7D8FCFF
:1084F00000F032FAF2F742F802210348F2F7C4FF23
:1085000010BD0000D0070020C407002010B5F2F70E
:1085100005FBFAF737FA01F0A9FDF7F7BBFAF9F70F
:1085200087F910BD10B5F6F711FD10BD10B532205A
:10853000F6F7D0FAF7F74AFB06480068401C0549F1
:10854000086008460068142803D300200860F0F78C
:10855000A3F810BD080100200CB500BF0548006855
:108560000090044800680190019900988842F5D174
:1085700000980CBD0001002000B589B00C480790A0
:108580000C4806900C4801900C4800900C4805904F
:108590000C4804900C4803900C4802900C4808903A
:1085A00000F002FC69460B4800F070F909B000BD0C
:1085B000E9C40000918D0100F38501001D860100D2
:1085C000018601002B8601000F860100398601001B
:1085D000D985010020C50100704710B5FBF758F898
:1085E000F5F7F6FC02F080F8F2F7A6FAFAF7DCF9F4
:1085F00010BD10B50120F0F7BBFE0446204610BDAB
:1086000010B50120F0F7A8FE0446204610BD10B5B5
:108610000120F0F7FFFC0446204610BD10B50020F5
:10862000F0F7A6FE0446204610BD10B50020F0F776
:1086300093FE0446204610BD10B50020F0F7EAFC7A
:108640000446204610BD000070B53148006831492D
:10865000096840182E490860084600687D21C90055
:10866000884211D32A480068EFF76AFD06467D214B
:10867000C90027480068EFF763FD254801602648D8
:108680000068801924490860244840682149096825
:1086900040182249486008460068002837D1002564
:1086A000084684682EE02068002829D01B496068AD
:1086B00049680022D243511A884205D2174960689E
:1086C00049684018606002E00020C0436060A16813
:1086D0006068884214D3206801280AD100202060F5
:1086E000002D03D10D492069886004E020692861CC
:1086F00001E000206060E068002801D0E068804769
:1087000025462469002CCED100200449486070BD64
:10871000FC000020F800002000010020BC18002010
:1087200010B5FBF74FFD322000F00AF80349322064
:10873000FBF720FD00F008F910BD0000498601009C
:1087400010B504460D48046000200D4908600D492D
:1087500008600D49086048608860FFF7FDFE0B491E
:1087600008600020486088600120C860032008611C
:10877000052048610720886110BD0000F800002036
:10878000FC00002000010020BC180020A0180020E0
:1087900070B5FFF722FFFFF7DFFE05463A48006895
:1087A000A84203D8384800682C1A06E0364800680A
:1087B0000021C943081A4019441C33480560406829
:1087C00000193149486008464068022806D3084627
:1087D0000079C007C00F4860FFF782FE2A48806812
:1087E00000192949886008468068052807D38868E9
:1087F0000521EFF7A5FC24488160FFF793FE22488E
:10880000C06800192049C8600846C0680A2807D314
:10881000C8680A21EFF794FC1B48C160FFF73EFED1
:1088200019480069001918490861084600691428A8
:1088300007D308691421EFF783FC13480161FFF7A0
:1088400042FE1148406900190F49486108464069D5
:10885000322807D348693221EFF772FC0A48416198
:10886000FFF754FE084880690019074988610846E7
:108870008069642807D388696421EFF761FC0248A6
:108880008161FFF7CFFD70BDA01800200288264B44
:108890001A8042885A8082889A80C288DA80028947
:1088A0001A8142895A8182899A81C289DA81028A2F
:1088B0001A82428A5A82828A1C4B1A80C28A1C4BB4
:1088C0001A80028B1B4B1A80428B5A80828B9A80B3
:1088D000C28BDA80028C1A81428C5A81828C9A81F6
:1088E000C28CDA81028D1A82428D5A82828D124B9D
:1088F0001A80C28D114B1A80114B0A681A604A689F
:108900005A608A689A60CA68DA600A691A614A69B4
:108910005A618A699A61CA69DA610A6A1A625522D9
:10892000084B1A70704700003607002032070020FD
:10893000340700204A0700202E07002030070020BF
:10894000181D00202D07002010B50024FBF776F835
:108950002046FAF789FE10BD10B500F035F900F099
:108960003FFB0448006A002802D00249086A804799
:1089700010BD0000181D002000B589B00C480790FC
:108980000C4806900C4801900C4800900C4805904B
:108990000C4804900C4803900C4802900C48089036
:1089A00000F096FA69460B48FFF770FF09B000BD6A
:1089B000E9C40000918D0100F38501001D860100CE
:1089C000018601002B8601000F8601003986010017
:1089D000D985010020C5010010B580201B494871D0
:1089E0001A201A49203908722B2048723C208872BC
:1089F0004D20C872002016494860F2F73BFC15492B
:108A000008600020C04314490860144908601448F5
:108A100014490860114903221202891848600F495D
:108A2000891888600D498918C8600C49891808613F
:108A30000A498918486109498918886107498918CC
:108A4000C861AC200849487010BD000020040240F5
:108A500000B00140B006002080E200E000E100E04C
:108A6000C0C0C0C000E400E0001002400146002089
:108A700007E04200054B9A5A8A4200DD03E0421C9F
:108A8000D0B20A28F5D300BF704700003607002097
:108A90000146002007E04200054B9A5A8A4200DD59
:108AA00003E0421CD0B20A28F5D300BF7047000093
:108AB0004A0700200148007A70470000F41C00209B
:108AC0000148007A70470000E81C0020FEB500272E
:108AD000002001900090009045E03648C0690028D1
:108AE00003D03448C1690220884732488068002892
:108AF00004D0304988688047044600E000242D48AF
:108B0000C068002804D02B49C8688047054600E0AB
:108B10000025AC4201DD264600E02E46264880882E
:108B2000B04203DA2448C089B04205DC002701982E
:108B3000401CC0B2019003E0781CC7B20020019035
:108B40000098401CC0B2009000980A2800D30EE0A4
:108B5000052F02D30520194908720198052802D370
:108B60000920164908721548007A0028B5D000BFC0
:108B70001248007A00281CD05520114908700D4871
:108B8000806900280AD00B49886980470D4908721E
:108B90000849886980470B49487203E00020094969
:108BA000087248720348006A002802D00149086A26
:108BB0008047FEBD181D00204A070020001D002030
:108BC0002C0700200C1D0020FEB56B488069002892
:108BD00020D06949886980476849497A884210D11C
:108BE0006648408866490988884205DA63484088B3
:108BF000401C6249488012E06048407A5F49087230
:108C00000DE000205D4948805B49886980475B49E9
:108C1000487204E00020594948800872487256485A
:108C20000068002803D054490868804701905248E2
:108C30004068002803D05049486880470090019858
:108C4000012857D100980128FBD14B4840690028E2
:108C500004D0494948698047064600E00026464856
:108C60000069002804D0444908698047074600E0AD
:108C70000027B74201DD3D4600E035464148007817
:108C800032280FD23F48406840193E4948600846A4
:108C90000078401C08700A4611785068EFF750FAC7
:108CA00085B211E0002037490870486008464068E6
:108CB0004019486008460078401C08700A46117840
:108CC0005068EFF73DFA85B22846FFF7CFFE04461D
:108CD0002C48417AA1423DD100202B4908802948E7
:108CE00040882A490988884205DA26484088401C7D
:108CF000244948803EE02348007A07280ED9092CF1
:108D000003D0082C01D0072C06D109201D49087278
:108D100000201A49087201E01A4804721948007AC2
:108D200001280CD1012C01D0022C06D101201549BB
:108D3000087200201149087201E0124804721148BB
:108D4000007A012816D00F48007A072812D80D485B
:108D500004720FE000200B4948800B480088401C3B
:108D60000949088008460088052803D300200880A8
:108D700004484472FEBD0000181D0020F41C0020B1
:108D800034070020E81C0020600700203207002084
:108D900010B500240120FBF737F9012801D1012487
:108DA00000E00024204610BD10B5002034490870B2
:108DB0003449087048804860087248723249087027
:108DC000488048600872487230490870488048609E
:108DD000087248722E4908704880486008724872CC
:108DE0002C48007855283ED07D20C0002A490880B4
:108DF00002202A4908807D20C000294908800220DD
:108E000028490880002028490880284848802848A8
:108E100088802848C880284808817D20C001488172
:108E2000264888812648C881264808820020C043F9
:108E300048820020244908801C4848801C488880BB
:108E40001C48C8801C4808817D20C00148811B48FF
:108E500088811B48C8811B4808820020C043488283
:108E600055200C4908701948C069002804D01748DB
:108E7000C169FF2005308847FFF728FE10BD0000BC
:108E80002C070020E81C0020F41C0020001D0020FE
:108E90000C1D00202D0700202E0700203007002089
:108EA0003207002034070020360700206419000034
:108EB000581B0000282300001C25000074400000FF
:108EC00044480000384A00004A070020181D0020CE
:108ED00010B500202F4908702F490870488048605D
:108EE000087248722D4908704880486008724872BC
:108EF0002B490870488048600872487229490870F8
:108F000048804860087248722748007855283ED04B
:108F10007D20C000254908800220254908807D2049
:108F2000C0002449088002202349088000202349EA
:108F3000088023484880234888802348C8802348E5
:108F400008817D20C0014881214888812148C8814D
:108F5000214808820020C043488200201F49088021
:108F600017484880174888801748C88017480881E4
:108F70007D20C0014881164888811648C88116485E
:108F800008820020C0434882552007490870FFF737
:108F90009DFD10BD2C070020E81C0020F41C0020C3
:108FA000001D00200C1D00202D0700202E07002092
:108FB0003007002032070020340700203607002049
:108FC00064190000581B0000282300001C25000025
:108FD0007440000044480000384A00004A0700205E
:108FE000FEB569488069002820D0674988698047B4
:108FF0006649497A884210D16448408864490988A2
:10900000884205DA61484088401C6049488012E087
:109010005E48407A5D4908720DE000205B49488057
:109020005949886980475949487204E000205749E6
:1090300008724872488054480068002804D0524999
:1090400008688047019001E0002001904E48406888
:10905000002804D04C4948688047009001E0002077
:1090600000900198012853D100980128FBD146486F
:109070004069002804D0444948698047064600E01A
:10908000002641484069002804D03F4908698047CC
:10909000074600E00027B74201DD3D4600E03546C7
:1090A0003C48007832280FD23A4840684019394984
:1090B000486008460078401C08700A4611785068DD
:1090C000EFF73EF885B211E00020324908704860A1
:1090D000084640684019486008460078401C0870FF
:1090E0000A4611785068EFF72BF885B22846FFF74B
:1090F000CFFC04462748417AA14234D14088264912
:109100000988884205DA23484088401C2149488064
:1091100039E00020214908801E48007A092809D139
:10912000092C01D0082C03D109201A49087201E04A
:10913000184804721748007A012809D1012C01D07F
:10914000022C03D101201349087201E01148047276
:109150001048007A012816D00E48007A092812D04B
:109160000C4804720FE000200A4948800B48008830
:10917000401C0A49088008460088052803D30020BF
:10918000088004484472FEBD181D00200C1D0020FC
:1091900030070020001D00202E0700205E07002061
:1091A000012803D14A1E0B4B1A8312E0022803D177
:1091B0004A1E084B5A830CE0042804D14A1E054B72
:1091C000E0331A8305E0082803D14A1E014BE0333F
:1091D0005A837047602A044008B50D49C97C009144
:1091E00000210B4AD174012806D11146C978042206
:1091F0001143074AD17003E00549C978044AD17088
:109200000349C97801221143014AD17008BD000009
:10921000602A044008B50948C0780421084307497A
:10922000C8700846C078FE2108400449C870084646
:10923000C07C00900020C87408BD0000602A044073
:10924000012803D14A1E0B4B1A8112E0022803D1D8
:109250004A1E084B5A810CE0042804D14A1E054BD3
:10926000C0339A8305E0082803D14A1E014BC0335E
:10927000DA837047802A044008B51049C978009104
:1092800000210E4AD170012808D10C492039C97833
:1092900008221143094A203AD17005E007492039D4
:1092A000C978064A203AD17004492039C978022287
:1092B0001143024A203AD17008BD0000802A0440C0
:1092C00008B50A48C078082108430849C87008460C
:1092D000C078FD2108400549C87004482030C07896
:1092E0000090002001492031C87008BD602A044068
:1092F0000648C078FE2108400449C8700846C07876
:10930000FD2108400149C87070470000602A0440F0
:1093100010B5044601211020F1F75AFF207800F023
:109320009FFB207800280CD1FE48C078FE21084021
:10933000FC49C8700846C07804210843F949C87040
:109340000FE0F848C0782278012191408843F54920
:10935000C8700846C0782278042191400843F1493A
:10936000C870A07805280AD1E078052807D0EE4813
:109370008068007840210843EB4989680870E078EC
:1093800000287DD1A07D2178490088400001E17C42
:1093900022785200914009010843E349096809789D
:1093A0000843E1490968087020788100DE484430AC
:1093B00040580078217B084321788A00DA494431FB
:1093C000895808703820005DA178084321788A0008
:1093D000D5491831895808706078C007C00F002837
:1093E0001DD020788100D048203040580078617B23
:1093F00004221143084321788A00CB49203189583F
:10940000087020788100C848443040580178A07B1B
:10941000014320788200C44844308058017060784D
:109420000221084002281ED120788100BE48203049
:1094300040580078E17B40221143084321788A009C
:10944000B94920318958087020788100B6484430E5
:1094500040580178207C4000014320788200B248C7
:10946000443080580170607804210840042820D1DD
:1094700020788100AC48283040580078E17B00E03B
:109480003BE00C221143084321788A00A649283189
:109490008958087020788100A348443040580178EA
:1094A000A07C80000143207882009F48443080588F
:1094B000017060780821084008281ED120788100BA
:1094C0009948283040580078E17BC0221143084376
:1094D00021788A00944928318958087020788100C1
:1094E0009148443040580178607DC00001432078A5
:1094F00082008D48443080580170E07801287DD189
:1095000089480068007888490968087020788100D7
:109510008548283040580078002120788200824811
:109520002830805801703820005DA17808432178E8
:109530008A007D491831895808707A48C07900201E
:109540007849C8716078C007C00F00281BD0207808
:1095500081007548203040580078E17D084321782B
:109560008A007149203189580870A088401E6E49D0
:10957000496D08806B48C07921788A0000219140AC
:1095800008436849C87160780221084002281DD14B
:10959000207881006448203040580078617E0901BD
:1095A0000843C1B2207882005F48203080580170A3
:1095B000E088401E5C49896D08805A48C07921784E
:1095C0008A000021914008435649C87160780421FF
:1095D000084004283BD12078810053482830405867
:1095E0000078E17E084321788A004F492831895864
:1095F00008702089401E4C49C96D00E05AE008807F
:109600004848C07921788A000021914008434549A3
:10961000C871607F01280CD1207881004248283031
:109620004058007821788A003F49283189580870CD
:109630000DE0207881003C4828304058007808210F
:10964000084321788A0038492831895808706078A1
:109650000821084008283CD1207881003248283071
:1096600040580078A17F09010843C1B220788200E8
:109670002D482830805801706089401E2A49096EA3
:1096800008802848C07921788A0000219140084349
:109690002449C8712020005D01280CD12078810068
:1096A000214828304058007821788A001E49283106
:1096B000895808700DE0207881001B4828304058F8
:1096C00000788021084321788A0017492831895879
:1096D0000870E078022802D0E07803287ED1124892
:1096E000006800781049096808703820005DA1788A
:1096F000084321788A000C49183189580870A088DD
:10970000401E0949496D08806078022108400228FE
:109710003CD16078217889008840034949680978FC
:10972000084303E0602A0440C8180020CA49496879
:109730000870E088401EC849896D08806078C04381
:10974000217889008840C449C96C09780840C24919
:10975000C96C087020788100BF48383040580178C3
:109760002420005D014320788200BB4838308058B7
:1097700001702320005D4000217889008840B649AF
:10978000496909780843B449496908706078042137
:10979000084004283AD16078217889008840AE4991
:1097A000496809780843AC49496808702089401E17
:1097B000A949C96D08806078C04321788900884034
:1097C000A549C96C09780840A349C96C087020787C
:1097D0008100A14838304058017800E05FE0262041
:1097E000005D40000143207882009B48383080585B
:1097F00001702520005D800021788900884096490D
:1098000049690978084394494969087060780821D2
:109810000840082838D160782178890088408E492E
:109820004968097808438C49496808706089401E76
:109830008949096E08806078C04321788900884092
:109840008549C96C097808408349C96C087020783B
:10985000810081483830405801782820005D800020
:109860000143207882007C483830805801702720DE
:10987000005DC000217889008840774949690978EE
:109880000843754949690870E078032807D1724890
:1098900080680078012108436F4989680870E07882
:1098A00004286ED10121F1F793FC6B480068007821
:1098B000E02108436849096808703820005DA178F4
:1098C000084321788A0064491831895808702B2090
:1098D000005DC0002A21095D890008433921095D26
:1098E00008435D498968097808435B4989680870BD
:1098F0003020005D80013221095D090108433421D7
:10990000095D890008433621095D084321788A00F2
:1099100051494431895809780843C1B220788200FE
:109920004D484430805801702C20005D4000217863
:109930000901884049490978084348490870607816
:10994000C007C00F00282DD0207800281AD1A08889
:10995000401E4149496D08803F48406D0188E08DB7
:109960000818401E3C49496D08803B48C06C00788F
:1099700021788A000121914008433749C96C087059
:1099800010E058E0A088401E3349496D08803248F5
:10999000C06C0178207882000120904081432E48DD
:1099A000C06C017060780221084002280FD1E08865
:1099B000401E2949896D08802748C06C00782178AD
:1099C0008A000221914088432349C96C087060785D
:1099D0000421084004280FD12089401E1E49C96D6A
:1099E00008801D48C06C007821788A0004219140CD
:1099F00088431949C96C0870607808210840082814
:109A00000FD16089401E1449096E08801248C06C4D
:109A1000007821788A000821914088430E49C96C5A
:109A200008702078002802D1E08D0C49C8820020FF
:109A30000A492031C88020788100074830304058DA
:109A400000783A21095D084321788A0002493031C3
:109A50008958087010BD0000C8180020602A044012
:109A6000002802D0012850D125E02949294A116057
:109A7000491C5160491C9160C91C5161C91D91610B
:109A8000491C1162491C9162891C1163491C916334
:109A9000891E1164491D5165891C91651C49F43169
:109AA000D165891C11661C4911651949C91CD1640D
:109AB000C91C51642AE01649164A1160491C5160BC
:109AC000491C9160C91C5161114A1C321149CA617B
:109AD000521C4A62521CCA62921C4A63521CCA63DC
:109AE000911E0C4A1164491D5165891C91650849F4
:109AF000F831D165891C1166074911650449C91CF3
:109B0000D1640A1D03498A6400E000BF00BF7047AA
:109B1000642A0440C8180020583C044010B511487D
:109B2000007801281DD1F2F709FD012819D10E484E
:109B30000078F92805D20C480078401C0A490870C2
:109B400002E000200849087008480078F92805DA82
:109B500006480078401C0549087002E000200349CF
:109B6000087010BDAC0000206300002062000020DF
:109B700038B515A0006800900024FEF79BFF01286F
:109B80001DD11248007801281CDAF6F725FA104991
